:020000040800F2
:1000000000000220A9340108799700087B970008B6
:100010007D9700087F970008819700080000000086
:1000200000000000000000000000000083970008AE
:10003000859700080000000087970008899700084E
:10004000ED340108ED340108ED340108ED34010808
:10005000ED340108ED340108ED340108ED340108F8
:10006000ED340108ED340108ED340108397A000857
:10007000ED340108ED340108ED340108ED340108D8
:10008000ED340108ED340108ED340108ED340108C8
:10009000ED340108ED340108ED340108C59900087C
:1000A000ED340108ED340108ED340108ED340108A8
:1000B00085990008ED340108ED340108ED3401089C
:1000C000ED340108ED340108ED340108ED34010888
:1000D000ED340108ED340108D99A0008ED34010827
:1000E000ED340108ED3401088D970008ED34010866
:1000F000ED340108ED340108ED340108ED34010858
:10010000ED340108ED340108ED340108ED34010847
:10011000ED340108ED340108ED340108ED34010837
:10012000ED340108ED340108ED340108ED34010827
:10013000ED340108ED340108ED340108ED34010817
:10014000ED340108ED340108ED340108BD970008D5
:10015000ED340108ED340108ED340108ED340108F7
:10016000ED340108ED340108ED340108ED340108E7
:10017000ED340108ED340108ED340108ED340108D7
:08018000ED340108ED34010823
:100188000CB9050800000020300C0020300C0020BD
:10019800D43C002008B5074B186809F073FA0EF034
:1001A80017F9054B054806221A70BDE8084001F00A
:1001B800D0BC00BF40260020CD250020A80F00207D
:1001C80008B5034801F0C5FC024B00221A7008BDAF
:1001D800FC170020CD25002008B5054B0122002082
:1001E8001A7005F0E9FE0348BDE8084001F0B1BC0B
:1001F800582C00206C1500202DE9F041144C2046A5
:1002080004F05DF800201349134A03F00FFE134968
:10021800134A0746002003F009FE1249124A06460F
:10022800002003F003FED22105463A4623460A2061
:1002380003F014FFD22132462346FA2003F00EFFC2
:100248005A20D2212A462346BDE8F04103F006BFD2
:10025800801300203EA50508C901000847A5050828
:10026800E10100084FA505089D01000808B5054BE8
:10027800012200201A7005F09FFE0348BDE80840DF
:1002880001F067BC582C00206C15002008B5034805
:1002980001F05FFC024B00221A7008BDFC17002019
:1002A800CD25002008B5054B07221A700EF090F8EE
:1002B8000348BDE8084001F04CBC00BFCD25002034
:1002C800801300202DE9F041144C204603F0F7FF7D
:1002D80000201349134A03F0A9FD1349134A07469E
:1002E800002003F0A3FD1249124A0646002003F03D
:1002F8009DFDD22105463A4623460A2003F0AEFE6C
:10030800D221324623465A2003F0A8FEAA20D22141
:100318002A462346BDE8F04103F0A0BEA80F0020FE
:100328003EA505089502000858A50508AD02000875
:1003380061A5050875020008014801F00ABC00BF64
:100348009411002010B5094C204603F0B8FF002096
:100358000749084A03F06AFDD221024623464FF4B2
:100368008270BDE8104003F079BE00BFB4160020CB
:100378006AA505084103000870B50C4C0C4D2068AF
:100388004FF6E076314603F095F82068294603F0E9
:100398003FF86068314603F08DF86068294603F03D
:1003A80037F8BDE8704004F0C3B900BF300C002036
:1003B80060AB050838B52B4CFFF7DEFF002005F0D1
:1003C800FBFD237A23B90A203221274A05F002FFD0
:1003D800637A23B90A206421244A05F0FBFE214CE4
:1003E800A37A23B90A209621214A05F0F3FEA37ABD
:1003F8001C4DFBB16B7AEBB12B7ADBB100232B726E
:100408006B72AB721B4B286801221A704FF6E071B1
:1004180003F050F82868184902F0FAFF686817498D
:1004280002F0F6FF0BF06BFC04F082F9144804F0BC
:10043800C3F90DE00B4C4FF47841206803F03AF80B
:100448002068104902F0E4FF60680F4902F0E0FFFD
:10045800FFF792FF00200BF015FC0C48BDE8384070
:1004680001F077BB300C002071A505087FA50508B1
:100478008EA50508CD2500209CA5050861AB0508BB
:1004880080969800B0A5050863AB0508FC17002006
:1004980008B500200BF0F6FB0248BDE8084001F063
:1004A80058BB00BFFC17002038B5FFF765FF0DF0FB
:1004B800A7FF3C213F220023DF2005F06DFE4FF40B
:1004C80080600EF0E1FC124C3E223C21DF2000232C
:1004D80005F062FE012323720E4B4FF6E075186893
:1004E80009F0D0F82068294602F0E4FF20680A499C
:1004F80002F08EFF6068294602F0DCFF6068074959
:1005080002F086FF04F014F9054B00221A7038BD7A
:10051800300C002040260020C2A50508D5A50508F6
:10052800CD25002038B5FFF727FF0DF069FF6E21B4
:100538003F220023DF2005F02FFE4FF486400EF007
:10054800A3FC124C3E226E21DF20002305F024FE7E
:10055800012363720E4B4FF6E075186809F092F8A4
:100568002068294602F0A6FF20680A4902F050FFD9
:100578006068294602F09EFF6068074902F048FF5C
:1005880004F0D6F8054B00221A7038BD300C002054
:1005980040260020E8A50508F9A50508CD25002076
:1005A80010B5FFF7E9FE0DF02BFFA0213F22002335
:1005B800DF2005F0F1FD4FF402400EF065FC114C10
:1005C8003E22A021DF20002305F0E6FD0123A372CF
:1005D8000D4B186809F056F820684FF6E07102F0E4
:1005E80069FF2068094902F013FF6068084902F0B2
:1005F8000FFF04F09DF864200BF004FA054B00226D
:100608001A7010BD300C0020402600200AA60508EC
:1006180061AB0508CD2500202DE9F74F3A4D3B4E3B
:100628000024284603F04BFE224623464FF6FF716E
:1006380037480094019402F001FF4FF6E078042750
:10064800F06041462246234632480097019402F062
:10065800F5FE23463060414622462F480097019414
:1006680002F0ECFE2D4970602D4A204603F0DEFBB7
:100678002C492D4A0746204603F0D8FB2B492C4A23
:100688008046204603F0D2FB2A492B4A8146204661
:1006980003F0CCFB29492A4A8346204603F0C6FBCF
:1006A80021468246F2682B46204603F0D7FC5A21A1
:1006B80032682B460A2003F0D1FC6E2172682B4663
:1006C8000A2003F0CBFC9B213A462B46FA2003F084
:1006D800C5FC692142462B46FA2003F0BFFC3721AE
:1006E8004A462B46FA2003F0B9FCC82152462B464D
:1006F800AA2003F0B3FCF020C8215A462B4603B0C9
:10070800BDE8F04F03F0AABC24140020300C0020F0
:100718001EA6050826A6050839A6050848A6050840
:10072800A905000850A605082D05000840A60508DB
:10073800B104000858A60508990400085FA6050832
:10074800BD03000838B50C4C4FF6E0752068294603
:1007580002F0B0FE2068094902F05AFE6068294696
:1007680002F0A8FE6068064902F052FE03F0E0FFBE
:10077800BDE8384003F0DCBF300C002026A6050891
:1007880066A6050870B52DED028B9FED248A88B00A
:100798000A26F0EE488A03E0B0EE608AF0EE418A5D
:1007A8000CF07BFD8DED000ACDED010A9DE80300FC
:1007B80004AB83E80300F0EE680AB0EE480A9DED4A
:1007C800041ADDED051A8DED028ACDED038A0CF0D1
:1007D80005FBCDED010A8DED000A9DE8030002AD91
:1007E80085E80300013E6C46DDED020A9DED031A23
:1007F800D2D19FED0B0A0CF047FD8DED000ACDED2F
:10080800010A9DE8030085E80300DDED030A9DED7C
:10081800020A08B0BDEC028B70BD00BF00000000EA
:10082800CDCCCC3D2DE9F74F564D574CDFF86491B0
:10083800DFF864814FF6E07005F092FB286811F04C
:1008480037FD064668680F4611F032FD3246CDE99D
:1008580000013B464946204616F0F0FB224600239D
:100868000520372105F0B6FC2869484F484E11F09D
:100878001FFD824668698B4611F01AFD5246CDE984
:1008880000015B463946204616F0D8FB2246002375
:100898000520692105F09EFC286B11F009FD8246B0
:1008A800686B8B4611F004FD5246CDE900015B46AA
:1008B8004146204616F0C2FB002305209B21224614
:1008C80005F088FC31462A6C204616F0B7FB224614
:1008D80000239B21A22005F07DFC4FF4FC6005F06D
:1008E8003FFBA86811F0E4FC8246E8688B4611F0EB
:1008F800DFFC5246CDE900015B464946204616F02A
:100908009DFB224605205021002305F063FCA869C1
:1009180011F0CEFC8246E8698B4611F0C9FC5246BC
:10092800CDE900015B463946204616F087FB224692
:1009380000230520822105F04DFCA86B11F0B8FCBE
:100948008246E86B8B4611F0B3FC5246CDE90001B4
:100958005B464146204616F071FB00230520B42172
:10096800224605F037FC31466A6C204616F066FBD5
:10097800A220B4212246002303B0BDE8F04F05F0C1
:1009880029BC00BF603A0020400C00208BA6050857
:10099800AEA6050879A605089DA6050808B5002095
:1009A80005F00AFB0A4B1B780B2B0BD8DFE803F08A
:1009B8000A0A0A0A0A0A08060A0A0A0A054802E08E
:1009C800054800E00548BDE8084001F0C2B800BF8E
:1009D800CD25002080130020A80F0020FC17002040
:1009E8002DE9F14F2D4C204603F069FC00202C49DD
:1009F8002C4A03F01BFA2C492C4A8146002003F0AC
:100A080015FA2B492B4A0746002003F00FFA2A490A
:100A18002A4A0646002003F009FA2949294A0546C8
:100A2800002003F003FA2849284A8046002003F0F2
:100A3800FDF92749274A8246002003F0F7F9D22119
:100A480083464A462346E62003F008FB28203A4618
:100A58002346014603F002FB46213246234628205E
:100A680003F0FCFA64212A462346282003F0F6FA0C
:100A7800822142462346282003F0F0FA52462346B4
:100A88002820A02103F0EAFA28205A46BE2123464E
:100A980001B0BDE8F04F03F0E1BA00BF6C150020CB
:100AA800B3A60508A5090008BCA605083514000862
:100AB800C7A6050811140008D1A60508ED130008FB
:100AC800DCA60508C9130008E7A60508A513000851
:100AD800F1A6050881130008023810B50A2800F2AB
:100AE8003484DFE810F00B000F00D0003A01250233
:100AF800BB01D002EA0232049903ED03BDE81040BD
:100B08000BF06AB900204FF6E0710BF0BBFA6420D5
:100B18004FF6E0710BF0B6FAC8204FF6E0710BF013
:100B2800B1FA4FF6FF7005F01BFA00237D20DC2197
:100B3800B14A05F04FFB4EF29C7005F011FAAF4B2D
:100B48001C78022C32D0052C6CD0012C40F0FD838F
:100B5800B4204FF4F0610BF095FA05202146A84A1D
:100B6800002305F037FB05205221A64A002305F093
:100B780031FBB621A44A0023052005F02BFB4FF4D6
:100B8800F06005F0EDF940F2131021469C4A00236D
:100B980005F020FB40F2131052219B4A002305F078
:100BA80019FB40F21310B621984A2CE0A0204FF40C
:100BB800F0610BF067FA05200121924A002305F045
:100BC80009FB05205221924A002305F003FBB621B8
:100BD8008D4A0023052005F0FDFA4FF4F06005F07A
:100BE800BFF940F213100121864A002305F0F2FAFA
:100BF80040F213105221844A002305F0EBFA854A8B
:100C080040F21310B621002305F0E4FA4EF29C706E
:100C180005F0A6F90520A2217F4A0023BDE810406F
:100C280005F0D8BA64204FF4F0610BF02BFA204697
:100C380001217A4A002305F0CDFAB621724A002331
:100C4800204605F0C7FA4FF4F06005F089F940F244
:100C580013100121714A002305F0BCFA40F2131069
:100C68005221694A002305F0B5FAB62140F2131063
:100C78006B4A002305F0AEFA4EF29C7005F070F94D
:100C880020465221C8E700204FF6E0710BF0FAF930
:100C980031204FF6E0710BF0F5F963204FF6E07163
:100CA8000BF0F0F995204FF6E0710BF0EBF9C72047
:100CB8004FF6E0710BF0E6F94EF29C7005F050F932
:100CC800052001210023574A05F084FA0520202138
:100CD8000023554A05F07EFA052052210023534A85
:100CE80005F078FA052084210023514A05F072FAAC
:100CF800B6210520444A002305F06CFA4FF4F06051
:100D080005F02EF9012140F213100023454A05F0A1
:100D180061FA40F213102021464A002305F05AFADE
:100D280040F213105221384A002305F053FA40F2DA
:100D380013108421404A002305F04CFAB6213F4A9B
:100D480040F21310002305F045FA4FF6FF7005F046
:100D580007F97D20DC213A4A5FE700204FF6E07171
:100D68000BF090F927204FF6E0710BF08BF94F202C
:100D78004FF6E0710BF086F977204FF6E0710BF033
:100D880081F99F204FF6E0710BF07CF9C7204FF6F0
:100D9800E0710BF077F94EF29C7005F0E1F8052050
:100DA80001210023184A05F015FA05201621002311
:100DB800244A05F00FFA05203E210023224A05F0B7
:100DC80009FA052066210023204A05F003FA8E213E
:100DD800002305201E4A05F0FDF905201D4AB6210D
:100DE800002305F0F7F94FF6FF7005F0B9F87D20FC
:100DF800DC21194A11E700BFC7A605081C0300201B
:100E0800F7A6050800A70508CBAC0508F6A605084F
:100E1800FBA60508FFA6050832A7050805A70508CB
:100E280004A705081EA7050809A7050819A70508A6
:100E38000EA7050813A7050818A705081DA7050884
:100E4800D1A6050821A7050825A7050829A705088B
:100E58002DA7050831A7050835A7050800204FF676
:100E6800E0710BF00FF931204FF6E0710BF00AF941
:100E780063204FF6E0710BF005F995204FF6E0710D
:100E88000BF000F9C7204FF6E0710BF0FBF84EF2BB
:100E98009C7005F065F8052001210023BF4A05F084
:100EA80099F9052020210023BD4A05F093F9052072
:100EB80052210023BB4A05F08DF905208421002327
:100EC800B94A05F087F9B6210520B84A002305F08C
:100ED80081F94FF4F06005F043F8012140F2131056
:100EE8000023B34A05F076F940F213102021B14AE5
:100EF800002305F06FF940F213105221AB4A00238A
:100F080005F068F940F213108421AB4A002305F07C
:100F180061F9B621A94A40F21310002305F05AF9E5
:100F28004FF6FF7005F01CF87D20DC21A44A74E61A
:100F3800A44B1C78022C32D0052C5DD0012C40F03B
:100F48008B8000204FF6E0710BF09CF834204FF6B0
:100F5800E0710BF097F864204FF6E0710BF092F80F
:100F68004FF6E07198200BF08DF84EF29C7004F06B
:100F7800F7FF05202146944A002305F02BF90520A8
:100F88002021924A002305F025F905205021904A96
:100F9800002305F01FF9052084218E4A59E000201E
:100FA8004FF6E0710BF06EF852204FF6E0710BF03F
:100FB80069F890204FF6E0710BF064F84FF6E07195
:100FC800B4200BF05FF84EF29C7004F0C9FF0520C6
:100FD8000121814A002305F0FDF805203E217C4AC5
:100FE800002305F0F7F805207C217A4A002305F054
:100FF800F1F80520A0212BE000204FF6E0710BF05E
:1010080041F82E204FF6E0710BF03CF87F204FF6A8
:10101800E0710BF037F84FF6E071AD200BF032F8C5
:101028004EF29C7004F09CFF204601216B4A00237D
:1010380005F0D0F820463221654A002305F0CAF8A9
:1010480020466B21634A002305F0C4F82046992105
:10105800634A002305F0BEF84FF4F06004F080FF07
:10106800604A00230520B62105F0B4F84FF4FC616E
:10107800C8200BF007F84FF6FF7004F071FF8720C7
:10108800DC21594AC9E500204FF6E0710AF0FAFF61
:1010980063204FF4FC610AF0F5FF4FF6E071C720BA
:1010A8000AF0F0FF4FF6FF7004F05AFF002005F039
:1010B80059F8A520D7214D4AAFE5042005F052F88C
:1010C80000204FF6E0710AF0DDFF31204FF6E071A5
:1010D8000AF0D8FF63204FF6E0710AF0D3FF95209D
:1010E8004FF6E0710AF0CEFFC7204FF6E0710AF024
:1010F800C9FF4EF29C7004F033FF05200121002344
:101108003B4A05F067F8052020210023314A05F005
:1011180061F8052052210023364A05F05BF80520C6
:1011280084210023344A05F055F80520B621334AB6
:10113800002305F04FF84FF6E07004F011FF40F27D
:101148000B1001212E4A002305F044F840F22B1021
:1011580020212C4A002305F03DF840F223105221AB
:10116800294A002305F036F840F21B108421274A4B
:10117800002305F02FF8B621254A002340F213106A
:1011880005F028F84FF6FF7004F0EAFE002004F09E
:10119800E9FF6E20D2211F4ACFE000BF41A7050812
:1011A80045A7050862A7050849A70508CBAC0508A7
:1011B80052A705084EA705084DA7050851A7050819
:1011C80056A705081C03002005A705082AA7050837
:1011D80022A7050871A7050832A7050826A705084C
:1011E80061A70508E2AD0508F1A6050879AB050871
:1011F80065A7050870A7050873A7050877A7050858
:101208007CA705081EA7050883A7050887A7050862
:101218008CA7050892A70508042004F0A3FF002066
:101228004FF6E0710AF02EFF27204FF6E0710AF022
:1012380029FF4F204FF6E0710AF024FF77204FF680
:10124800E0710AF01FFF9F204FF6E0710AF01AFFC5
:10125800C7204FF6E0710AF015FF4EF29C7004F0BB
:101268007FFE052001210023384A04F0B3FF052042
:1012780016210023364A04F0ADFF05203E21002345
:10128800344A04F0A7FF05206621334A002304F0FE
:10129800A1FF05208E21314A002304F09BFFB621CF
:1012A8002F4A0023052004F095FF4FF6FF7004F045
:1012B80057FE002004F056FF6420D221294A3CE062
:1012C800042004F04FFF00204FF6E0710AF0DAFE28
:1012D80043204FF6E0710AF0D5FE85204FF6E07105
:1012E8000AF0D0FE4FF6E071C7200AF0CBFE4EF2AE
:1012F8009C7004F035FE052001211B4A002304F0F0
:1013080069FF05204521194A002304F063FF0520E1
:101318008721134A002304F05DFFB621144A0023F5
:10132800052004F057FF4FF6FF7004F019FE002067
:1013380004F018FF0F4A7D20D221002304F04AFF51
:101348000420BDE8104004F00DBF10BD98A70508A3
:101358004EA7050853A705089DA70508A0A70508D7
:1013680032A70508A3A70508ACA7050805A705081F
:10137800CBAC05083FAC050810B5064C064806235B
:10138800237000F0E6FB2078FFF7A6FBBDE81040CD
:101398000DF04EBD582C00205817002010B5064CF3
:1013A80006480723237000F0D4FB2078FFF794FB4E
:1013B800BDE810400DF03CBD582C00205817002007
:1013C80010B5064C06480523237000F0C2FB2078B0
:1013D800FFF782FBBDE810400DF02ABD582C002015
:1013E8005817002010B5064C06480423237000F057
:1013F800B0FB2078FFF770FBBDE810400DF018BD7A
:10140800582C00205817002010B5064C0648032316
:10141800237000F09EFB2078FFF75EFBBDE81040CC
:101428000DF006BD582C00205817002010B5064CAA
:1014380006480223237000F08CFB2078FFF74CFB52
:10144800BDE810400DF0F4BC582C002058170020BF
:1014580038B5094C05464FF6E071206802F02AF8C5
:1014680020680DB1054900E0054901F0D1FFBDE84C
:10147800384003F05DB900BF5C0C0020B0A7050838
:10148800C3A70508194B10B51C78012C05D006D345
:10149800022C0CBF3024002402E0002400E01024B9
:1014A80004F1C80006F01AFB11490246114815F06C
:1014B800C5FD04F1CC0006F011FB0D4902460E48AB
:1014C80015F0BCFD04F1D00006F008FB08490246FF
:1014D8000A4815F0B3FD04F1D40006F0FFFA0449F8
:1014E80002460748BDE8104015F0A8BD1C0E0020B4
:1014F800AEA6050810260020342600204A2C00201D
:10150800FC25002010B5E82006F0E8FA0F4C02464A
:1015180021460F4815F092FDEC2006F0DFFA21462F
:1015280002460C4815F08AFDF02006F0D7FA21464D
:101538000246094815F082FDF42006F0CFFA02466B
:1015480006482146BDE8104015F078BDAEA605084E
:1015580010260020342600204A2C0020FC250020DC
:101568000E4A012310B513700D4A002414700D4A59
:10157800204613700AF086FB204604F01DFD0A4B36
:1015880003221A700AF0DCFE0BF021FC074B084816
:101598001C70BDE8104000F0DCBA00BF582C0020D9
:1015A800770D0020750D0020CD250020343800204F
:1015B8003812002038B50D4B0D4D00241C700D4B12
:1015C80028681C700C4B4FF6E0711C7001F072FF1C
:1015D80028680A4901F01CFF03F0AAF8204604F025
:1015E800EBFC0748BDE8384000F0B3BAD40D002042
:1015F8005C0C0020770D0020CD25002065AB050888
:10160800FC17002007B50E4B0E481A78D2F10102DC
:1016180038BF00221A700C4B05221A7000F099FA94
:10162800022201238DE80C00B02060211022322311
:101638000DF09CFD03B05DF804EB03F079B800BF32
:10164800D40D0020F0100020CD2500202E4A0023C4
:1016580010B513702D4A13700DF0E2F904460028F6
:1016680042D02B4C4FF6E071206801F023FF206830
:10167800284901F0CDFE60684FF6E07101F01AFFCD
:101688006068254901F0C4FEA0684FF6E07101F0DA
:1016980011FFA068214901F0BBFE03F049F84FF49F
:1016A8007A600AF0AFF920684FF6E07101F002FFA6
:1016B80020681B4901F0ACFE60684FF6E07101F04C
:1016C800F9FE6068164901F0A3FEA0684FF6E071C4
:1016D80001F0F0FEA068124901F09AFE03F028F824
:1016E800BDE8104003F024B80CF072FE204604F068
:1016F80063FC0C4B0C4804221A7000F02AFABDE86F
:101708001040FFF71FB800BFD40D0020770D002050
:101718005C0C0020D6A70508EAA70508FAA7050863
:1017280064AB0508CD250020241400202DE9F04FD6
:101738006A4DDFF8F4916A4E85B000244FF6FF78C1
:10174800284602F0BCFD41462246234665480094DF
:10175800019401F073FE0427039041462246234674
:1017680048460097019401F069FE414630602246E0
:10177800234648460097019401F060FE4146706098
:101788002246234648460097019401F057FEA8F5E3
:101798000048B060414622462346534800970194CA
:1017A80001F04CFE4146F060224623464F48009720
:1017B800019401F043FE41463061224623464C48DD
:1017C8000097019401F03AFE234670614146224693
:1017D80048480097019401F031FE4749B061474AF3
:1017E800204602F023FB4649464A8046204602F03E
:1017F8001DFB4549454A8246204602F017FB4449ED
:10180800444A0746204602F011FB4349434A8146B1
:10181800204602F00BFB4249424A8346204602F02A
:1018280005FB21468446039ACDF808C02B4620467E
:1018380002F014FC052132682B46A02002F00EFCB1
:10184800692172682B46782002F008FC7D21B26875
:101858002B46782002F002FC2821F2682B4605204E
:1018680002F0FCFB4B2132692B46052002F0F6FB07
:10187800052072696E212B4602F0F0FB9121B269B6
:101888002B46052002F0EAFBD2213A462B460520DA
:1018980002F0E4FBD22142462B46602002F0DEFB38
:1018A800D2214A462B46B02002F0D8FBD22152461C
:1018B8002B464FF4807002F0D1FBB4215A462B46D8
:1018C800052002F0CBFBDDF808C06020B421624699
:1018D8002B4605B0BDE8F04F02F0C0BBC81400208D
:1018E8005C0C00200AA8050814A805081BA8050810
:1018F80021A8050827A805082DA8050855160008D9
:1019080035A80508BD1500083DA805080D160008EE
:1019180046A80508691500084EA805080D15000811
:1019280057A805088D14000861AB0508654A00230F
:101938002DE9F04713700125634ADFF8BC81137065
:10194800A842014688F8005003D0022840F0B3802E
:101958003EE04FF4747006F0A8F80AF017FC5B4BF1
:101968005B4A1B68934209DD5A4A5B4912688A42FE
:1019780007DD5A498A4204DC022210E0B3F5FA5F17
:101988001ADB544A564912688A4201DC002206E0F2
:1019980054498B4210DD544B9A420DDC0122534BC3
:1019A80001201A7005F056FA0120FFF751FD4F4B40
:1019B8001978012901D107E0FEE702D302297AD17B
:1019C80002E04020002100E0402007F06BFA72E0BE
:1019D800C82006F083F80446CC2006F07FF80746B6
:1019E800D02006F07BF80646D42006F077F881462A
:1019F8000AF0CCFB354B37491A68A242184602DB7D
:101A08000B68BB4213DD3A4B04601E60394B0F6014
:101A1800C3F800900AF0F6F8374B01221A70374ADB
:101A28000520B4210023BDE8F04704F0D3BB94425D
:101A380018D19F4216D12E4B1B689E4212D12D4BB6
:101A48001B6899450ED14FF47470294688F80050E8
:101A580006F02BF82A4B00221A602A4B4FF07E52D0
:101A68001A6028E0244B02251D7029464FF4747033
:101A780006F01BF8154B1B6806EE906A1C1BF8EE67
:101A8800E67A06EE904AB8EEE67A1D4B87EE277A9C
:101A9800284683ED007A164B1B6806EE903AB8EE9E
:101AA800E67A184BC7EE277AC3ED007A05F0D2F92B
:101AB8000020FFF7CDFC0AF004FBBDE8F04702F078
:101AC80037BE00BFD40D0020770D00204C26002023
:101AD8005FE31600642C002080D1F0087F74D21ACE
:101AE8004FDA11001FA107007FD1F0081C0E00205B
:101AF800402C0020F8250020C901002060A8050816
:101B0800C82500200826002008B500F053FFFEF77E
:101B180073FB00F04FF800F06FF8FEF77DFDFEF75D
:101B2800D1FBFEF75DFF01F055FBFFF7FFFD01F06C
:101B380027F9FEF707FC01F049FA00F073FB00F003
:101B480087FD00F091FE00F065FABDE8084000F05E
:101B580033BB10B5044628B90F48104A104B53211F
:101B680003F00EF80F4B1868844213D010B1C36904
:101B780000219847002004F01FFA002004F006FA1C
:101B88004FF6FF7004F0ECF9E3692046012198470D
:101B9800044B1C6010BD00BF74A805082C2604085F
:101BA80090A80508780C00200048D2E7FC17002010
:101BB8000CF0F6BE10B5084C204602F080FB002061
:101BC8000649074A02F032F9D22102462346FA2092
:101BD800BDE8104002F042BA600E0020AEA8050829
:101BE800B91B0008024B034801221A70FFF7B1BF66
:101BF800CD250020C81400202DE9F743374D384F74
:101C0800384E0024284602F05AFB2246234647F65F
:101C1800FF7135480094019401F010FC4FF6FF78ED
:101C2800814641462246234638460094019401F0F5
:101C380005FC41463060224623463846009401940C
:101C480001F0FCFB4146706022462346384600946A
:101C5800019401F0F3FB2346B06041462246384622
:101C68000094019401F0EAFB2049F060204A2046E4
:101C780002F0DCF81F49204A0746204602F0D6F851
:101C8800214680464A462B46204602F0E7F93C2189
:101C980032682B46192002F0E1F95A2172682B4666
:101CA800192002F0DBF97821B2682B46192002F0DE
:101CB800D5F99621F2682B46192002F0CFF9D221E6
:101CC8003A462B46EC2002F0C9F99C20D221424624
:101CD8002B4603B0BDE8F04302F0C0B9381200202B
:101CE80061AB05087C0C0020A0A80508ADA8050874
:101CF800ED1B0008B6A80508C91E000870B5474EB8
:101D0800474C327847492DED028B142592B005FBDC
:101D180002420C320FA815F091F933780E2B05FB0F
:101D280003F504EB050332D8D3ED016A9B6807EE8F
:101D3800103A6359B8EEE68A06EE903ADFED3A7A41
:101D4800F8EEC78AB8EEE67A88EE278AC8EEA78A40
:101D5800C7EE277A17EE900A10F0AAFA02460B4649
:101D68006846324915F06AF918EE100A10F0A0FA20
:101D780002460B4605A82E4915F060F918EE900AA0
:101D880010F096FA02460B460AA82A4929E093ED74
:101D9800017A9B6807EE903A635906EE903AF8EE9E
:101DA800E78AF8EEE67AB8EEC78A17EE900A10F0DE
:101DB8007FFA02460B4668461F4915F03FF918EEB0
:101DC800100A10F075FA02460B4605A81B4915F0D3
:101DD80035F918EE900A10F06BFA0B4618490246CE
:101DE8000AA8184C15F02AF92068174901F010FBC9
:101DF80020680FA901F00CFB6068694601F008FB38
:101E0800A06805A901F004FBE0680AA901F000FB3D
:101E180002F08EFC12B0BDEC028B70BD462600208D
:101E280000000020BFA8050800007A44CAA80508D9
:101E3800DBA80508ECA80508FDA805080EA90508F3
:101E48001FA905087C0C00206AAB050808B5144BCF
:101E5800144A1B780D2B01D8012104E00E2B01D167
:101E6800022100E000211170142253430E49C85882
:101E7800CA184FF47A730D4958430860516892683C
:101E88004B430B490B600B4B1A6009F0BBFE0A4B26
:101E98000A4801221A70BDE80840FFF75ABE00BF81
:101EA800462600201C0E0020000000204C260020A2
:101EB800642C0020402C0020CD250020C8140020D0
:101EC800C4E700BF4FF6FF7070474FF6FF707047CA
:101ED8001FB5002947D04FF2DE7004F06DF80020DE
:101EE80004F040F90F2004F03BF81F4C1F4A412131
:101EF80001230A2004F06EF9042004F033F9236862
:101F080028209621042B24DC0123194A04F062F9C5
:101F180003A90DF10E02206804F0E2FB0F2004F083
:101F28001FF8BDF80C00BDF80E1014380F24282235
:101F3800002380B2009404F043F8BDF80E10BDF8F9
:101F48000C000094143989B22822012304F038F8CF
:101F580009E0084A012304F03DF91E20A521064A9C
:101F6800012304F037F91FBD8C0C002030A90508A7
:101F780043A905085FA9050875A9050837B51E4CCA
:101F88002368042B05462BDC01A80DF1060104F09B
:101F9800A5FBBDF80630BDF80420184904200DF053
:101FA8003BFA2368002B04DA1548164A164B5921C8
:101FB80005E0042B05DD1248124A144B5A2102F0A1
:101FC800DFFD04EB8302BDF8041001339180BDF8F6
:101FD80006102360052BD18008D1201D04F000FCD9
:101FE80000230B482360FFF7B4FD03E028460121D6
:101FF800FFF76EFF3EBD00BF8C0C00208CA90508C2
:10200800D1A905083E260408F3A905080AAA050867
:102018001016002037B50B4C204602F050F90A4B39
:102028000A49009300250120094A0A4B019501F04D
:10203800EEFF294602462346284603B0BDE8304055
:1020480002F00CB8DC120020D91E0008CD1E0008D2
:10205800D31E0008851F00084FF6FF7070474FF623
:10206800FF70704730B54FF6E07087B003F0A4FFFB
:10207800002004F077F80F2003F072FF00212C4AAB
:102088002C4C01230A2004F0A5F8002003F068FF77
:10209800042004F067F80A201921274A012304F0D4
:1020A80099F82521254A01230A2004F093F81F20D6
:1020B80003F056FF01230A203721214A04F08AF849
:1020C8002378002B31D001231E2096211D4A04F0CD
:1020D80081F862881C4902A814F0B0FF01231E2071
:1020E800A22102AA04F076F8A288184902A814F0DE
:1020F800A5FFAE2102AA01231E2004F06BF80F20D1
:1021080003F02EFF6088A188143880B20F2528229A
:102118000023009503F054FFA188608800951439C6
:1021280089B22822012303F04BFF07B030BD00BF5E
:1021380038AA0508A40C00204AAA05086AAA0508B6
:102148008AAA0508ADAA0508BFAA0508CCAA0508E9
:1021580001B187E7704713B50DF1060101A804F036
:1021680071FA144B01221A705988BDF80420891A93
:102178000E311C2919460AD89C88BDF80600201A79
:102188000E301C2803D899680131996001E00023BA
:102198008B60084B9968012905DD00229A601A7046
:1021A800FFF702FD05E05A80BDF806209A80FFF788
:1021B80059FF1CBDA40C002037B50B4C204602F07B
:1021C8007EF80A4B0A49009300250120094A0A4B68
:1021D800019501F01CFF294602462346284603B014
:1021E800BDE8304001F03ABF101600205921000820
:1021F80061200008672000085F21000808B5064B29
:1022080000221A70054B186814F0AEFB0448BDE8AC
:102218000840FFF79EBC00BFCD25002020360020D7
:10222800FC1700202DE9F04F514D524E85B0002487
:10223800284602F044F82246234647F6FF714E48E6
:102248000094019401F0FAF84FF6FF7703903946AD
:102258002246234649480094019401F0EFF8394694
:1022680030602246234646480094019401F0E6F87F
:102278004FF001087060224623464FF6E07141484E
:10228800CDF80080019401F0D9F82346B0603946B2
:1022980022463D48CDF80080019401F0CFF83B4933
:1022A800F0603B4A204601F0C1FD3A493A4A0746E8
:1022B800204601F0BBFD3949394A8046204601F0E5
:1022C800B5FD3849384A8146204601F0AFFD374907
:1022D800374A8246204601F0A9FD3649364A8346E8
:1022E800204601F0A3FD21468446039ACDF808C094
:1022F8002B46204601F0B2FE3C2132682B461420C2
:1023080001F0ACFE3C2172682B46EC2001F0A6FEE1
:10231800B421B2682B460F2001F0A0FED2213A4624
:102328002B46E62001F09AFE642142462B46052002
:1023380001F094FE4A462B460520872101F08EFEC7
:1023480052462B460520D22101F088FED2215A465A
:102358002B46502001F082FEDDF808C09B20D221D8
:1023680062462B4605B0BDE8F04F01F077BE00BFCE
:10237800040F0020B00C0020D9AA0508E3AA05081C
:102388005DA805085FAB050861AB0508ADA80508A1
:102398000522000840A60508ED23000850A60508F8
:1023A800ED240008ECAA0508F5250008F4AA05089C
:1023B800B1250008FCAA05086D25000808B50CF031
:1023C8001FF84FF441400CF05FFD044B186807F00C
:1023D80059F9034B09221A7008BD00BF4026002096
:1023E800CD25002010B50C4CFFF7E8FF0B4A002361
:1023F800B420052103F0EEFEA0684FF6E07101F06D
:1024080059F8A068064901F003F80BF0F9FFBDE898
:10241800104002F08DB900BFB00C002067AB050872
:1024280004AB0508264B2DE9F7431888C00014F0C3
:1024380093FA054628B90520B421224A2B4603F011
:10244800C9FE214BDFF878801D6000240BF0D8FF0F
:1024580026461E4FDFF8889023E009F005FA3B680E
:10246800D9F8000045F8083C7B6845F8043C184B4F
:102478001B68C01807F006F9164B186809F0C2FA6D
:10248800B8F8000094FBF0F080B24FF4FC630093BE
:1024980028210246322303F0EFFC04F59E7401362E
:1024A8000334B8F800300835B342D6DA0A4B186856
:1024B80007F0E8F8094B09221A70BDE8FE8300BF4F
:1024C8002C3A00201DAB050820360020EC370020F0
:1024D800C4250020F825002040260020CD25002016
:1024E8002836002010B5094CFFF79CFFA0684FF66E
:1024F800E07100F0DFFFA068054900F089FF0BF0EC
:102508007FFFBDE8104002F013B900BFB00C0020F7
:102518002BAB050810B5074C4FF6E071A06800F02A
:10252800C9FFA068044900F073FFBDE8104002F03D
:10253800FFB800BFB00C002045AB050810B5074C2C
:102548004FF6E071A06800F0B5FFA068044900F0FC
:102558005FFFBDE8104002F0EBB800BFB00C0020F0
:102568005BAB050810B50C4C0B2323700B4B0122F9
:102578001A70002002F0EEFF0948FFF7EAFA207807
:10258800FEF7AAFA074B032093ED000A0BF047FF6A
:10259800BDE81040D2E700BF582C00207A0D00207B
:1025A800581700202403002038B50C4D0C232B703D
:1025B8000B4B01241C70002002F0CCFF0948FFF7E8
:1025C800C8FA2878FEF788FA074B204693ED000AE8
:1025D8000BF025FFBDE83840B0E700BF582C0020BD
:1025E8007A0D0020581700202403002010B50C4C49
:1025F800092323700B4B01221A70002002F0AAFF56
:102608000948FFF7A6FA2078FEF766FA074B02207A
:1026180093ED000A0BF003FFBDE810408EE700BF02
:10262800582C00207A0D0020581700202403002081
:102638000CF07CBA034A044800231370034A137051
:10264800FFF787BA34380020FC170020CD2500207A
:102658002DE9F743384D394EDFF8FC800024284631
:1026680001F02DFE2246234647F6FF7134480094B8
:10267800019400F0E3FE4FF6FF7781463946224683
:10268800234630480094019400F0D8FE3946306063
:102698002246234640460094019400F0CFFE394676
:1026A80070602246234640460094019400F0C6FE1E
:1026B8002346B0603946224640460094019400F013
:1026C800BDFE2149F060214A204601F0AFFB2049B8
:1026D800204A0746204601F0A9FB214680464A4683
:1026E8002B46204601F0BAFC3C2132682B462820B4
:1026F80001F0B4FC5A2172682B46192001F0AEFC97
:102708007821B2682B46192001F0A8FC9621F268BE
:102718002B46192001F0A2FCD2213A462B46EC2088
:1027280001F09CFC0520D22142462B4603B0BDE8AF
:10273800F04301F093BC00BF4C100020C00C0020F7
:1027480075AB05087DAB0508ADA805083D26000852
:1027580088AB05083926000861AB050870B5064640
:1027680000200D46144603F0FDFC4FF6FF7003F001
:10277800F7FBF2B273208621002303F00DFDEAB2C5
:102788007320AE21002303F007FDE2B27320D621A7
:102798000023BDE8704003F0FFBC08B5084B2020BB
:1027A8001860084B1860084B58221A600146FFF75A
:1027B800D5FF0648064B1860BDE8084006F062BF22
:1027C800D8010020D4010020D0010020C0E1E4009D
:1027D800EC25002008B5094B20201860084B58212B
:1027E8001960084B02461860FFF7B8FF0648074B08
:1027F8001860BDE8084006F045BF00BFD8010020BA
:10280800D4010020D001002080969800EC250020FB
:1028180008B5094B58201860084B20211960084B4F
:102828000A461960FFF79AFF0648074B1860BDE88B
:10283800084006F027BF00BFD8010020D4010020BF
:10284800D0010020404B4C00EC250020034A0448EE
:1028580000231370034A1370FFF77BB93438002044
:10286800FC170020CD2500202DE9F74F444D454E9B
:10287800DFF83C810024284601F021FD224623464A
:1028880047F6FF7140480094019400F0D7FD4FF6D9
:10289800FF7783463946224623463C4800940194F4
:1028A80000F0CCFD3946306022462346404600946D
:1028B800019400F0C3FD3946706022462346404625
:1028C8000094019400F0BAFD2346B06039462246D0
:1028D80040460094019400F0B1FD2D49F0602D4A66
:1028E800204601F0A3FA2C492C4A0746204601F05D
:1028F8009DFA2B492B4A8046204601F097FA2A492F
:102908002A4A8146204601F091FA214682465A46D3
:102918002B46204601F0A2FB3C2132682B461920A9
:1029280001F09CFB5A2172682B46192001F096FB96
:102938007821B2682B46192001F090FB9621F268A5
:102948002B46192001F08AFBD2213A462B46EC206F
:1029580001F084FB822142462B46192001F07EFBC0
:10296800AA214A462B46192001F078FB1920524625
:10297800D2212B4603B0BDE8F04F01F06FBB00BF7A
:10298800A0180020D00C002090AB05089EAB0508CD
:10299800ADA8050855280008ABAB0508192800089C
:1029A800B4AB0508DD270008BDAB0508A327000860
:1029B80061AB050810B50B4C204601F080FC0020E7
:1029C8000146224600F09AFD00200749074A01F017
:1029D8002DFAD221024623464FF48270BDE81040FA
:1029E80001F03CBB58170020C6AB05081D2A00089B
:1029F80070B5C9240AE0A8B200223146013502F0B8
:102A08004BFCF02DF7D10134EF2C02D00025A6B2F3
:102A1800F1E770BD10B51A4C2378092B08D1194A73
:102A280000231370184A1370FFF7E2FF174823E0DA
:102A38000A2B0ED1164B186813F096FF154A00237F
:102A48001370114A1370144A1370FFF7D1FF13481B
:102A580012E0002002F07EFD114A00231360114AA3
:102A680013800D4B02221A700F4B186806F00AFEED
:102A780022780E4B0E481A70BDE81040FFF769B86F
:102A8800CD2500207A0D0020770D0020040F0020AE
:102A9800203600207B0D0020343800204C10002008
:102AA800C40D0020D20D002040260020EA25002079
:102AB80094110020034B01224FF4FC601A7003F0BC
:102AC8004FBA00BF770D0020044B054800221A704A
:102AD800044B0C221A70FFF73CB800BF770D00209A
:102AE800A0180020CD25002007B50A4A002313703E
:102AF80004228DE80C00C6201022232356210CF056
:102B080035FB054B05480A221A7003B05DF804EB43
:102B1800FFF71FB8770D0020CD2500204C100020AE
:102B280007B50A4A0023137004228DE80C00972089
:102B38001022232356210CF019FB054B05480922C6
:102B48001A7003B05DF804EBFFF703B8770D0020A7
:102B5800CD250020040F002007B50B4B00221A706A
:102B6800082203238DE80C004920102223233D214D
:102B78000CF0FCFA054B064801221A7003B05DF808
:102B880004EBFEF7E6BF00BF770D0020CD2500203F
:102B9800C814002008B50D4B002018700C4B187095
:102BA8000C4B18700C4B08221A700C4B187003F061
:102BB80003FA0B4B012119704FF080400EF027FCEF
:102BC8000848BDE80840FEF7C4BF00BFF125002053
:102BD800D40D0020770D0020CD250020582C002092
:102BE80038360020600E002070B51F4C1F4E20683C
:102BF8004FF6E075294600F05DFC20681C4900F09E
:102C080007FC6068294600F055FC6068194900F027
:102C1800FFFBA068294600F04DFCA068164900F0AB
:102C2800F7FB01F085FD4FF47A6008F0EBFE2068B1
:102C3800294600F03FFC2068314600F0E9FB606857
:102C4800294600F037FC6068314600F0E1FBA068D7
:102C5800294600F02FFCA068314600F0D9FBBDE8FA
:102C6800704001F065BD00BFE00C002064AB0508B2
:102C7800D6A70508EAA70508FAA705080C4B10B55A
:102C880000241C700B4B01221A70204608F0FAFF32
:102C9800204603F091F9084B0B221A7009F050FBFB
:102CA8000AF095F80548BDE81040FEF752BF00BF8E
:102CB800770D0020582C0020CD2500206C15002011
:102CC8000F4A002310B513700E4A13700BF0A8FEBC
:102CD800044628B1FFF788FFBDE8104001F028BD81
:102CE80003F06AF909F052FA074B1C70074B0722E8
:102CF8001A7009F045FA0648BDE81040FEF729BFEA
:102D0800D40D0020770D0020582C0020CD25002060
:102D180080130020144A002310B51370134A13704F
:102D2800134A13700BF07CFE28B1FFF75DFFBDE876
:102D3800104001F0FDBC03F03FF90E4B01241C705C
:102D480009F024FA06F00CFD0B4B06221A7009F064
:102D580017FA4FF0804021460EF059FB0748BDE8AE
:102D68001040FEF7F6BE00BFF1250020D40D00206C
:102D7800770D002038360020CD250020A80F002030
:102D88002DE9F04F6D4DDFF810928BB000244FF60F
:102D9800FF78284601F093FA4146224623466848C0
:102DA8000094019400F04AFB4FF6E0760427049063
:102DB80031462246234663480097019400F03EFBC3
:102DC80031460590224623465F480097019400F05B
:102DD80035FB414606902246234648460097019413
:102DE80000F02CFB594E41463060224623464846A7
:102DF8000097019400F022FB23467060414622466A
:102E080048460097019400F019FB5149B060514AB7
:102E1800204601F00BF85049504A0746204601F079
:102E280005F84F494F4A8046204600F0FFFF4E49BB
:102E38004E4A8146204600F0F9FF4D494D4A8246E8
:102E4800204600F0F3FF4C494C4A8346204600F0E8
:102E5800EDFF4B494B4A84462046CDF80CC000F0A4
:102E6800E5FF49490790494A204600F0DFFF4849F5
:102E78000890484A204600F0D9FF21460990049A54
:102E88002B46204601F0EAF82146059A2B46C82031
:102E980001F0E4F80A21069A2B46C82001F0DEF872
:102EA800552132682B46782001F0D8F869217268DC
:102EB8002B46782001F0D2F87D21B2682B46782085
:102EC80001F0CCF805203A4628212B4601F0C6F837
:102ED800D22142462B46052001F0C0F8D2214A46AD
:102EE8002B46562001F0BAF8D22152462B46A6208E
:102EF80001F0B4F8B4215A462B46052001F0AEF88B
:102F0800DDF80CC0B42162462B46562001F0A6F825
:102F1800B421079A2B46A62001F0A0F8B421089AFC
:102F28002B46F62001F09AF8099AF620D2212B4672
:102F38000BB0BDE8F04F01F091B800BFFC170020BE
:102F4800CBAB0508D4AB0508E1AB0508E00C0020C5
:102F5800ECAB0508612B0008F4AB0508852C0008CC
:102F6800FDAB05081D2D000806AC0508C92C000896
:102F78000FAC05089D2B000818AC0508292B000884
:102F880021AC0508F12A00082AAC0508D12A000856
:102F980032AC0508BD2A000861AB050807B5032354
:102FA80008228DE80C004920102223233D210CF033
:102FB800DDF8044B044801221A7003B05DF804EBF5
:102FC800FEF7C7BDCD250020C81400202DE9F74322
:102FD800314E324F324D0024304601F070F922460E
:102FE800234647F6FF712F480094019400F026FA13
:102FF8004FF6FF78814641462246234638460094DC
:10300800019400F01BFA41462860224623463846C0
:103018000094019400F012FA414668602246234663
:1030280038460094019400F009FA2346A860414606
:10303800224638460094019400F000FA1A49E860E4
:103048001A4A204600F0F2FE214607464A46334611
:10305800204601F003F83C212A683346192000F085
:10306800FDFF5A216A683346192000F0F7FF7821DE
:10307800AA683346192000F0F1FF9621EA68334622
:10308800192000F0EBFFEC20D2213A46334603B07A
:10309800BDE8F04300F0E2BFF010002061AB050886
:1030A800EC0C00203AAC0508ADA80508A52F0008CF
:1030B8001C4B1A781C4B10B51A7009F047F91B4BBA
:1030C8001B4A00241C6002202346CA2103F082F810
:1030D800204608F0D7FD174B1C80174B1C70174B68
:1030E8001B78023B052B1CD8DFE803F003070B1302
:1030F800170FBDE81040FEF799B9BDE81040FEF77C
:1031080083B9BDE81040FEF76DB9BDE81040FEF781
:1031180045B9BDE81040FEF753B9BDE81040FEF7C9
:103128002BB910BDEA250020CD250020C40D0020B4
:1031380060AB05083436002034380020582C0020B5
:1031480008B5084B186806F09DFA002002F034FF15
:1031580009F0F6F8044B05480B221A70BDE8084040
:10316800FEF7F7BC40260020CD2500206C15002076
:10317800114B10B500241C70104B186806F082FA29
:10318800204602F019FF0E4B1B780B2B0ED8DFE8F8
:1031980003F006060D0D0D0D0A080D0D0D06094864
:1031A80002E0094800E00948FEF7D3FC084B1C7010
:1031B800BDE8104009F0C4B8582C00204026002073
:1031C800CD250020FC17002080130020A80F002028
:1031D800343800202DE9F041144C204601F06FF8F6
:1031E80000201349134A00F021FE1349134A0746E9
:1031F800002000F01BFE1249124A0646002000F08B
:1032080015FED22105463A462346E62000F026FF61
:103218004B2132462346642000F020FF64206921B8
:103228002A462346BDE8F04100F018BF941100205B
:10323800B3A605087931000842AC050849310008F1
:103248004EAC0508B930000808B508B143682BB979
:103258000348044A044B9B2101F092FC586908BDBD
:103268005BAC0508502604087DAC050808B5FFF7D7
:10327800EBFF8068123080B208BD08B5FFF7E4FFA5
:103288004068063080B208BD2DE9F84F04468846EC
:10329800FFF7DAFF6689E589074606F1030905F1B4
:1032A8000F0AB8F1000F1FD01F2002F059FE204668
:1032B800FFF7DCFF83462046FFF7DFFF294603467A
:1032C8005FFA8BF2F0B202F08BFE042002F04AFFA4
:1032D8000B364FF6FF70033502F042FEB0B2A9B2CA
:1032E8003A68012302F076FF3D69204641464A4686
:1032F8005346A847BDE8F88F13B504460DF10601FB
:1033080001A803F09FF92046FFF79EFF6389BDF8E7
:103318000410BDF80620C91AE389D21A0339C36814
:103328000F3A204698471CBDF7B5044614200D46B1
:1033380016461F4613F010FB089BC7600361064B37
:103348000649074A80E8700000930190054B002069
:1033580000F05DFEFEBD00BF913200088332000818
:103368007532000801330008704708B508B1436892
:103378002BB90448044A054BAD2101F001FC5869FA
:1033880008BD00BF9CAC0508682604087DAC05088C
:10339800F8B505460E46FFF7E8FF836B04461BB1F8
:1033A80028463146984700E018466F8994F83C3023
:1033B800ED890EB9034310D0208E02F0D1FD608E46
:1033C80002F0E4FD94F8350002F0CCFE94F83430B5
:1033D80038462946224602F0FDFE002384F83C3098
:1033E800F8BD08B5FFF7C1FF90F83500BDE8084003
:1033F80002F0CDBE38B5FFF7B8FF044613F0A4FEBF
:10340800054694F8350002F0BDFE684380B238BD29
:1034180038B50D46FFF7A9FF29462E22044613F0BA
:10342800C3FE50B1204629462E2213F00FFF002379
:1034380084F82E30012384F83C3038BD2DE9F74359
:10344800074640200E461546984613F085FA04466E
:1034580028B91148114A124B4E2101F091FB114B2A
:10346800114A12498DE818000020114B00F0CFFDD9
:1034780039468146FFF7CCFF9DF82830268684F828
:1034880035300B9B6586A363002384F8348084F869
:103498003C304846BDE8FE839CAC050880260408FD
:1034A800BAAC050899330008EB330008FD3300086F
:1034B8007133000810B50C46FFF757FF0123048647
:1034C80080F83C3010BD00BF4FF4A0707047C82092
:1034D80070477047074B1B78022B07B508D1064B7E
:1034E8001B78022B04D001A80DF1060103F0AAF8FD
:1034F8000EBD00BF34380020582C002073B50A4B8D
:1035080006460D461446009300200849084A094B10
:10351800019000F07CFD294602462346304602B061
:10352800BDE8704000F09ABDDB340008D1340008D3
:10353800D7340008DD34000813B502AB03E90600F0
:10354800436843B1027C0124082A9C7004D11B699A
:103558002146984700E01C4620461CBD30B500288F
:103568002BD0058B002425E0036A1A7C012A05D19B
:103578005B681A888A421BD1187F30BD052A06D19C
:103588005B681A888A4213D193F82C0030BD032A4D
:1035980006D15B681A888A420AD193F8250030BDA3
:1035A800062A05D15B681A888A4201D1D87A30BDCB
:1035B80001340430AC42D7D3002030BD08B1817546
:1035C80001207047F8B504460D46D0B1E175D0F832
:1035D80098309847012D0DD12746002606E0F86956
:1035E80000F10802436906CA98470136238B04375D
:1035F8009E42F4D3D4F898302046294698470120B3
:10360800F8BDF8BDF8B50546084617460E4613F04E
:103618009BFD013FB84234BF04463C463CB12846B6
:103628003146224613F012FE00232B55F8BD2C70AC
:10363800F8BDF7B5044600200090019000296CD031
:103648000E8B68E000F1080351F823301D7C042D2F
:1036580004D15D682D88954247D0013000F10803F8
:1036680051F823301D7C012D04D15D682D889542C9
:103678003BD0013000F1080351F823301D7C052DA3
:1036880004D15D682D8895422FD0013000F10803E0
:1036980051F823301D7C032D04D15D682D88954297
:1036A80023D0013000F1080351F823301D7C022D8E
:1036B80004D15D682D88954217D0013000F10803C8
:1036C80051F823301D7C072D04D15D682D8A954261
:1036D8000BD0013000F1080351F823301D7C062D72
:1036E80008D15D682D88954203D103F10801204671
:1036F80015E0013000F1080351F823502B7C082B0A
:1037080009D16F683F88974204D105F10801204626
:103718001A4605E00130B04294D320466946082293
:1037280013F0CAFB2046FEBDF8B505460F461646FF
:10373800002830D04388032B2FD0202013F00CF919
:10374800044600282BD040F80C5B39460C22FFF7C2
:1037580059FF1820E66113F0FFF80646B8B10223B6
:103768000374012363760F4B446063600E4BA360C0
:10377800002323766B8805EB830201339BB2012B70
:1037880050606B800CD16A685268137608E0204656
:1037980013F0EAF804E0064602E0002600E00646D8
:1037A8003046F8BDCCA504086AA2040837B54568B8
:1037B80002AB03E906003DB3037C0124042B85F822
:1037C800314022D1688E02F0CBFB95F8300002F030
:1037D800C9FC95F8343043B9BDF80200BDF80610AD
:1037E800AA1C234602F0F6FC0FE0012B03D108487F
:1037F80040F2395104E0022B07D1054840F241510B
:10380800044A054B01F0BCF92C4620463EBD00BFDA
:10381800CDAC050840710408CBAC0508F8B50446E2
:103828000F46164610B3838A0A2B20D0202013F0A7
:1038380093F80546E8B14460102200F108003946C3
:10384800FFF7E0FE4FF6FF73A08A2B801F236B80E3
:1038580000232B76831D013080B20128EE6144F8E5
:103868002350A08207D1A3691876F8BDF8BD0020BF
:10387800F8BD0120F8BD0120F8BD2DE9F3471D462C
:103888004B1C984282460C461746BDF828600DDD51
:1038980095420BDC01320AF101035B1A521BC8B2D4
:1038A800D2B29BB22946009602F092FBAAF1020A14
:1038B8003046C4EB0A0A02F053FB4FF000084FF001
:1038C80001091FFA8AFA0BE0601C08EB050180B2B7
:1038D80089B252460023009602F072FB09F10109F1
:1038E8007B1B08F1010899451FFA88F8ECD3BDE85D
:1038F800FC87F8B5C7B2144638461E460D4602F096
:1039080071FB621E92B23846294602F06BFB3046C4
:1039180002F026FB022606E0A21B92B23846294690
:1039280002F060FB0136A642F6D3F8BD73B5044633
:103938000E4600F11E001546009200233C2280B27C
:103948001E3E02F03DFBB1B220463C220123009509
:1039580002F036FB7CBD73B504460E4601381546A9
:1039680000920023032280B2013E02F029FBB1B28B
:10397800204603220123009502F022FB7CBDF7B507
:10398800089D2E7BEF7A1C463604AB7A06EB072699
:10399800F618431A687B06EB00602D18002001908A
:1039A800121B08462146009501F002FFFEBD30B506
:1039B800456885B004AB03E906007DB101242C738A
:1039C8006D68BDF80800BDF80A109DF80C209DF838
:1039D8000E300095FFF7D3FF204600E0284605B0DB
:1039E80030BD2DE9F04385B004AB03E90600446817
:1039F800BDF80860BDF80C70002C41D0012384F894
:103A0800263094F825300BB9A26800E06268FFB24E
:103A1800BDF80A109DF80E30009230463A46FFF77E
:103A2800AEFF04F10C08022002F09CFB404613F0A4
:103A38008BFB054600B1451E0F3F0024153E1FFABB
:103A480087F90DE002F098FB02F09CFB04FB106183
:103A580089B248462022002302F0D6FB0134E4B2A2
:103A6800AC42EFD3002002F07BFAB8B2B1B24246C2
:103A7800012302F0C9FB002002F074FB012000E0E2
:103A8800204605B0BDE8F0832DE9F04385B004ABCE
:103A980003E906004568BDF80860BDF80C70002D04
:103AA8003CD001236B762B7EBDF80A10012B0CBF8E
:103AB8006A68AA689DF80E300092FFB23A4630460E
:103AC800FFF75DFF0C35022002F04CFB284613F08F
:103AD8003BFB0E3F81460024163E1FFA87F80DE097
:103AE80002F04AFB02F04EFB04FB106189B240462B
:103AF8002022002302F088FB0134E4B24C45EFD9C0
:103B0800002002F02DFAB8B2B1B22A46012302F021
:103B18007BFB002002F026FB012000E0284605B0D0
:103B2800BDE8F0832DE9F04F85B00546DDF84090FB
:103B3800029148469046039313F006FBDDF838A03F
:103B4800DDF83CB00646294600242F4611E024B192
:103B5800B4420CBF5B46534600E0039B01F10805E5
:103B6800ADB200932846029A4346FFF708FF013496
:103B78002946B442EBDD002002F0F2F9022002F0FF
:103B8800F1FA7D1D08F10508A8B21FFA88F14A4626
:103B9800012305B0BDE8F04F02F01CBB70B54068CA
:103BA80086B006AB03E9060000282ED0012380F872
:103BB8002D308668164BF21A534243EB020390F8F5
:103BC8002C205AB1002B134D134B144A08BF1D4625
:103BD800134B00F11C0418BF13460AE0002B0D4DCF
:103BE8000D4B0E4A18BF1D460D4B00F10C0408BFC3
:103BF8001346BDF81200BDF81410BDF81620009643
:103C080001950294FFF78EFF012006B070BD00BF3A
:103C1800B07A0408EC760408927C0408CE7804088C
:103C2800747E040870B5446886B006AB03E90600E4
:103C380004B301236377A668104B227FF11A4B4225
:103C480043EB01030AB10BB904E01BB966680C4DDC
:103C58000C4B01E00C4D0D4BBDF81200BDF81410D3
:103C6800BDF8162000960C3401950294FFF75AFF10
:103C7800012000E0204606B070BD00BFFC850408A6
:103C8800388204081A840408D2870408A88904081A
:103C98002DE9F04385B004AB03E906004468BDF89C
:103CA8000860BDF80A90BDF80C50BDF80E80002CD5
:103CB80000F08C800123A3740220676802F052FA96
:103CC8004FF6FF7002F062F9002002F049F9EDB2F8
:103CD8005FFA88F8A6F1160189B230462A464346AB
:103CE8000097FFF74CFE277A002F2ED1A28A234691
:103CF80000E00137974204D29969097E043300290C
:103D0800F7D002F039FA02F03DFAA9F116091FFAC4
:103D180089F90E2101FB10914FF6FF7208F1010895
:103D28005FFA88F389B2009248462A46FFF7A5FD54
:103D3800022002F017FA1F2002F012F9A38A002BC2
:103D480038D0103DE8B2303E2CE0E3685C68A28AC7
:103D58002346013A002700E00137974204D29969C7
:103D6800097E04330029F7D002F006FA02F00AFAB5
:103D78000E2101FB10914FF6FF7208F101085FFA5E
:103D880088F389B2009248462A46FFF776FD02205A
:103D980002F0E8F91F2002F0E3F8A38A53B1103DBE
:103DA800E8B21A3E0637B1B254F827200123083288
:103DB80002F02AFA002002F0D5F94FF6FF7002F05F
:103DC800E5F81F2002F0CCF8012000E0204605B0FD
:103DD800BDE8F0832DE9F0410546362088461446B3
:103DE8001F4612F0B9FD0646E0B120F8025B4146D5
:103DF8002E22FFF707FCBDF8183086F8344073868A
:103E08001820012386F8307086F8313012F0A4FDAE
:103E1800044618B104234660037404E0304612F0E7
:103E2800A3FD00E004462046BDE8F081F8B506464B
:103E380024200F46154612F08FFD0446D8B10F4BCB
:103E4800068083600E4B39464360102200F10C0057
:103E5800FFF7D8FB01260023182025622377667711
:103E680012F07AFD054610B14460067404E020465D
:103E780012F07AFD00E005462846F8BDFC850408E6
:103E880056800408F8B506462C200F46154612F051
:103E980063FD0446E8B120F80C6B39461922FFF798
:103EA800B1FB0D4BA562A3600C4B6360002384F843
:103EB80025301820012384F8263012F04DFD0546E0
:103EC80018B103234460037404E0204612F04CFD4B
:103ED80000E005462846F8BD089F0408A69B04088C
:103EE80010B50446142012F037FD20B1002343809A
:103EF800014B0480036110BD3137000838B5054611
:103F0800442012F029FD0446C0B10E4B05824360DF
:103F18000D4B0360012383740023037283820B4BD0
:103F28000364182012F018FD054618B107234460F1
:103F3800037404E0204612F017FD00E00546284609
:103F480038BD00BF9C9704089293040825380008E0
:103F58002DE9F04105463420884614461F4612F0E4
:103F6800FBFC064620B3144B05808360134B414687
:103F78004360102200F10C00FFF744FB214606F1D4
:103F88001C001022FFF73EFB002386F82C30182077
:103F98000123376386F82D3012F0DEFC044618B191
:103FA80005234660037404E0304612F0DDFC00E0AF
:103FB80004462046BDE8F081B07A04080A75040872
:103FC8002DE9F041044614200D461646984612F095
:103FD800C3FC0746B8B1069B048003610023C37283
:103FE80001234560068180F80A800373182012F0C7
:103FF800B3FC044618B106234760037404E038464E
:1040080012F0B2FC00E004462046BDE8F0812DE93C
:10401800F041044618200D461646984612F09CFCBE
:104028000746B8B101238370069B04800361079B90
:1040380045608660C0F80C804361182012F08CFC43
:10404800044618B108234760037404E0384612F0A8
:104058008BFC00E004462046BDE8F0812DE9F341E1
:1040680098461B8B1D2B05460C4617464FF0000043
:1040780000F2B480B5F5A07F0090019000F2AE8008
:10408800F02900F2AB80127CADF80610511EADF895
:104098000250072900F28A80DFE801F045595E04E2
:1040A800456A14767B684E4A7A611A8893F83430E8
:1040B8003A80013BDBB2012B7FD8ADF80240ADF866
:1040C80006507AE005F11602ADF8002004F1160258
:1040D800ADF8042002AE434A16E903007A6107F1FD
:1040E800080282E8030003F10802013348F822704D
:1040F800A8F818307B681A8A187A3A8000286CD198
:10410800FFF7FCFE3849436859603849DF600126EB
:10411800163D196002461E72A8B2E1B24346FFF787
:104128009DFF30465AE0012A0CBF314B314B78686D
:104138007B6130F80C3B3B8013F006F8431CDB0036
:104148001A34ED18ADF80440ADF8005035E07B683E
:10415800294A1B687A6102E0284A7B687A611B88D1
:1041680014353B80ADF800501434ADF8044024E019
:104178007B68234A7A611A883A801A899B7AAD1833
:10418800ADF80050E418F0E77E681E4B7B61338879
:1041980038463B8073689847013D4519ADF8005093
:1041A800B36838469847013C0419DEE71648174AB1
:1041B800174B40F21A3100F0E3FC02AA12E903009F
:1041C80007F1080383E80300B8F8183003F1080280
:1041D800013348F82270A8F818300120BDE8FC81A6
:1041E800B5370008993C0008888F04087E8B0408BE
:1041F8002D3C0008A53B0008913A0008EB3900085F
:10420800B739000841350008CDAC050850710408DD
:10421800CBAC0508F8B51646002834D01378002B27
:104228002ED0028B002327E0046A257C042D21D19F
:1042380065682F888F421DD195F8313053B16F8E44
:1042480001F0B4FE04F1080268866369204606CAD4
:1042580098476F86A81C31462E22FFF7D3F995F8A8
:1042680031307BB104F108026369204606CA9847D9
:104278000120F8BD013304309342D5D30020F8BDA6
:104288001846F8BD0120F8BD70B5B8B1068B0446D4
:10429800002310E0256A287C04280AD16D68288844
:1042A800884206D11046A91C2E22FFF7ABF901203F
:1042B80070BD01330434B342ECD3002070BD38B56F
:1042C800044620B3134BC361134BC0F89830134B0B
:1042D800C0F89C30124B00257822C0F8A0308575B4
:1042E800C5750583294600F1200012F027FED4F891
:1042F80098302046294698470A4A1388312B07D810
:10430800094941F8234001331380012038BD38BDE5
:10431800284638BDCD350008C53500086535000884
:104328003B360008FC0C0020441900202DE9F04120
:104338000446002800F0B380078B02460025A8E059
:10434800136A1E7C042E00F08780012E23D1586842
:1043580003888B4240F09B8005F1080712F004FBAC
:1043680054F827004FF00008C0F8048012F0FCFA57
:10437800228B531E9D4208D00732238354F8221003
:1043880044F8271044F8228002E044F82780258367
:104398003046BDE8F081052E5ED0032E5CD0022E9B
:1043A80013D15B68186803888B4270D14388013B3E
:1043B8009BB243800BB912F0D7FA05F1080654F8FE
:1043C8002630586812F0D0FA4EE0072E21D15E68E8
:1043D800338A8B425BD1002706E0BB1D013756F8B4
:1043E800230012F0C1FAFFB2B38ABB42F5D8002706
:1043F800B78205F1080654F82630586812F0B4FA66
:1044080054F8260033E044F8267025830120BDE8DF
:10441800F081062E1ED1586803888B4237D105F1EA
:10442800080612F0A1FA54F826000027476012F097
:104438009BFA228B531E9D4209D00833013A54F847
:104448002310228344F8261044F82370DEE744F84A
:1044580026701AE0082E1AD1586803888B4216D1A4
:1044680012F082FA05F1080654F826000027476082
:1044780012F07AFA228B531E9D42C4D0073254F8A8
:10448800221044F8261044F822702383BEE7013531
:104498000432BD42FFF454AF0020BDE8F081BDE80E
:1044A800F08170B5044600282AD0068B751E0836A0
:1044B80000EB86061EE056F8043D1A7C042A13D049
:1044C800012A11D0052A0FD0032A0DD0022A02D1C1
:1044D8005B681B6809E0072A02D15B68198A05E056
:1044E800062A01D0082A04D15B6819882046FFF7FC
:1044F8001DFF013D681CDED100232383012070BD10
:1045080070BDF0B528B30023068B1A461EE0046A76
:10451800257C072D18D16468258A8D4214D1A78A75
:10452800002504EB83040DE004EB050C0435DCF8EE
:1045380018C09CF818C0BCF1010F03F1010301D1A8
:10454800D8B2F0BDBB42EFD301320430B242DED361
:104558000020F0BD70B508B3048B00231BE0026A8D
:10456800157C072D15D15268158A8D4211D100236B
:10457800958A11461C46012007E013B996693076E2
:1045880001E08E69347601330431AB42F5D3012062
:1045980070BD01330430A342E1D3002070BD2DE982
:1045A800F04128B30023078B1A461EE0046A257CD5
:1045B800072D18D16468258A8D4214D1B4F814C027
:1045C800002504EB83040CE066190435B66996F8F7
:1045D8001880B8F1010F03D106F10800BDE8F08199
:1045E80001336345F0D301320430BA42DED30020F0
:1045F800BDE8F0812DE9F04700282FD00023B0F85E
:1046080018C01D4627E0046A267C072E21D164685D
:10461800268A8E421DD1B4F81480002604EB830943
:1046280015E009EB0604A7693C7E012C0DD192F830
:1046380000A0BAF1000F08D007F1080011461022B7
:10464800FEF7E0FF2046BDE8F08701330436434516
:10465800E7D3013504306545D5D30020BDE8F087A0
:10466800F0B5B0B1068B002510E0046A277C062F50
:104678000AD1646827888F4206D123819DF81430B7
:104688006260A3720120F0BD01350430B542ECD35D
:104698000020F0BD10B500210446FEF793FF204628
:1046A8000121BDE81040FEF78DBF38B598B1048BE5
:1046B800024600230CE0106A058804328D4206D1B8
:1046C80000F10802436906CA9847012038BD013342
:1046D800A342F0D3002038BD10B50C460021FEF7E8
:1046E80071FF20460121BDE81040FEF76BBF13B5EE
:1046F80002AC04E90C00BDF80230834206D8BDF8CC
:104708000030834234BF0020012000E00020BDF8C3
:1047180006308B4206D8BDF804308B4234BF0021E6
:10472800012100E00021002818BF0846C0B21CBDC6
:1047380038B5114B114A1988002319E052F8045F63
:10474800A87D012812D100240CE004F1080355F8D3
:104758002300037C082B03D1436800211B69984779
:104768000134A4B22B8BA342EFD838BD01339BB2DE
:104778008B42E3D138BD00BFFC0C0020401900205B
:10478800704770B5094CA5787DB9094B1E78012E84
:104798000BD16368013363606268064B9A4204D99F
:1047A800284601F0A1FCA670656070BDFC0C0020D5
:1047B8009801002040420F00054A9060134602E02D
:1047C80099680139996091680029F9D1704700BF4B
:1047D800FC0C0020F0B585B001F032FF002800F095
:1047E8004981002502A80DF10A01ADF80850ADF87D
:1047F8000A5001F027FF03A80DF10E01ADF80C5087
:10480800ADF80E5001F06AFFBDF80C10BDF8082095
:104818000091BDF80E10BDF80A3001912C46964D56
:10482800964908200AF0F8FDA878012803D101F07C
:104838005BFCAC7019E1924B5B78012B40F0158161
:10484800AB78002B40F011816B6029888D4A09E113
:1048580052F8046FB07D012840F002810025FAE08B
:1048680005F10803BDF8080056F82340BDF80A1002
:1048780004F108030CCBFFF73AFF002800F0E980A9
:10488800237C013B062B00F29F80DFE803F004291C
:10489800159D1F9D4C006668012304F108053377B8
:1048A80095E8060063692046984700233377204639
:1048B800636995E8060086E0636893F8252012F19D
:1048C800FF3218BF012283F8252077E0636893F848
:1048D8002C2012F1FF3218BF012283F82C206DE042
:1048E8006268137E1568002B6ED16E882F462946A4
:1048F800184606E051F804EFDEF804E001338EF8BC
:104908001800B342F6D301231376002607E057F8C0
:10491800040F00F10802436906CA984701366B88FC
:104928009E42F4D350E0656820892E68A37B227BE1
:104938000096A0F1160189B2FFF721F81420FFF7BD
:104948003BFF2B7AC3B9AF8A29461A461E4609E0AF
:10495800886990F818E00676BEF1010F08BF134683
:1049680004310132BA42F3D301220BB9AB6924E016
:10497800053355F8233020E06368DB685A68002364
:10498800908A154619461F4609E0AE6996F818E060
:104998003776BEF1010F08BF0B460435013181425D
:1049A800F3D3411E8B4203D1053052F8203003E087
:1049B80004D2073352F8233001221A7604F1080290
:1049C80006CA636920469847237C013B072B4CD8CD
:1049D800DFE803F00410074B0A0D123A63681B6AFC
:1049E80034E063689B6A2DE063681B6B2AE06368A8
:1049F8001B6927E0636824E063681A7A7AB9988AA1
:104A08001946013800E00132824204D28C69247EC2
:104A18000431002CF7D0063253F8223011E0DB685D
:104A28005A68908A11460138002300E00133834216
:104A380004D28C69247E0431002CF7D0063352F856
:104A48002330DB69984710E06368DB6820469847A5
:104A58000BE00135ADB2338BAB423FF601AF04E05A
:104A680001339BB28B427FF4F3AE01F02FFE0F208F
:104A7800FFF7A2FE05B0F0BDFC0C0020F3AC050862
:104A88009801002040190020034B9A6812B19A68D7
:104A9800013A9A60704700BFFC0C00202DE9F347EB
:104AA8000120DFF8D080DFF8D09001460CF04EF8F6
:104AB800012400254FF48076022740466946009677
:104AC8008DF804708DF805408DF806508DF8074074
:104AD8000BF094FC4046082122460BF00FFD244BB6
:104AE800DFF898801A6844F2A243B2FBF3FA0AF19D
:104AF800FF3A204621461FFA8AFA0CF057F8C8F800
:104B080004A048464146A8F80050A8F80250A8F862
:104B1800085088F80A500CF0E5FB7023A8F80C3010
:104B28000423A8F810300AF1FF3A6323642203FB38
:104B38000AF3B3FBF2F39BB2C8F8143008F10C0186
:104B48004846A8F80E40A8F81870A8F81A50A8F80F
:104B58001C60A8F81E500CF0E3FC484621460CF0F7
:104B680056FC484621460CF05CFFBDE8FC8700BFB8
:104B7800E401002000000240000001400C0D00206C
:104B880083B50E460746154910201C4615460AF0FF
:104B980043FC102012490AF03FFC102011490AF08A
:104BA8003BFC10200E490AF037FC002310200E4968
:104BB80001930AF031FC334610200C493A460AF0BA
:104BC8002BFC10200A492A460AF026FC1020094925
:104BD80022460AF021FC019B0133E7E72DAD0508C9
:104BE80032AD050852AD050862AD050872AD05087D
:104BF80087AD050898AD050808B5164B1A6A013245
:104C08001A621A6A012A1A4603D0134840F21E2172
:104C18000FE05862194602E04B6A013B4B62506A4A
:104C28000C4B0028F8D11A6A012A06D00A4840F22B
:104C380029210A4A0A4BFFF7A3FF1A6A013A1A62A6
:104C48001B6A2BB10448054A064B40F22B21F2E7B8
:104C580008BD00BF0C0D0020A9AD05082EA9040849
:104C6800D3AD0508E4AD050810B5084C02210022B3
:104C780020460BF038FC44F6FF70FFF7BDFF2046D6
:104C880002210122BDE810400BF02DBC00040240B7
:104C98000C4B0D491A6844F2A2436428B2FBF3F3A3
:104CA800D4BF20EAE0706420013B9BB24B60013B1B
:104CB80058436422B0FBF2F080B2486103480C31DB
:104CC8000CF0B1BBE40100200C0D002000000140F5
:104CD80010B5134B93F828202AB11248124A134BE7
:104CE80040F209310EE0012283F8282066234FF0B4
:104CF800C042013BDBB2108033B90A480A4A0C4B68
:104D080040F21331FFF73CFF1488A4B28442F0D17B
:104D1800084B1980024B002283F8282010BD00BFE1
:104D28000C0D0020A9AD050838A90408F5AD050843
:104D3800CBAC05080000026010B5FFF7AFFE642099
:104D4800FFF7A6FF21210720FFF7C2FF3220FFF758
:104D580053FF01210020FFF7BBFF3220FFF74CFF74
:104D680023210720FFF7B4FF3220FFF745FF00217A
:104D78001020FFF7ADFF41F28830FFF73DFF3321E8
:104D88000720FFF7A5FF3220FFF736FF112046F670
:104D98003001FFF79DFF3220FFF72EFF4FF4C0616F
:104DA8000220FFF795FF3220FFF726FF122046F674
:104DB800EB41FFF78DFF3220FFF71EFF03204AF675
:104DC800A401FFF785FF3220FFF716FF00210C2012
:104DD800FFF77EFF3220FFF70FFF0D2040F60C0192
:104DE800FFF776FF3220FFF707FF0E204FF42C5114
:104DF800FFF76EFF3220FFF7FFFEB0211E20FFF7FE
:104E080067FF3220FFF7F8FE012042F63F31FFF737
:104E18005FFF3220FFF7F0FE05200021FFF758FF63
:104E28003220FFF7E9FE00210620FFF751FF32206C
:104E3800FFF7E2FE16204EF61C71FFF749FF3220FD
:104E4800FFF7DAFE172040F20311FFF741FF322087
:104E5800FFF7D2FE00210B20FFF73AFF3220FFF7C1
:104E6800CBFE00210F20FFF733FF3220FFF7C4FEEF
:104E780041200021FFF72CFF3220FFF7BDFE422022
:104E88000021FFF725FF3220FFF7B6FE002148205A
:104E9800FFF71EFF40F23F143220FFF7ADFE214618
:104EA8004920FFF715FF3220FFF7A6FE00214A2010
:104EB800FFF70EFF3220FFF79FFE00214B20FFF780
:104EC80007FF3220FFF798FE44204FF46F41FFF7A9
:104ED800FFFE3220FFF790FE00214520FFF7F8FE85
:104EE8003220FFF789FE21464620FFF7F1FE3220E7
:104EF800FFF782FE302040F20771FFF7E9FE32200B
:104F0800FFF77AFE31204FF40171FFF7E1FE3220FE
:104F1800FFF772FE32204FF40171FFF7D9FE40F21D
:104F280002543220FFF768FE21463320FFF7D0FEF7
:104F38003220FFF761FE342040F20751FFF7C8FE28
:104F48003220FFF759FE35204FF40171FFF7C0FEFC
:104F58003220FFF751FE36204FF40171FFF7B8FEFB
:104F68003220FFF749FE21463720FFF7B1FEA4F5AE
:104F780000743220FFF740FE21463A20FFF7A8FED2
:104F88003220FFF739FE2F2041F2BE21FFF7A0FEA5
:104F98003220FFF731FE21463B20FFF799FE3220F1
:104FA800FFF72AFE00212320FFF792FE3220FFF7A9
:104FB80023FE00212420FFF78BFE3220FFF71CFE82
:104FC80025204FF40041FFF783FE3220FFF714FE3F
:104FD80000214F20FFF77CFE3220FFF70DFE4E2008
:104FE8000021FFF775FE3220BDE8104004E608B541
:104FF800124B93F829202AB11148124A124B40F259
:1050080023310FE0012283F82920222166234FF063
:10501800C042013BDBB2118033B90948094A0B4B46
:105028004FF44F71FFF7ACFD108880B22228F0D101
:10503800024B002283F8292008BD00BF0C0D002078
:10504800A9AD050845A90408F5AD0508CBAC0508C8
:1050580010B51B4B032826D8DFE800F0021A080E0B
:105068001C8841F2280246F628000AE01C8841F212
:10507800080246F6080004E01C8841F2300246F6B1
:10508800300049F241318C4214BF014611460BE011
:10509800188846F6200249F24131884214BF114669
:1050A8004FF4815100E000211A8848F689139A428A
:1050B80002D11120FFF70CFEBDE8104097E700BFB2
:1050C8009A010020014B18800A2095E50000026033
:1050D8004FF0C043188003F500331A881A881888DF
:1050E80080B270474FF0C04322221A8003F5003384
:1050F80082B01A8892B2ADF806201B889BB2ADF830
:105108000630BDF8060080B202B07047072040F2B2
:105118007311DDE507200021DAE582B0044BADF814
:105128000600BDF8062092B25A8502B0704700BF4B
:105138000C0D002082B0044BADF80600BDF8062027
:1051480092B25A8002B070479A010020014B80B297
:1051580018807047000002604FF0C04380B218808A
:105168007047024B80B21880704700BF0000026091
:105178004FF0C04380B218807047024B80B218804D
:10518800704700BF0000026082B0044B0190019A92
:10519800DA62DA6A002AFCD102B070470C0D0020EE
:1051A80070B54FF0C0452A242C800A4C060AC0B2BC
:1051B80026802080100AD2B2208022802B222A80CA
:1051C8000A0A2280C9B21A0ADBB22180228023800F
:1051D80070BD00BF0000026010B50B4614460246C1
:1051E800FFF7DEFF4FF0C0432C22A0B21A80BDE8C3
:1051F800104067E70B4B1A8848F689139A4210B596
:1052080004460AD1C1F1EF014E2089B2FFF760FDD3
:105218004F202146BDE810405AE502460B46BDE83E
:105228001040BDE79A01002008B5FFF7E3FF0F4BD8
:105238001B78012B4FF0C0420D4B0FD12E2111804E
:105248001A881A881B8892B202F0FC0002F478428D
:1052580042EAC000C3F3C423184308BD22211180C9
:105268001A881A88188880B208BD00BF141A00204E
:105278000000026070B5074D0646012421463046FD
:10528800FFF7D2FF0134A4B2C82C25F8020FF5D1DC
:1052980070BD00BF3638002010B5084B1B78012BB5
:1052A800144602D1BDE8104096E7FFF7A3FFFFF7C9
:1052B8009EFE2046BDE8104004E700BF141A0020F7
:1052C80070B5074D064601242146013435F8022FF2
:1052D8003046A4B2FFF7E0FFC82CF5D170BD00BF7F
:1052E8003638002070B505460E46FFF7C3FF012487
:1052F8002146013428463246A4B2FFF7CDFFC82C18
:10530800F6D170BD2DE9F84F0C4693460546C718EF
:10531800DFF82CA00AE0BAF82A20B1B292B24046CF
:10532800FFF7BAFF01364E45F5DB0135BD4205DA18
:10533800264604EB0B091FFA85F8F4E7BDE8F88F59
:105348000C0D00202DE9F04104460D461646BDF827
:105358001880032B39D8DFE803F00B3519273819E3
:1053680080B2294642460137FFF796FFBFB200E0F8
:105378000027B742F3D1BDE8F081E01B80B229468F
:1053880042460137FFF788FFBFB200E00027B74267
:10539800F3D1BDE8F081E91B89B2204642460137C6
:1053A800FFF77AFFBFB200E00027B742F3D1BDE8AC
:1053B800F081791989B2204642460137FFF76CFF20
:1053C800BFB200E00027B742F3D1BDE8F08170B565
:1053D800194B1A4A598E92F9004064180025A4B254
:1053E8008AB0AC4208BF0124C62C28BFC624157059
:1053F8000F264FF6FF721E865C865A8519202B46AB
:10540800009221460A22FFF79DFF21463046FFF70A
:105418000BFF224603460A4902A811F00FFE02AA12
:1054280006A8084911F00AFE3220D22106AA2B4606
:1054380000F0D0FE0AB070BD0C0D0020811A0020CB
:105448000AAE050812AE05082DE9F341BDF8205053
:105458000C4690461F461A46002306460095FFF75D
:1054680071FF611E414430463A46002389B20095D7
:10547800FFF768FF30462146424601230095013E6A
:10548800FFF760FFBF19B8B22146424601230895CD
:1054980002B0BDE8F04155E770B50D461C49044619
:1054A800088848F6891188422CD1C5F1F001661E9A
:1054B8009E198A1AC5F1EF0392B29BB29A422CBF89
:1054C80011461946EF2928BFEF219A4238BF1346E3
:1054D80043EA0121B6B289B24420FFF7F9FBA6429C
:1054E80034BF314621464520FFF7F2FBA64238BFBC
:1054F800264640F23F139E4234BF314619464620A5
:10550800FFF7E6FB20462946BDE8704072E600BF7B
:105518009A01002000200146F0224FF4A073BBE757
:1055280070B54FF0C0452A242C80094C060A268005
:105538002080080A208021802B212980110A2180BF
:1055480022801A0A228023802C232B8070BD00BF62
:105558000000026070B5114B1B78012B044607D17F
:10556800002040F23F110246EF23FFF7D9FF04E085
:10557800FFF7D0FF0020FFF76BFDF02509E0013EA3
:105588002046B6B2FFF79EFD002EF8D1013DADB220
:1055980015B14FF4A076F2E770BD00BF141A0020D1
:1055A8002DE9F04F1C463E4B87B01B78039183468C
:1055B8009DF8441010980591012B039B0490924686
:1055C8001FFA8BF09AB208D1411E531E0919534491
:1055D80089B29BB2FFF7A4FF09E01FFA8AF51146CA
:1055E800A3B22A46FFF758FF0020FFF731FD002736
:1055F800DDF80C803E4640F23F1CA14639E0BBF185
:10560800000F2EDB65452CDC0398002829DBB8F158
:10561800EF0F26DC220702D1002CC8BF0136214932
:105628002140002903DA013961F00F010131059A9F
:105638000AB1C1F10F01049830F8162003FA01F1FC
:105648000A4012B26AB118494A8D029392B2A8B2BE
:105658001FFA88F1CDF804C0FFF71EFEDDF804C07C
:10566800029B013401354C45C9DB0136013708F18D
:105678000108574503DA5D4600240123F3E7084B88
:105688001B78012B08D1002040F23F110246EF237E
:1056980007B0BDE8F04F43E707B0BDE8F04F39E782
:1056A800141A00200F0000800C0D00202DE9F74F80
:1056B8001F463B4BDDF830801B7816469DF834209A
:1056C800012B044601920D4680B28AB208D1411ED0
:1056D800531EC9199B1989B29BB2FFF721FF09E034
:1056E8001FFA86FE1146BBB27246FFF7D5FE0020B0
:1056F800FFF7AEFC4FF0000BDA463DE0002C30DB44
:1057080009EB040340F23F1293422ADC002D28DB08
:105718000BEB0503EF2B24DC19F00F0F04D1B9F1C3
:10572800000FC8BF0AF1010A1E4B09EA0303002B48
:1057380003DA013B63F00F030133019A0AB1C3F1A5
:105748000F03012202FA03F338F81A2013401BB2A0
:1057580013B1154B588D01E0144A508880B2FFF7F9
:10576800B1FC09F1010901E04FF00009B945C5DBB9
:105778000AF1010A0BF1010BB345F5DB084B1B7865
:10578800012B08D1002040F23F110246EF2303B05D
:10579800BDE8F04FC4E603B0BDE8F04FBAE600BF7D
:1057A800141A00200F0000800C0D00209A01002020
:1057B8002DE9F0411C4F069C3F789DF81C60012F95
:1057C80002FB03F580B28FB209D1411ECB1899B202
:1057D8007B1E9A1893B23A46FFF7A2FE07E092B2F0
:1057E8009BB23946FFF758FE0020FFF731FC00272F
:1057F80009E034F8020B1EB1030A43EA002080B224
:10580800FFF760FC0137AF42F3DB074B1B78012B36
:1058180007D1002040F23F110246EF23BDE8F041D6
:105828007EE6BDE8F04175E6141A00202DE9F04344
:105838001F2093B0FFF78EFE4FF47840FFF78AFEE3
:105848004FF6E0754FF4FC60FFF784FE2846FFF73B
:1058580081FE0020514CFFF77DFE00204FF6FF79B6
:10586800014664220346A4F82A90CDF80090FFF779
:1058780069FD00200A2164220346CDF80090FFF755
:1058880061FD00200146642201234FF478476585B5
:105898000095FFF757FD7720EF21C82200234FF42A
:1058A800FC6667850097FFF74DFDBD213222012375
:1058B80040F23F1066850096FFF744FDA020322293
:1058C8000023782167850097FFF73CFDA020782109
:1058D800322201234FF01F0866850096FFF732FD3C
:1058E800A020782132220223A4F82A80CDF8008053
:1058F800FFF728FDA0207821322203236585009533
:10590800FFF720FD264B2749A3F8028002AD3C2271
:10591800284611F0D1FAEB20C32105223023009547
:105928000025A4F82A900195FFF7C0FE32210A202D
:1059380096220B4667850097FFF786FD32213C20AB
:1059480096220B4666850096FFF77EFD32210B46B0
:1059580096226E20A4F82A80CDF80080FFF774FD07
:10596800FFF7D8FBFFF7D2FB3220FFF791F9284663
:10597800FFF78EF96420FFF78BF90B4B03F1100248
:105988008DE8240028465A681B682946FFF710FF4F
:105998001195119B01331193FBE700BF0C0D0020FB
:1059A8009A0100205AA9040818CE01082DE9F14FE0
:1059B800FFF774F84FF0C0456420FFF769F9012735
:1059C800FFF752F94FF028096D48FFF715F92F80B6
:1059D8000520A5F8009003F057FACF232B80694BD8
:1059E800002683221E801A8030221A80ED222A8007
:1059F8004FF064080322A3F800801A8012221A804C
:105A080081221A80E8222A8085221A8079221F8022
:105A18001A80CB222A8039221A804FF0340C0224B3
:105A28002C21F72219801E80A3F800C01C802A8030
:105A380020221A80EA222A80C0221E80C1211E80CC
:105A48002A8026221A80298011211980C5212980BF
:105A5800352119803E211980C7212980BE2119804E
:105A6800362129803A205521A3F8009028801980F2
:105A7800B12129804FF0100BF2211E80A3F800B04D
:105A88002980082119802A80E0221F804FF01F09F1
:105A98002A801A22A3F800904FF0180A1A800F21C2
:105AA8000A22A3F800A01A8019800621198045212E
:105AB8001980872119803221198007211A804FF017
:105AC800E10E19801C80052419801C801E80A5F811
:105AD80000E04FF0250E1E80A3F800E04FF0270EDF
:105AE800A3F800E01C80A3F800B04FF0090BA3F85E
:105AF80000B04FF0780B1880A3F800B04FF04D0BB2
:105B0800A3F800B01C800D24A3F800A01C80382442
:105B18001C8018802A20A3F80090EF2428802B20CE
:105B28001E801E801E801C8028803F201E801E80B4
:105B38001F801880B720A5F800C028801980B621DA
:105B480029801A8082221A801122A3F800E0404698
:105B58001E8029272A8003F097F940462F8003F0FA
:105B680093F90948FFF748F82C232F8030462B80FB
:105B780040F23F113246234601B0BDE8F04FCFE472
:105B8800400D03000000026040420F002DE9F04183
:105B9800022098B0012100240AF0D8FF012502262E
:105BA8008048169616A98DF85D408DF85E408DF8F0
:105BB8005F408DF85C500AF021FC182029460AF055
:105BC800C5FF284629460AF0D9FF21460C22764807
:105BD8000AF094FC0C22744829460AF08FFC042130
:105BE8000C2271480AF08AFC05210C226E480AF042
:105BF80085FC07210C226C480AF080FC08210C2245
:105C080069480AF07BFC09210C2267480AF076FCF7
:105C18000A2165480C220AF071FC0B2162480C220B
:105C28000AF06CFC0E210C225F480AF067FC0F2179
:105C38000C225D480AF062FC07210C225B480AF03E
:105C48005DFC08210C2259480AF058FC09210C2255
:105C580056480AF053FC0A210C2254480AF04EFC1C
:105C68000B210C2251480AF049FC0C210A464F48E6
:105C78000AF044FC0D210C224C480AF03FFC0E218E
:105C88000C224A480AF03AFC0C2248480F210AF034
:105C980035FC4CF6B3734448169316A98DF85C602E
:105CA8008DF85E408DF85F408DF85D500AF0A6FBD8
:105CB80016A94FF680733D4816938DF85C608DF8F1
:105CC8005E408DF85F408DF85D500AF097FB40F616
:105CD800B830FEF791FFFEF7C7FF40F6B830FEF781
:105CE8008BFF0F2311934FF4805310270DF13C08BD
:105CF800099368464FF40023109412941494159451
:105D080000940194029403970494069407940894C9
:105D18000A9405940B940C93CDF834800F95139541
:105D28000AF0E5F80523684611930F96109412942B
:105D380014941594CDF8388013950AF0D8F82946AC
:105D480020460AF054F940F6B830FEF755FF2046D1
:105D5800FFF7BEF904461649164E3846224609F0A2
:105D68005BFB41F289239C4248F68918124F01D007
:105D780044450ED1FEF7E0FF00233B70A6F80080F3
:105D880010200E4948F6891241F2892309F044FB94
:105D980005E0FFF70BFE49F241333D70338018B040
:105DA800BDE8F08100040240000C024000100240EF
:105DB80017AE05089A010020141A00202EAE050817
:105DC8004FF0C04336221A8003F50033012814BF70
:105DD800682048201880704770B5244B01228CB089
:105DE8001A7000240AE0A9B21F2230460135FFF7D5
:105DF80053FA642DF7D10134642C02D00025A6B2E1
:105E0800F1E73220014602460346FFF7C9F94FF091
:105E1800C0432E221A8003F5003300201E881C88F8
:105E28001D88A4B2B6B200F09BF8ADB22346104963
:105E38000095324603A811F001F900230A20C82171
:105E480003AA00F0C7F904F0FC0204F4784444EA19
:105E5800C20242EAD522074903A811F0EFF80A2046
:105E6800DC2103AA002300F0B5F9FEE7141A00208C
:105E78006DAE050885AE05082DE9F04F40F23F19D3
:105E8800484534BF04464C46EF2B34BF98464FF084
:105E9800EF084A4538BF9146EF2934BF0D46EF2534
:105EA800C4EB090AC5EB080785B0BAF1000FB8BF03
:105EB800CAF1000A002FB8BF7F424FF6FF734C4566
:105EC8002CBF1A4601221FFA8AFA454538BF01231A
:105ED800BFB202930FFA8AF63BB29E42BDF838B0C1
:105EE800019202DDC6F34F0607E0022693FBF6F6A1
:105EF8007642B6B201E01E4603E00FFA8AF35B422F
:105F08000393144A1378022B204629465A4602D195
:105F1800FDF721FD01E0FFF7BFF94C4501D14545EB
:105F280014D0039A33B2934205DD019AF31BA418E7
:105F38009BB2A4B200E0334636B23AB29642DADAFD
:105F4800029A5344AD189BB2ADB2D4E705B0BDE890
:105F5800F08F00BF582C0020004870471C1A002002
:105F680082B0064BADF80600BDF8062092B21A8042
:105F7800188880B202B0FFF7D0B800BF181A002006
:105F8800014B188880B27047181A002082B0064B5F
:105F9800ADF80600BDF8062092B21A80188880B2C3
:105FA80002B0FFF7C7B800BF1A1A0020014B1888C3
:105FB80080B270471A1A0020FFF7CCBAFFF76CBA04
:105FC80010B5BDF808400294BDE81040FFF7BAB913
:105FD80010B5BDF808400294BDE81040FFF734BA88
:105FE800FFF790B92DE9F04F4FEA420800253D4CE4
:105FF80085B082468B46C8F1030817462E461FFA1D
:1060080087F909EB0B0C228805EB0A031FFA8CFCB5
:106018009BB26146184692B2CDF804C00293FFF7CE
:106028003BF9C9EB0B0292B20392029B22880399B7
:10603800184692B2FFF730F9DDF804C02288C5EBA4
:106048000A039BB26146184692B20293FFF724F9FD
:10605800029B22880399184692B2FFF71DF905EBB7
:106068000B0292B2039209EB0A03228803999BB2AE
:10607800184692B20293FFF70FF9029B2288C5EBEC
:106088000B0C1FFA8CFC1846614692B2CDF804C07E
:10609800C9EB0A09FFF700F9228803991FFA89F961
:1060A80092B24846FFF7F8F82288DDF804C092B2A9
:1060B80048466146FFF7F0F8B8F1000F04DA08EB3C
:1060C800860808F1060805E0F31B08F10A0808EB42
:1060D8008308013F01360135BE42ADB28FD905B004
:1060E800BDE8F08F181A002008B9FFF713B8012887
:1060F80001D1FFF70BB87047704700200146F02226
:106108004FF4A073FFF7C8B9704708B505280CD835
:10611800DFE800F0121403050709094808BD09481B
:1061280008BD094808BD094808BD0948094A0A4B7D
:1061380040F24111FEF724FD084808BD084808BD93
:1061480088010020780100207001002068010020EB
:1061580090AE050896A90408CBAC0508900100206C
:106168008001002010B50446FFF7CFFF014B1860EF
:106178001C7110BDA0010020014B1879704700BFA9
:10618800A001002008B5FFF7C0FF808808BD08B54A
:10619800FFF7BBFFC08808BDF7B51F460B4B0C4E79
:1061A8001D681446EA882B68203C5443A4B2AE1BF1
:1061B80003EB440418BF0126AB888DE8500017B1E3
:1061C800FFF7EEF901E0FFF771FAFEBDA00100202C
:1061D800900100202DE9F0410F46984615460446E7
:1061E800084E08E0204643463946FFF7D5FF336896
:1061F8009B88E418A4B215F8012B002AF2D1BDE857
:10620800F08100BFA001002010B5044608462146D1
:10621800BDE81040DEE7094B70B5044618790E4614
:106228001546FFF7B4FFC6F1F001091A89B22046F6
:106238002A460023BDE87040CCE700BFA00100203B
:10624800704700BF044B1A680AB9044A1A601A68F2
:106258001018186010467047400D0020D43C0020EC
:106268004FF0FF30704708B50248034A034B372107
:10627800FEF786FCAFAE0508ACA90408CBAC050850
:106288000120704710B504460A4802210AF0E4FECE
:106298000028F9D0074821460AF0A7FE0548012141
:1062A8000AF0DAFE0028F9D00248BDE810400AF0EA
:1062B80099BE00BF0038004010B5194802210AF005
:1062C800CBFE0028F9D0164800210AF08EFE1448AB
:1062D80001210AF0C1FE0028F9D011480AF082FE17
:1062E8000402A4B2002301E001339BB2002BFBD0CF
:1062F8000B4802210AF0B0FE0028F9D00848002116
:106308000AF073FE064801210AF0A6FE0028F9D01B
:1063180003480AF067FE2043C0F3CB0010BD00BF5E
:10632800003800402DE9F0478AB00AAF0A20012161
:106338000AF00CFC4FF4604347F8143D474EDFF871
:1063480024A1012400254FF00208304639468DF873
:106358001A508DF818808DF819808DF81B400AF0B6
:106368004DF830460D2105220AF0C8F830460E21B6
:1063780005220AF0C3F8052230460F210AF0BEF8BC
:1063880021464FF480400AF005FC50460AF0E0FC34
:106398004FF48273ADF802304FF40073ADF80A3051
:1063A8003823ADF80C30504607236946ADF8103055
:1063B800ADF80050ADF80450ADF80650ADF80850EF
:1063C800ADF80E500AF0F6FC504621460AF08DFD55
:1063D800A9468DF81A5030464FF480553946059530
:1063E8008DF818408DF819808DF81B400AF006F8D2
:1063F800304629460AF073F84025394618488DF882
:1064080018908DF819808DF81A908DF81B40059515
:1064180009F0F4FF21464FF480400AF0C7FB06213B
:1064280003200AF051FE0C2307A88DF821300795A8
:106438008DF820908DF8224009F0D4FC17238DF8B0
:10644800243009A80F238DF825308DF826308DF8D3
:10645800274002F037FF0AB0BDE8F0870004024089
:10646800000C024000380040014B1878704700BF0C
:10647800440D0020024B5A889B8802800B8070478D
:10648800440D0020014B00221A707047440D002073
:10649800F0B593B068460021482210F04FFD6D46D4
:1064A800002464484FF480510AF01BF8002301E0EF
:1064B80001339BB2002BFBD09020FFF7E3FE0023B3
:1064C80001E001339BB2002BFBD0FFF7F5FE4FF440
:1064D8008051074657480AF002F8002301E00133CB
:1064E8009BB2002BFBD053484FF4805109F0F9FFC1
:1064F800002301E001339BB2002BFBD0D020FFF733
:10650800C1FE002301E001339BB2002BFBD0FFF753
:10651800D3FE4FF480510646464809F0E0FF45F89F
:10652800047B01342E6244484021E4B209F0C5FFDF
:1065380010B9092CB5D101E0092C78D19DE80C00DF
:10654800D218029B03980699D218049BC018059B81
:10655800C018079BCB180899032490FBF4F092FB12
:10656800F4F25B1893FBF4F3151AC11A9C1A002D68
:10657800B8BF6D420029B8BF4942002CB8BF644279
:10658800502D03DD502909DD502C50DC8D4205DAF1
:10659800AC424FF0020405DB111806E08C424FF0C4
:1065A800020401DAD11800E0C1180A9B099A0C9874
:1065B8000F9DD2180B9BD2180D9BC0180E9BC018AC
:1065C800109BEB18119D91FBF4F1032492FBF4F25C
:1065D80090FBF4F05B1993FBF4F3161AC41A9D1A96
:1065E800002EB8BF7642002CB8BF6442002DB8BF59
:1065F8006D42502E89B203DD502C09DD502D16DC7A
:10660800A64205DAB5424FF0020405DB131806E08E
:10661800A5424FF0020401DAD31800E0C318074A74
:1066280093FBF4F39BB2938001235180137013B052
:10663800F0BD00BF00040240000C0240440D0020E1
:10664800FFF712BFF7B505460C4601A80DF1060184
:10665800FFF710FF1B4BBDF80660BDF8040093E878
:106668000600724301FB002299685218164992FBF2
:10667800F1F207EE102AF8EEC77A40F23F17FCEE67
:10668800E77A17EE902A92B2B2F5207F28BF3A46F1
:106698002A801D69DA685B696E4302FB0060C018D6
:1066A80090FBF1F107EE101AF8EEC77AFCEEE77AE4
:1066B80017EE903A9BB2B3F5F07F28BFEF23238003
:1066C800FEBD00BF4C0D002040420F00FFF7DABEB0
:1066D800014B187E704700BF4C0D0020FFF7CABE63
:1066E800042808B505D90748074A084B7D21FEF755
:1066F80047FA054B03EB8000038B0B80438B138019
:1067080008BD00BFD0AE0508B2A90408EEAE050862
:1067180008B5082001F0BAF942F69643C31A584260
:1067280040EB030008BD10B50A2001F0D7F90C4C66
:1067380020600E2001F0D2F96060122001F0CEF93D
:10674800A060162001F0CAF9E0601A2001F0C6F92D
:1067580020611E2001F0C2F901236061237610BD7B
:106768004C0D002010B5FFF7DDFD01F06DFA044671
:1067780001F076FA074903462246202008F04CFE2D
:10678800FFF7C6FF28B101F079FA10B9BDE810404B
:10679800C9E710BD2AAF050810B5104C0A202168BA
:1067A80001F083F961680E2001F07FF9A1681220D9
:1067B80001F07BF9E168162001F077F921691A20C8
:1067C80001F073F961691E2001F06FF9082042F6A3
:1067D8009641BDE8104001F04BB900BF4C0D0020B8
:1067E8002DE9F04F0346A7B0B0F800C01C89868891
:1067F800DF885D89CDF810C0B249B0F802C0B3F89F
:106808000C90B3F80E80CDF824C00FFA84FB30B298
:1068180001220FFA87FE0BEB000C0A7629B20FFA59
:1068280089FACDF888C001EB0E0C0FFA88F2CDF882
:1068380090C00AEB0B0CCDF830C002EB010CCDF880
:1068480058C0B3F810C05B8ACDF800C00FFA8CFCB2
:1068580006910CEB00010A9102930CEB0A011BB2A2
:10686800239103EB0E010E9199182591049900FAD2
:1068780081F0584450446044DDF824C006990EFA6B
:106888008CFEDDF810C01FFA80FB1CFB0CF08E4458
:1068980016FB0600964414FB0400009A19FB090035
:1068A8009E4412FB02001FFA8EFA0BF0DFFCDDF8A3
:1068B80024C0029ACDE912011CFB0CF017FB07005B
:1068C80015FB050018FB080012FB02000BF0CEFCBC
:1068D800DDF824C0029ACDE9140104991CFB01F3E8
:1068E80017FB063615FB0466009B18FB096612FBAE
:1068F80003600BF0BBFCDDE91423CDE90001DDE901
:1069080012010BF029FD04460D46DDE9000102469F
:106918000B460BF021FD02460B46204629460BF09C
:1069280067FBCDE9180158460BF0B0FCCDE9100122
:10693800DDE91023DDE900010BF00EFDCDE90601CC
:1069480050460BF0A3FC804689464246DDE9120119
:106958004B460BF001FDDDE91023CDE91C01DDE913
:1069680014010BF0F9FC002206460F46564BDDE9F0
:1069780018010BF0F1FC424604460D464B46DDE992
:1069880006010BF0E9FC02460B460BF033FB02460E
:106998000B46204629460BF02DFB424604460D4681
:1069A8004B46DDE91C010BF0D7FC02460B4620469E
:1069B80029460BF01DFBDDE9102304460D46304641
:1069C80039460BF0C9FC02460B46204629460BF017
:1069D8000FFBDDF828C0CDE902014FEA8C10DDF885
:1069E80030C000EB0C20DDF810C0A0241CFB040014
:1069F8000BF03CFCDDF838C0CDE90A014FEA8C10F9
:106A0800DDF858C000EB0C20DDF824C01CFB0400A6
:106A18000BF02CFCCDE90C0150460BF027FCDDE90E
:106A28001023CDE91601DDE90C010BF095FC424677
:106A3800CDE91E014B46DDE90A010BF08DFC42460B
:106A4800CDE920014B46DDE900010BF085FC32461B
:106A58003B460BF0CDFACDE90E0158460BF006FC8B
:106A6800DDE91C23CDE91A01DDE906010BF0C0FAC6
:106A7800DDF88CC0C024CDE9060104FB0CF0DDF87C
:106A880088C0302505FB0C00DDF810C078261CFBFB
:106A980006000BF0EBFBDDF894C0824604FB0CF01B
:106AA800DDF890C005FB0C00DDF824C01CFB0600D7
:106AB8008B460BF0DBFBDDE9102306460F460BF097
:106AC8004BFC03E04C0D0020000014404246CDE989
:106AD80004014B46504659460BF03EFCDDE91423B1
:106AE80080468946DDE90A010BF036FCDDE9002322
:106AF80004460D46DDE90C010BF02EFC02460B4660
:106B0800204629460BF074FA0022A14B0BF024FC16
:106B1800DDE9202304460D46DDE91E010BF068FA85
:106B280002460B46DDE916010BF016FC02460B4641
:106B3800204629460BF05EFA002204460D46954B86
:106B4800DDE90E010BF008FC02460B4620462946FB
:106B58000BF050FADDE902230BF028FD88A3D3E9F6
:106B680000230BF0F9FB0BF091FE8B490860DDE97F
:106B78001223DDE90C010BF0EFFBDDE900230446ED
:106B88000D46DDE90A010BF0E7FB02460B462046FD
:106B980029460BF02DFA00227D4B0BF0DDFBDDE9D9
:106BA8001E2304460D46DDE920010BF021FA0246BA
:106BB8000B46DDE91A010BF0CFFB02460B462046D7
:106BC80029460BF017FA002204460D46714BDDE901
:106BD80006010BF0C1FB02460B46204629460BF086
:106BE80009FADDE902230BF0E1FC65A3D3E90023F0
:106BF8000BF0B2FB0BF04AFE674A5060DDE90E234A
:106C0800DDE90A010BF0A8FBDDE9062304460D4681
:106C1800DDE90C010BF0A0FB02460B462046294695
:106C28000BF0E8F9002204460D465A4BDDE918013D
:106C38000BF092FB02460B46204629460BF0DAF988
:106C4800DDE902230BF0B2FC4DA3D3E900230BF0DE
:106C580083FB0BF01BFE504B59469860DDE914236B
:106C680050460BF079FBDDE9002304460D4630461B
:106C780039460BF071FB02460B46204629460BF0BD
:106C8800B7F90022424B0BF067FB424604460D461B
:106C98004B46DDE904010BF0ABF902460B46DDE992
:106CA80016010BF059FB02460B46204629460BF00D
:106CB800A1F935A3D3E9002304460D46DDE90E0109
:106CC8000BF04AFB02460B46204629460BF092F988
:106CD800DDE902230BF06AFC29A3D3E900230BF0BA
:106CE8003BFB0BF0D3FDDFF8B0C0DDE91223CCF895
:106CF8000C00394630460BF02FFBDDE90023044633
:106D08000D46504659460BF027FB02460B462046D7
:106D180029460BF06DF900221D4B0BF01DFBDDE938
:106D2800042304460D46404649460BF061F90246E5
:106D38000B46DDE91A010BF00FFB02460B46204615
:106D480029460BF057F910A3D3E9002304460D4652
:106D5800DDE906010BF000FB02460B4620462946FA
:106D68000BF048F9DDE902230BF020FC04A3D3E97A
:106D780000230BF0F1FA0BF089FD074908610DE0DB
:106D88000000000080842E410000000000C0824006
:106D980000001440000089404C0D0020DDE90E235E
:106DA800504659460BF0D8FADDE9062304460D464D
:106DB800304639460BF0D0FA02460B4620462946A3
:106DC8000BF018F911A3D3E9002304460D46DDE9B9
:106DD80018010BF0C1FA02460B46204629460BF073
:106DE80009F9DDE902230BF0E1FB0AA3D3E900234B
:106DF8000BF0B2FA0BF04AFD034A506127B0BDE828
:106E0800F04FC9E4AFF300804C0D002000000000F3
:106E180000C082400000000080842E41AFF3008053
:106E2800064A074B1A60074A074B1A60074B42F29B
:106E380010721A60064B64221A60704740420F00B5
:106E48004C26002080C3C901642C0020402C00205F
:106E5800F8250020012808B503D05AD3022851D1BB
:106E68003CE02C4B1B78012B03D013D3022B49D1C8
:106E780021E0294BC820196800F017FE274BCC20C9
:106E8800196800F012FE264BD020196800F00DFE9C
:106E9800D42033E0204BD820196800F006FE1F4BA1
:106EA800DC20196800F001FE1D4BE020196800F095
:106EB800FCFDE42022E0184BF820196800F0F5FDED
:106EC800164BFC20196800F0F0FD154B4FF480704C
:106ED800196800F0EAFD4FF482700FE00E4BE820CD
:106EE800196800F0E2FD0D4BEC20196800F0DDFD9B
:106EF8000B4BF020196800F0D8FDF420094B1968F5
:106F080000F0D3FD04F0F0FE18B9BDE8084004F025
:106F1800FCBE08BD1C0E00204C260020642C00205E
:106F2800402C0020F825002008B52E4B1B78012B9B
:106F380002D0022B55D140E02B4B1B78012B03D0FC
:106F480013D3022B4DD121E0C82000F0C7FD274BF9
:106F58001860CC2000F0C2FD254B1860D02000F04E
:106F6800BDFD244B1860D42022E0D82000F0B6FDE7
:106F78001E4B1860DC2000F0B1FD1D4B1860E020AE
:106F880000F0ACFD1B4B1860E42011E0F82000F085
:106F9800A5FD164B1860FC2000F0A0FD144B1860EE
:106FA8004FF4807000F09AFD124B18604FF4827015
:106FB80000F094FD104B186008BDE82000F08EFD2D
:106FC8000A4B1860EC2000F089FD094B1860F0208E
:106FD80000F084FD074B1860F42000F07FFD064B9D
:106FE800186008BDC90100201C0E00204C26002096
:106FF800642C0020402C0020F825002008B504F05F
:1070080073FE10B1BDE808408EE7BDE8084007E709
:10701800064B07495960C021002219721E211A70B7
:10702800D9601A745A611A76DA617047481A0020D2
:1070380040787D0110B50321FF22C02001F02AFC11
:107048001F4C102180222060C02001F023FC112158
:1070580080222060C02001F01DFC122180222060C7
:10706800C02001F017FC132180222060C02001F00D
:1070780011FC142180222060C02001F00BFC152196
:1070880080222060C02001F005FC802220601621AB
:10709800C02001F0FFFB2060C0201721802201F0F2
:1070A800F9FB80222060B721C02001F0F3FB054BDB
:1070B80000221A745A611A76DA6101221A7010BD18
:1070C80020260020481A002038B5C0200321FF22BE
:1070D80001F0E0FB0B4D00242B19615D5A78C020AC
:1070E800023401F0D7FBC82CF6D1B121AC22C02064
:1070F80001F0D0FBC0200321002201F0CBFB0020CF
:1071080038BD00BFDEA904082DE9F34706460F463F
:1071180092461D461AB90C1FE401914635E005EE6A
:10712800902A06EE903AB8EE657AF8EE667AFC0197
:10713800C7EE277AA4F500749FED5C7A67EE877A2C
:1071480017EE900A0BF0B4F841EC100B0DF014FA9E
:1071580059EC108B494640460BF0C0FB24184FEA07
:10716800CA100BF083F8CDE9000128460BF07EF831
:107178004B4642460BF0F0F802460B46DDE90001AB
:107188000AF036FF0BF0AAFB8146002E14BF4FF021
:1071980022084FF01A08C5F307224146C02001F023
:1071A80079FB08F10101EAB2C02001F073FBC4F3D6
:1071B800014208F10201C02001F06CFBC4F3072270
:1071C80008F10301C02001F065FBE2B208F10401F7
:1071D800C02001F05FFBC9F3034305F4702243EAC2
:1071E800123208F10501C02001F054FB08F1060134
:1071F800C9F30722C02001F04DFB08F107015FFA2F
:1072080089F2C02001F046FBC020B121A02201F084
:1072180041FB07EE107A264CF8EEC77A0EBBD4ED88
:10722800015A06EE90AAB8EE657A05EE905AB8EEC5
:10723800666AF8EE656A0123C6EE266A237477EE5D
:10724800A67A67EE277A17EE900A0BF031F841EC30
:10725800100B0DF091F951EC100B0BF03FFB606136
:1072680020E005EE90AAD4ED016AB8EE656A05EE55
:10727800905AB8EE667AF8EE656A0123C6EE266A79
:10728800237677EEA67A67EE277A17EE900A0BF048
:107298000FF841EC100B0DF06FF951EC100B0BF0DF
:1072A8001DFBE0610020BDE8FC8700BF0000004333
:1072B800481A00200022012326E7012838B50D4688
:1072C80004D002280CBF3C242C2400E0342421469E
:1072D800C02001F059FB05F0070200F00F0040EA5A
:1072E80002122146C020BDE8384001F0D3BA2DE98A
:1072F800F3470A9C1D4607468A461646524B01E04C
:107308006D0864089C42FBD82DB906F10076043E4E
:10731800F601A94634E006EE905AB8EE667A06EE13
:10732800904AF8EE667AF601C7EE277AA6F5007657
:107338009FED467A67EE877A17EE900A0AF0B8FF53
:1073480041EC100B0DF018F959EC108B49464046EA
:107358000BF0C4FA3618E8010AF088FFCDE90001FD
:1073680020460AF083FF4B4642460AF0F5FF0246E4
:107378000B46DDE900010AF03BFE0BF0AFFA81464F
:10738800022F9BBF324BDB194FF0000893F8C880DF
:10739800C4F307224146C02001F07CFA08F101013C
:1073A800E2B2C9B2C02001F075FA08F10201C9B20F
:1073B800C6F30142C02001F06DFA08F10301C9B219
:1073C800C6F30722C02001F065FA08F10401C9B22A
:1073D800F2B2C02001F05EFA04F47024C9F303434A
:1073E80008F1050143EA1432C9B2C02001F052FA8B
:1073F80008F10601C9B2C9F30722C02008F107083D
:1074080001F048FA5FFA89F25FFA88F1C02001F0CA
:1074180041FABAF1010F0CBF2F220F220DB942F029
:107428004002012F06D002D3022F0AD105E0C02066
:10743800102104E0C020112101E0C020122101F038
:1074480029FA0020BDE8FC87FFFF0F000000004379
:10745800DEA9040807B5012300930023FFF747FFBF
:107468000EBD00280CBFFF22002208B5C020032152
:1074780001F010FA002008BD08B5C020B121AC22E7
:1074880001F008FA002008BD08B50420012109F020
:107498005DFB4FF480700121BDE8084009F086BB10
:1074A80007B50223009303238DF804300348002313
:1074B80069468DF8073008F0A1FF0EBD00080240AC
:1074C80030B5124D8BB0002406A806940794089492
:1074D800099408F061F900948DF804408DF805408E
:1074E8000294039404942846012469468DF81440B4
:1074F80008F023F928460B212246062308F098F9BC
:107508002846214608F062F90BB030BD0020014042
:1075180010B5002104460122302001F0BBF9C0B9A2
:10752800012001F0B1FC002CB8BF4034E4B21021B6
:107538002246302001F0AEF9012001F0A5FC3020F0
:107548001121224601F0A6F90120BDE8104001F002
:107558009BBC10BD10B5002104460122302001F06B
:1075680099F9C0B9012001F08FFC002CB8BF403454
:10757800E4B212212246302001F08CF9012001F0FA
:1075880083FC30201321224601F084F90120BDE854
:10759800104001F079BC10BD38B5012205460C46F3
:1075A8003020002101F076F9F0B9012001F06CFCDF
:1075B80025EAE5725F2AA8BF5F223B21D2B23020BC
:1075C80001F068F9012001F05FFC24EAE4725F2A07
:1075D800A8BF5F22D2B230203C2101F05BF9012024
:1075E800BDE8384001F050BC38BD302810B504461D
:1075F8000ADC10F17F0F02DB002802DB05E06FF0E8
:107608007E0404F5807400E03024002130200A460E
:1076180001F040F9A8B90120E4B201F035FC41219C
:107628002246302001F036F9012001F02DFC3020EF
:107638004221224601F02EF90120BDE8104001F058
:1076480023BC10BD282810B5044609DC10F1180F1A
:1076580002DB002802DB04E06FF017047F3400E04F
:107668002824002130200A4601F014F9A8B9012085
:10767800E4B201F009FC53212246302001F00AF956
:10768800012001F001FC30205421224601F002F9CA
:107698000120BDE8104001F0F7BB10BD08B530204F
:1076A8000021012201F0F6F860B9012001F0ECFB9D
:1076B80030203321402201F0EDF80120BDE80840D8
:1076C80001F0E2BB08BD10B530200021012201F015
:1076D800E1F8044660B9012001F0D6FB30203321DF
:1076E800224601F0D7F80120BDE8104001F0CCBBDC
:1076F80010BD10B530200021012201F0CBF804465E
:10770800A0B9012001F0C0FB34212246302001F04D
:10771800C1F8012001F0B8FB30203721224601F0E2
:10772800B9F80120BDE8104001F0AEBB10BD402003
:10773800EEE640200EE708B500210122302001F0D6
:10774800A9F8012001F0A0FB30203421024601F005
:10775800A1F8012001F098FB30203721024601F002
:1077680099F80120BDE8084001F08EBB08B500215A
:107778000122302001F08EF8012001F085FB302035
:1077880034210C2201F086F80120BDE8084001F000
:107798007BBB0000000000002DE9F04F984B994A90
:1077A8001968994B002914BF91469946974B2DEDBE
:1077B800048BC3F80090964B0025002287B01A80EE
:1077C800AA46AB46A8465AE0A2004046CDF804C0F7
:1077D80002920AF06DFD0746584601F100460AF08C
:1077E80067FD02460B46384631460AF001FC39F976
:1077F800243007EE103AF8EEC77A064617EE900ADC
:107808000F460AF055FD02460B46304639460AF047
:10781800F1FB0BF083F8074650460AF049FD044691
:10782800284601F100460AF043FDCDE90401DDE9EF
:107838000423204631460AF0DBFB029A09EB0203D7
:107848000446B3F9023007EE103AF8EEC77A0D464F
:1078580017EE900A0AF02CFD02460B4620462946F0
:107868000AF0C8FB0BF05AF8DDF804C0684A0CF1BE
:10787800010CC3465546A2F800C08246B846644B80
:10788800B3F800C00FFA8CF4B32C9DDD58460AF00B
:107898000FFDCDE9020140460AF00AFD0022064626
:1078A8000F465C4BDDE902010AF056FD02460B4625
:1078B800304639460AF09EFB0022574B0AF076FE06
:1078C8000BF02CF84CA3D3E9002309EE900ADDE96C
:1078D80002010AF041FD00224F4B0AF067FE0BF04F
:1078E8001DF809EE100A28460AF0E2FC0446504644
:1078F8000D460AF0DDFC002206460F4620462946C2
:10790800444B0AF029FD02460B46304639460AF038
:1079180071FB0022404B0AF049FE0AF0FFFF36A334
:10792800D3E9002308EE900A294620460AF014FD00
:107938000022394B0AF03AFE0AF0F0FF08EE100A6E
:1079480069EE287A58EE297A17EE900A0AF0B0FC08
:1079580068EE097A48EEA97A044617EE900A0D46B1
:107968000AF0A6FC45EC104B41EC110B0CF008FF9B
:1079780051EC100B0AF0D2FF28EE088A08EEA88A0C
:1079880007EE100A254B264CF1EE477AC3ED007A34
:1079980018EE100A0AF08CFC41EC100B0CF0FEFFFC
:1079A80029EE099A51EC100B09EEA99A0AF0B6FFD4
:1079B800206019EE100A0AF07BFC41EC100B0CF069
:1079C800EDFF51EC100B0AF0A9FFD4ED007A07EE99
:1079D800100A87EE877A134B1860134BFDEEE77A8F
:1079E80083ED007A114BC3ED007A07B0BDEC048B30
:1079F800BDE8F08FAFF30080912B50E67AB6EB3FED
:107A0800701A0020F2220020521D00206C1A00205B
:107A1800781A00200000E03F00005940682C002040
:107A2800802C0020742C0020702C0020741A002058
:107A380010B5084C204608F02EF9074B1860FFF7E0
:107A4800ABFE064B0649012220461A80BDE81040CD
:107A580008F0A2B910600240701A0020680D0020DA
:107A680020800010014B1868704700BF741A00206E
:107A780038B505460C460135C1F3072101F012FA65
:107A8800A8B2E1B201F00EFA00B238BD38B504462A
:107A980001F042F801340546A0B201F03DF8EDB21C
:107AA800C0B240EA052000B238BD37B50B0E8DF8DC
:107AB80004300B0C8DF805300B0A8DF806308DF864
:107AC8000710002400E0284601AB451CE15C0134A6
:107AD80001F0E8F9042CADB2F5D13EBD37B500246C
:107AE80000E02846451C01F017F801ABADB2E054A0
:107AF8000134042CF5D19DF805009DF804300004EC
:107B080040EA03609DF8073018439DF8063040EAC4
:107B180003203EBD37B500230193002400E028462A
:107B2800451C00F0F9FF01ABADB2E0540134042C60
:107B3800F5D19DED010A3EBD7047000038B50446F9
:107B4800642001F0A1F925786068AD00EDB22570D8
:107B580008F0B9FC237A40FA03F000F0030005436B
:107B6800104B257005F00F055A5D6378D218D2B214
:107B7800D3B20132D2B2022A637001D80022A270B5
:107B88005BB2012B03DD0123A3700023637094F91A
:107B98000130013303DAFF23A3700023637094F9E3
:107BA800020038BDAAAA0408F7B504200121234F12
:107BB80008F0CCFF02AD01214FF48040012408F009
:107BC800F5FF00264FF4B0733846694645F8083D7E
:107BD8008DF804608DF8074008F010FC102021464D
:107BE80008F0B4FF78236946154800938DF80460BF
:107BF8008DF8074008F002FC0420214608F0A6FF93
:107C080021464FF4804008F0D1FF1C2338466946CE
:107C180000938DF804608DF8074008F0EFFB022010
:107C2800214608F093FFB02306488DF804606946A2
:107C38008DF80740009308F0E1FBFEBD0008024004
:107C48000010024000040240802108B5034808F0F3
:107C580034FCD0F1010038BF002008BD0004024008
:107C680008B54FF48071044808F027FCD0F10100F2
:107C780038BF002008BD00BF0008024008B5FFF764
:107C8800E3FF08B1FFF7ECFFC0B208BD70B50028EC
:107C98003AD01E4B1A7880181D4AC0B292F90020BB
:107CA800187040B282421B4A02DD117801391970FE
:107CB80093F9001092F9002091FBF2F402FB1414DE
:107CC8001549E4B21C700A88144B1A80144B154AE3
:107CD80018881080144A92F9000064B2013094FBAD
:107CE800F0F200FB1240114C2688114C258800FB4D
:107CF800065008800F4908880F49098802FB0012BE
:107D08001A800E4B01221A7070BD00BF0E3A002077
:107D18003936002015360020443A00205A36002013
:107D28000C3A00200C380020463A00206837002022
:107D3800A83A0020D43A0020EA3700201436002060
:107D4800F0B5264A264C00231370264A2568167873
:107D5800254A12680FE0D45C2F197F7817F0040FBA
:107D680007D0302C02D12023135431E01B4A137062
:107D780003E00133DBB29E42EDDA184B1B788342F5
:107D8800194B16D9A9B11A68164C31211154302152
:107D98000BE01A681518125C2E2A19D0303AD2B2A4
:107DA800092A88BF29700130C0B222788242F0DAED
:107DB8000EE01B681A5C79B12E2A0DD05118C9B291
:107DC800392903D82F2998BF302100E039211954C7
:107DD800BDE8F040FCF7ACBCF0BD00BF6C0D002066
:107DE80048030020C83B0020303A002010B564202A
:107DF80001F04AF88648FFF7A1FE864B1B78044637
:107E08000C2B00F26981DFE813F00D000D0067010B
:107E18007500750037008C008E00BE00C100DB00C5
:107E28008E004301FFF71CFF18B10120F9F77EFD12
:107E380052E1794B1888794B1B88C01A784B1B88FC
:107E480090FBF3F0774B1A88774B1B88D31A774A45
:107E5800128893FBF2F3DBB2C0B2032B00F2D3809B
:107E6800DFE803F002040608714A40E0714A3EE088
:107E7800714A3CE0714A3AE0FFF7F2FED8B10021BE
:107E88000A226F4810F02AFA6E4B002118600A2265
:107E98006D4810F023FA6D4B18600420FEF762F964
:107EA800962005216A4A0023FEF794F90020FEF780
:107EB80059F907F021F8584B1888584B1B88C01AF5
:107EC800574B1B8890FBF3F0564B1A88564B1B8870
:107ED800D31A564A128893FBF2F3DBB2C0B21BB135
:107EE800012B40F0908001E0554A00E0564A594B7A
:107EF8001A6088E0002800F0EF80574B1A7806DDFA
:107F08000132D2B2102A1A7008D9112205E0013ABA
:107F1800D2B2112A1A7001D900221A70F9F7EEFEAE
:107F2800DAE04E4B1870002C00F0D6804C4B1B78D2
:107F3800022B40F0D1804B4B1A78A418E4B20322EC
:107F4800B4FBF2F102FB1144E4B21C70464B474A01
:107F58001B5D022B137009D0052B0CD0012B40F0B0
:107F6800BB804FF491706921414A08E04FF4917049
:107F78006921404A03E0404A4FF491706921002387
:107F8800FEF728F9A8E0354B1870A5E0FFF768FE62
:107F9800A0B10021394810F0EDF8394B042083EDE9
:107FA800000AFEF7DFF8B4200521364A0023FEF761
:107FB80011F9FAF7AFFA0020FEF7D4F82F4A16E0C5
:107FC800FFF74EFE90B100212F4810F0D3F82F4B49
:107FD800042083ED000AFEF7C5F896200521294AFA
:107FE8000023FEF7F7F80020FEF7BCF8264A194BE5
:107FF8001A60094B1888094B1B88C01A084B1B8844
:1080080090FBF3F0C0B22146FFF79AFE64E000BF90
:10801800A8010020CD250020443A0020A83A0020DD
:10802800683700200C3A0020EA370020D43A0020B4
:1080380010260020342600204A2C0020FC25002091
:10804800B03A0020C4010020203A0020C0010020DE
:1080580065AF0508303A0020462600203C3A00204B
:1080680034380020D50D0020300300201C030020E8
:1080780075AF050878AF05087BAF05082C360020DA
:10808800240300207EAF050850360020200300207E
:10809800FFF7E6FD08B107F007F914B1254B0122F7
:1080A8001A70254B1A68A41814F5967FB8BF234A8E
:1080B8001C60B8BF1A601B68B3F5967F03DD1E4BC2
:1080C8004FF496721A601B4C23782BB11C4B18681E
:1080D80001F0D8FA002323701A48FFF72FFD1A4B36
:1080E8001B78013B0A2B24D8DFE803F0062323235F
:1080F8002015152311111500FFF7C8FDFFF7A4FD82
:10810800002816D00220BDE81040F9F70FBC0F4B2D
:108118001B78022B0AD100280D4B01D1187010BD15
:1081280001DD012200E0FF221A7010BDBDE81040F9
:10813800ACE510BD48260020403A0020D4FEFFFFE1
:10814800EC250020B4010020CD2500203438002083
:10815800811A002010B58CB01E490F2268460EF017
:10816800ABFE1D490F2204A80EF0A6FE1B490F22E4
:1081780008A80EF0A1FE00210822302000F08AFB9A
:10818800012000F081FE002404AB1DF80420E15C0E
:10819800302000F07FFB0134012000F075FE0F2C29
:1081A800F2D100210922302000F074FB012000F0F8
:1081B8006BFE002408AB1DF80420E15C302000F0C1
:1081C80069FB0134012000F05FFE0F2CF2D10CB0E6
:1081D80010BD00BFBCAA0408CBAA0408DAAA040888
:1081E80010B58CB01E490F2268460EF065FE1D4979
:1081F8000F2204A80EF060FE1B490F2208A80EF0FB
:108208005BFE00210822302000F044FB012000F032
:108218003BFE002404AB1DF80420E15C302000F094
:1082280039FB0134012000F02FFE0F2CF2D1002180
:108238000922302000F02EFB012000F025FE00244A
:1082480008AB1DF80420E15C302000F023FB01346A
:10825800012000F019FE0F2CF2D10CB010BD00BFA8
:10826800E9AA0408F8AA040807AB040810B58CB0FA
:108278001E490F2268460EF01FFE1D490F2204A852
:108288000EF01AFE1B490F2208A80EF015FE002159
:108298000822302000F0FEFA012000F0F5FD00244D
:1082A80004AB1DF80420E15C302000F0F3FA01343F
:1082B800012000F0E9FD0F2CF2D100210922302025
:1082C80000F0E8FA012000F0DFFD002408AB1DF8FB
:1082D8000420E15C302000F0DDFA0134012000F0D8
:1082E800D3FD0F2CF2D10CB010BD00BF16AB0408A3
:1082F80025AB040834AB040807B50220012108F0B7
:1083080025FC012300938DF8043002238DF80530F5
:108318000448002369468DF806308DF8073008F0C8
:108328006DF80EBD0004024010B5084C0121002272
:10833800204608F0D8F840F2FF4000F0A5FD0121E2
:1083480020460A46BDE8104008F0CDB800040240B7
:1083580008B5FFF7E9FF00210A46302000F09AFA35
:10836800012000F091FD01210A46302000F092FA28
:10837800012000F089FD00210122302000F08AFA56
:10838800012000F081FD01210822302000F082FA4E
:10839800012000F079FD02210122302000F07AFA54
:1083A800012000F071FD00210A46302000F072FA29
:1083B800012000F069FD1B21CD22302000F06AFA6F
:1083C800012000F061FD04210322302000F062FA50
:1083D800012000F059FD06210922302000F05AFA48
:1083E800012000F051FD07210822302000F052FA48
:1083F800012000F049FD08217022302000F04AFADF
:10840800012000F041FD1E213020B02200F042FA88
:10841800012000F039FD05219122302000F03AFAC0
:10842800012000F031FD0D210322302000F032FA46
:10843800012000F029FD0E210022302000F02AFA48
:10844800012000F021FD14218022302000F022FAC2
:10845800012000F019FD0B218822302000F01AFAC3
:10846800012000F011FD0C218222302000F012FAC8
:10847800012000F009FD12218822302000F00AFABC
:10848800012000F001FD13218C22302000F002FAB7
:10849800012000F0F9FC00210A46302000F0FAF92A
:1084A800012000F0F1FC3D210222302000F0F2F919
:1084B800012000F0E9FCFFF74DFEFFF791FEFFF702
:1084C800D5FE30200021012200F0E4F9012000F05F
:1084D800DBFC3D216422302000F0DCF9012000F0B3
:1084E800D3FC03210022302000F0D4F9012000F051
:1084F800CBFC04210022302000F0CCF9012000F050
:10850800C3FC00210122302000F0C4F9012000F052
:10851800BBFC0C210822302000F0BCF9012000F03F
:10852800B3FC0D210822302000F0B4F9012000F03E
:10853800ABFC0E210822302000F0ACF9012000F03D
:10854800A3FC0F210822302000F0A4F9012000F03C
:108558009BFC00210A46302000F09CF9012000F025
:1085680093FC02224021302000F094F9012000F011
:108578008BFC30204121002200F08CF9012000F012
:1085880083FC3F21D422302000F084F9012000F040
:108598007BFC00210122302000F07CF9012000F052
:1085A80073FC10210F22302000F074F9012000F034
:1085B8006BFC11210F22302000F06CF9012000F033
:1085C80063FC12210022302000F064F9012000F041
:1085D8005BFC13210022302000F05CF9012000F040
:1085E80053FC09213C22302000F054F9012000F00E
:1085F8004BFC00210122302000F04CF9012000F052
:1086080043FC30203421024600F044F9012000F0F8
:108618003BFC30203721024600F03CF9012000F0F5
:1086280033FC36210322302000F034F9012000F019
:108638002BFC39210322302000F02CF9012000F016
:1086480023FC3B213C22302000F024F9012000F0DB
:108658001BFC3C210A46302000F01CF9012000F0E8
:1086680013FC00210A46302000F014F9012000F024
:108678000BFC5121C022302000F00CF9012000F041
:1086880003FC52213020002200F004F90120BDE84B
:10869800084000F0F9BB00BF2DE9F04F454E464DAC
:1086A80093B001214FF4001008F050FA304607F05B
:1086B800F3F94FF0C0630293404B0393404B0024FF
:1086C80004934FF4B4794FF400334FF480684FF4B7
:1086D80000674FF4005A4FF4807B304602A90C9390
:1086E80001930997CDF8189005940794CDF8208048
:1086F800CDF828A0CDF82CB00D9407F059FA2246F1
:108708003046304907F0AFFA3046012107F0B5FA94
:1087180001210A464FF0402008F086FC284607F061
:10872800BBF9294A019B0392284A0C9304922846D4
:10873800402202A9059209970294CDF8189007944F
:10874800CDF82080CDF828A0CDF82CB00D9407F0F6
:108758002FFA224628461E4907F085FA28460121A5
:1087680007F08BFA42F2107701220221194808F02B
:108778005BFC384600F088FB3046012107F053FACD
:108788000121284607F04FFA384600F07DFB0B23FD
:108798008DF8443011A801238DF845408DF84640E6
:1087A8008DF8473000F08EFD384600F06DFB13B0B1
:1087B800BDE8F08F10600240886002400C40004025
:1087C800F2220020521D00200C3C004022200020F4
:1087D800821A0020003C004002481021012207F0C4
:1087E80099BA00BF1060024013B50220012108F0B9
:1087F800ADF94FF410730E4C009302238DF804303A
:108808008DF8053001238DF806302046002369468F
:108818008DF8073007F0F2FD20460621042207F004
:108828006DFE20460921042207F068FE1CBD00BF2A
:108838000004024030B5154D85B001214FF40010F9
:1088480008F0A8F9284607F06FFE0023ADF80430B9
:108858004BF6FF73ADF806303323ADF808304FF40C
:108868008063ADF80A304FF48043ADF80C3004ACA7
:10887800074B2846012144F8103D07F0F7FE28462B
:10888800694607F07FFE05B030BD00BF00540040C8
:10889800801A060073B54FF4961306460D46144623
:1088A800019304E0019B5A1E0192002B57D03148D6
:1088B8004FF4003107F0F2FF0028F3D12D480121D1
:1088C80007F0E0FE4FF48053019304E0019B5A1E29
:1088D8000192002B45D02748274907F0CAFF0028F6
:1088E800F4D024483146002207F0E4FE4FF48053C8
:1088F800019304E0019B5A1E0192002B33D01D48BE
:108908001E4907F0B6FF0028F4D01A48294607F098
:1089180054FF4FF48053019303E0019B5A1E0192C8
:108928001BB31448164907F0A4FF0028F5D01148D6
:10893800214607F042FF4FF49613019303E0019B91
:108948005A1E01929BB10B480E4907F0A7FF002859
:10895800F5D00848012107F0A1FE002008E0012019
:1089680006E0022004E0032002E0042000E00520E5
:108978007CBD00BF005400400100030082000700D6
:10898800800007000400001037B54FF49613044622
:108998000D46019305E0019B5A1E0192002B00F041
:1089A8009B8056484FF4003107F078FF0028F2D139
:1089B8005248012107F066FE4FF48053019305E009
:1089C800019B5A1E0192002B00F088804B484C49AD
:1089D80007F04FFF0028F3D048482146002207F04F
:1089E80069FE4FF48053019304E0019B5A1E0192E3
:1089F800002B75D04148434907F03BFF0028F4D0CD
:108A08003E48294607F0D9FE4FF48053019304E00D
:108A1800019B5A1E0192002B64D038483A4907F04E
:108A28003DFF0028F4D03548012107F02BFE4FF414
:108A38008053019304E0019B5A1E0192002B53D0EE
:108A48002E482F4907F015FF0028F4D02B4821465F
:108A5800012207F02FFE4FF48053019304E0019B9D
:108A68005A1E0192002B41D0244C2849204607F079
:108A780015FF0028F3D02046002107F023FE2046EA
:108A88000121238B07F00AFE4FF48053019304E081
:108A9800019B5A1E0192002B2AD018481C4907F046
:108AA800FDFE0028F4D0154807F089FE4FF48053E6
:108AB8000193124A03E0019B591E0191D3B1138817
:108AC8009B05F8D4012104460C4807F0FBFD0B4830
:108AD800104907F0FDFE0EE001240CE002240AE034
:108AE800032408E0042406E0052404E0062402E048
:108AF800072400E0082420463EBD00BF0054004083
:108B080001000300820007000400001002000010AA
:108B1800400000100004001013B54FF496130446EB
:108B2800019305E0019B5A1E0192002B00F0AF80D3
:108B380060484FF4003107F0B1FE0028F2D15D48DB
:108B4800012107F09FFD4FF48053019305E0019B3D
:108B58005A1E0192002B00F09C805648564907F097
:108B680088FE0028F3D05348A021002207F0A2FD78
:108B78004FF48053019305E0019B5A1E0192002B8C
:108B880000F089804B484D4907F073FE0028F3D068
:108B9800210A484807F011FE4FF48053019304E07E
:108BA800019B5A1E0192002B77D04248444907F096
:108BB80075FE0028F4D0E1B23E4807F0FEFD4FF400
:108BC8008053019304E0019B5A1E0192002B66D04A
:108BD80038483B4907F062FE0028F4D035480121A7
:108BE80007F050FD4FF48053019304E0019B5A1E97
:108BF8000192002B55D02F482F4907F03AFE002844
:108C0800F4D02C48A121012207F054FD4FF48053E1
:108C1800019304E0019B5A1E0192002B43D0254C7E
:108C28002849204607F03AFE0028F3D020460021C4
:108C380007F048FD20460121238B07F02FFD4FF454
:108C48008053019304E0019B5A1E0192002B2CD003
:108C580018481D4907F022FE0028F4D0154807F0EF
:108C6800AEFD4FF480530193124A03E0019B591E55
:108C78000191E3B113889905F8D4012104460D4800
:108C880007F020FD0B48114907F022FE10E00124EF
:108C98000EE002240CE003240AE0042408E0052482
:108CA80006E0062404E0072402E0082400E0092482
:108CB80020461CBD0054004001000300820007004C
:108CC8000400001002000010400000100004001012
:108CD80013B54FF496130446019305E0019B5A1E01
:108CE8000192002B00F0AF8060484FF4003107F08C
:108CF800D5FD0028F2D15D48012107F0C3FC4FF4EF
:108D08008053019305E0019B5A1E0192002B00F04D
:108D18009C805648564907F0ACFD0028F3D05348CC
:108D2800A021002207F0C6FC4FF48053019305E010
:108D3800019B5A1E0192002B00F089804B484D4937
:108D480007F097FD0028F3D0210A484807F035FDC1
:108D58004FF48053019304E0019B5A1E0192002BAB
:108D680077D04248444907F099FD0028F4D0E1B291
:108D78003E4807F022FD4FF48053019304E0019B25
:108D88005A1E0192002B66D038483B4907F086FDF1
:108D98000028F4D03548012107F074FC4FF48053C3
:108DA800019304E0019B5A1E0192002B55D02F48D5
:108DB8002F4907F05EFD0028F4D02C48A12101229C
:108DC80007F078FC4FF48053019304E0019B5A1E8E
:108DD8000192002B43D0254C2849204607F05EFD20
:108DE8000028F3D02046002107F06CFC2046012122
:108DF800238B07F053FC4FF48053019304E0019B4D
:108E08005A1E0192002B2CD018481D4907F046FD28
:108E18000028F4D0154807F0D2FC4FF48053019392
:108E2800124A03E0019B591E0191E3B113889C0586
:108E3800F8D4012104460D4807F044FC0B481149B9
:108E480007F046FD10E001240EE002240CE00324A4
:108E58000AE0042408E0052406E0062404E00724C8
:108E680002E0082400E0092420461CBD005400400C
:108E78000100030082000700040000100200001037
:108E8800400000100004001082B0002304E0019BA1
:108E980001330193009B01330093009B8342F6D377
:108EA80002B0704737B54FF4805304460D4601931E
:108EB80004E0019B5A1E0192002B6DD03C484FF4F0
:108EC800003107F0EBFC0028F3D13948012107F005
:108ED800D9FB4FF48053019304E0019B5A1E019281
:108EE800002B5BD03248334907F0C3FC0028F4D08C
:108EF8002F48A021002207F0DDFB4FF48053019397
:108F080004E0019B5A1E0192002B49D028482A49A7
:108F180007F0AFFC0028F4D0210A254807F04DFCE3
:108F28004FF48053019304E0019B5A1E0192002BD9
:108F380038D01F48214907F09CFC0028F4D0E1B242
:108F48001B4807F03AFC4FF48053019303E0019B60
:108F58005A1E019243B31648184907F08AFC0028A4
:108F6800F5D01348294607F028FC4FF496130193CF
:108F780003E0019B5A1E0192C3B10D48104907F046
:108F88008DFC0028F5D00A48012107F087FB0D4821
:108F9800FFF77AFF00200AE0012008E0022006E03F
:108FA800032004E0042002E0052000E006203EBD86
:108FB8000054004001000300820007008000070001
:108FC80004000010A0860100F7B54FF48053044652
:108FD8000D461646019304E0019B5A1E0192002B90
:108FE80074D040484FF4003107F058FC0028F3D102
:108FF8003C48012107F046FB4FF48053019304E0FD
:10900800019B5A1E0192002B62D03648364907F060
:1090180030FC0028F4D03348A021002207F04AFB96
:109028004FF48053019304E0019B5A1E0192002BD8
:1090380050D02C482D4907F01CFC0028F4D0210AF8
:10904800284807F0BAFB4FF48053019304E0019BD2
:109058005A1E0192002B3FD02248254907F009FCEF
:109068000028F4D0E1B21F4807F0A7FB4FF4805363
:10907800019304E0019B5A1E0192002B2ED019483F
:109088001B4907F0F6FB0028F4D000244FF496178C
:1090980010E0295D134807F090FB019703E0019B5E
:1090A8005A1E0192E3B10F48124907F0F7FB002856
:1090B800F5D00134E3B2B342EBD30A48012107F0FB
:1090C800EDFA0D48FFF7E0FE00200AE0012008E075
:1090D800022006E0032004E0042002E0052000E06E
:1090E8000620FEBD00540040010003008200070076
:1090F8008000070004000010A086010013B50520B9
:10910800012107F023FD184C4FF4E053009302238C
:109118008DF804308DF805302046002369468DF817
:1091280006308DF8073007F069F920460A21062233
:1091380007F0E4F920460C21062207F0DFF90622A1
:1091480020460B21A4F5006407F0D8F94FF400433A
:1091580020466946009307F051F920460F21062260
:1091680007F0CCF91CBD00BF000802401FB504463B
:10917800FFF7C2F8FFF75EFBFFF7EAF8FFF7BEFF5D
:1091880001214FF4004007F005FD02940F4C102315
:10919800ADF80230204600236946ADF80430ADF83A
:1091A8000C30ADF80030ADF8063007F022FE694605
:1091B8004FF0402007F0F1FE2046012107F0A1FE04
:1091C8004FF04020012107F09CFE1FBD003C0040ED
:1091D80082B0002304E0019B01330193009B01331B
:1091E8000093009B8342F6D302B0704707B5042072
:1091F800012107F0ABFC01214FF4804007F0D6FCB9
:109208004FF40073009300238DF8043003480123C2
:1092180069468DF8073007F0F1F80EBD00080240E6
:109228000D4B07B51A680D484FF47A73B2FBF3F289
:109238000B4B013A5A600B4AF02182F823100022A6
:109248009A6007221A60084B084A00930121084BCC
:1092580002F010F80EBD00BFE401002050260020E7
:1092680010E000E000ED00E000030020E402002030
:109278004C020020054B1A6812B11A68013A1A60AC
:10928800034B1A6801321A60704700BF0C26002091
:109298002426002082B0044B0190019A1A601A68B3
:1092A800002AFCD102B070470C260020704700BF8E
:1092B80040F0BE60024B40F42020D860704700BFE9
:1092C80000ED00E0C37810B503B3164B4278DB68B5
:1092D8008478DB43C3F30223C3F10401C9B202FA61
:1092E80001F10F2242FA03F2C9B222400A430E4B9F
:1092F80001781201CB18D2B283F800230378012237
:10930800590903F01F0302FA03F307E00378012267
:10931800590903F01F0302FA03F32031024A42F805
:10932800213010BD00ED00E000E100E021F06041D7
:1093380021F07F01014B08439860704700ED00E081
:10934800044B1A6909B1104301E022EA00001861D0
:10935800704700BF00ED00E0044B1A6804280CBFFA
:1093680042F0040222F004021A60704710E000E0A4
:10937800014B93ED000A7047702C0020014B93EDD0
:10938800000A7047682C0020014B93ED000A7047D3
:109398007C2C0020014B93ED000A70476C2C0020B8
:1093A800014B93ED000A7047802C0020014B93ED90
:1093B800000A7047742C002008B5FDF73BFE00201A
:1093C800012324210246FDF79FFE124B1B78013B27
:1093D800DBB20020012B05D80146FDF76EFF012006
:1093E800002104E00721FDF768FF01200721FDF7B0
:1093F80064FF63221221C020FFF74CFA02200121EA
:10940800FDF75BFFFEF738F80120BDE80840FEF7DE
:1094180028B800BF1C0E00200E4B1B78062B05D168
:109428000D4B0E4A196812688A181A600C4B1B7883
:10943800013BDBB2012B084B196805D8094A914258
:1094480007DD01321A607047074A914201DD013297
:109458001A607047CD250020442C0020C425002028
:109468001C0E00207FD1F008FF27ED080F4B1B785A
:10947800062B05D10E4B0F4A196812688A1A1A6012
:109488000D4B1B78013BDBB2012B094B05D80B4A6E
:109498001968914208DC1A6070471A68B2F57A2F89
:1094A800DCBF4FF47A221A60704700BFCD25002038
:1094B800442C0020C42500201C0E002020A10700F9
:1094C8002DE9F04F6A4B6B4C1B688DB019220A903E
:1094D80069485343B0FBF1F01C190D4608F0C6FE6D
:1094E80041EC100B0BF048F851EC100B09F0F6F9B1
:1094F80010F0010F804618BF00F1FF3805FB08F097
:1095080008F0B4FE064620460F4608F0AFFE0246B5
:109518000B463046394609F049F804460D4645ECF5
:10952800104B0BF029F857EC106B204632463B469F
:10953800294608F05DFDCDE902013946304609F0BB
:10954800CDF947A3D3E900230B90DDE9020109F027
:109558007FF9002858D1012000264FF0150931461F
:1095680007464FF0000A4FF0000B03E0304639463B
:10957800069E049FA7FB0A23541807FB0B333F4A98
:1095880043F100050023A242AB41CDE904453ED397
:10959800A6FB0A23141806FB0B33384843F10005D1
:1095A8000021A042A941CDE9064530D3DDE90201F9
:1095B8002DA3D3E90023049C069D09F049F940BB7B
:1095C800DDE9022300202E4908F0F0FF82468B4691
:1095D8004BEC10AB0AF0D0FF5046594653EC102B19
:1095E8008DED080B08F004FDCDE90201DDE9080165
:1095F80009F042FC09F1FF395FFA89F982468B4686
:10960800B9F1000FB2D104E00125002401E035468C
:109618003C460B9A0A9BD1B25BB9184622462B46A8
:10962800FDF772FD0A98012300930146424603465E
:1096380009E022462B460120FDF766FD0120009037
:10964800014642460023FDF752FEFDF715FF0120B3
:109658000DB0BDE8F04FFDF704BF00BFAFF30080C9
:10966800956479E17FFDA53DBBBDD7D9DF7CDB3DA6
:10967800403A002040787D0100E9A435FFFF0F0043
:109688000000F03F2B4A2C4B1278012A10B51860C5
:109698000BD12A4A904201DD01321A60284A1B6820
:1096A80093420EDC244B1A600BE0022A09D1254AAA
:1096B800904201DD01321A60234A1B6893420FDC95
:1096C8000CE01D4B214A1968914201DD01321A60F4
:1096D8001B68B3F57A2F03DC4FF47A22164B1A6015
:1096E800154B1B4A19681B4B1B4C1B68CB18934224
:1096F80023601ADC0020FFF7E3FE01202168FFF752
:10970800DFFE0C4B1B78013BDBB20020012B05D898
:109718000146FDF7D2FD0120002104E00721FDF7F5
:10972800CCFD01200721FDF7C8FD034B1A680B4B40
:109738001A6010BD1C0E0020442C00207FD1F008B8
:1097480020A107007F74D21A60E31600FF27ED08F6
:1097580080D1F0085C2C0020602C002028360020E6
:10976800014B18688EE700BF40260020AFF3008049
:109778007047FEE7FEE7FEE7FEE770477047704771
:1097880002F036B910B5094CA37A4BB1084B1A68E8
:1097980022F006021A6000F013F8204600F047FE97
:1097A8004FF48020BDE8104006F084BB502600200E
:1097B80010ED00E0014801F009B800BF5026002074
:1097C800364BD3F8882042F47002C3F88820344B13
:1097D8001A6842F001021A6000229A60196821F0A2
:1097E800847121F4803119602E495960196882B05A
:1097F80021F480211960DA60009201921A6842F41B
:1098080080321A601A6802F400320192009A01321A
:109818000092019A1AB9009AB2F5A06FF2D1204BC2
:109828001B6813F4003318BF01230193019B012B1C
:109838002ED11B4B1A6C42F080521A641A4A1168D6
:1098480041F4804111609A689A609A6842F4004233
:109858009A609A6842F4A0529A60144A5A601A6848
:1098680042F080721A6019680D4A8901FBD5104BC5
:1098780040F205611960936823F0030393609368CD
:1098880043F002039360936803F00C03082BFAD1AA
:10989800024B4FF000629A6002B0704700ED00E0A2
:1098A800003802401030002400700040085440077F
:1098B800003C0240184B194A996801F00C01042930
:1098C80003D0082903D0164B19E0164B17E0596846
:1098D8005A6811F4800F596814BF124B104B02F0EC
:1098E8003F02B3FBF2F30C4A5268C2F30142C1F3E0
:1098F8008811013252004B43B3FBF2F3074A13605D
:10990800054B9A68054BC2F303129A181968127925
:1099180021FA02F21A60704700380240E401002080
:109928000024F40000127A0037B51C230124002516
:1099380001A88DF804308DF805508DF806408DF893
:109948000740FFF7BFFC2046214607F023F90A49E4
:1099580040F2E1434B6040F24F130B800D814D8084
:109968004FF0804007F0BEFC4FF080402146224671
:1099780008F07DF83EBD00BF842C002008B54FF0EC
:109988008040012108F088F880B101214FF0804023
:1099980008F08DF8FEF72AFA054B064A11781A786E
:1099A8008A181A70044B1A8801321A8008BD00BF41
:1099B800F12500203C3A0020780D002008B5402011
:1099C80006F06AFA30B1FCF763FD4020BDE80840B4
:1099D80006F070BA08BD0000014608B5044808F052
:1099E80025FA0348402108F0CEFA0028F9D008BD2E
:1099F80000440040F0B589B04FF4E13301200193F1
:109A080000232B4CADF808301E460146ADF80A304D
:109A1800ADF80C30ADF810300C23ADF80E3007F06F
:109A280095F84FF40030012107F0B4F820680221BE
:109A3800072206F063FD07226068032106F05EFD39
:109A48000125022704232068059305A98DF81A60CB
:109A58008DF81B508DF818708DF8197006F0CEFC33
:109A680008236068059305A98DF8187006F0C6FCF0
:109A7800A06801A908F030F92A4640F225510D489E
:109A880008F068FA262307A88DF81C308DF81D60A9
:109A98008DF81E608DF81F50FFF714FCA06829464A
:109AA80008F097F9044A054B1A6009B0F0BD00BFE9
:109AB800F801002000440040E1990008CC3B002058
:109AC800024B9868002108F084B900BFF801002013
:109AD80010B5094C40F22551204608F05EFA50B105
:109AE800A288D2B2112A02D1044B01211970044B69
:109AF80019884A401A8010BD004400407F0D00209C
:109B0800880D00207047704773B50120014607F0A3
:109B18001DF8264C4FF4D8530093022303268DF8E2
:109B280004302046002369468DF806308DF807304A
:109B38008DF8056006F062FC204608210A2206F02E
:109B4800DDFC204609210A2206F0D8FC20460B211C
:109B58000A2206F0D3FC0A2220460C2106F0CEFC8D
:109B680001254FF480632046694600938DF806501E
:109B78008DF807508DF8056006F040FC0A210A466A
:109B8800204606F0BBFC29464FF4804007F00EF84B
:109B98008020294606F0E6FF4FF08050294607F05E
:109BA80035F8284606F086F97CBD00BF0000024063
:109BB80007B54FF4C060FFF77BFB43238DF80430F3
:109BC8000322012301A88DF805308DF806208DF8B1
:109BD8000730FFF777FB0EBD782358430723B0FB08
:109BE800F3F0002301338342FCD970474FF47A73B2
:109BF8005843F1E737B50023104C0193054603207D
:109C0800FFF7EAFFEB681A69013C019213D0019A49
:109C1800002AF4DA019A42F001020192019A1A61CB
:109C2800064A1969013A019102D00199C907F8D485
:109C38000320FFF7D1FF00203EBD00BF410D030008
:109C480010B5C47874B900EB820003339B10D0F8C8
:109C5800D000224603E051F8044C0132046004317C
:109C68009A42F8D1002010BD033230B59210D0F8D6
:109C7800D0400B46002003E02568013043F8045C1F
:109C880004339042F8D101EB800030BD0122F0B5D9
:109C98000023827040220129C37082800CD10823DE
:109CA8000370042343704FF4A073C380022303722C
:109CB800C1724FF0A04309E041B90C230370062399
:109CC80043704FF4A063C3801F4BC17203F5006259
:109CD8000261C3604678044601461A46002508E03A
:109CE80002F5106C02F530620A65C1F814C001353E
:109CF8003A460431B54202F12007F1D303F58062F8
:109D0800426103F58862C0F8CC20067803F5A065A7
:109D18000146002203E0C1F88C500132203504319D
:109D2800B242F8D31946002202E0C4F8CC1001323E
:109D38000434B24201F58051F7D303F56063C0F8EB
:109D48000C310020F0BD00BF0000044038B5037A94
:109D5800C2680025012B044625D1936B417A65F32F
:109D6800104309B143F480139363D36823F4800349
:109D780023F0500343F010036FF3C3036FF3C713CB
:109D88006FF351436FF3D343D3602046FFF732FF9D
:109D9800E378012B3ED1052363F34405E36845F0DE
:109DA80020059D6036E0D36843F04003D360FFF799
:109DB80021FF237A627A032B14BF4FF434134FF434
:109DC8003C130AB143F48013E26814209363FFF74D
:109DD8000DFFE268217AD368032908BF43F4803372
:109DE800D360237A032B15D1156B012363F39B658D
:109DF8006FF3D7552D2345F0805563F3164515634A
:109E0800C820FFF7F3FEE36845F400051D63C8208A
:109E1800FFF7ECFEE378012B07D1E3689D68052284
:109E280062F3440545F020059D60002038BDC368F5
:109E38009A6842F001029A6000207047C3689A68E5
:109E480022F001029A600020704707B500230193B1
:109E5800019B43F020030193019B61F38A13019353
:109E6800019BC2681361064B1169013B019102D045
:109E780001998806F8D40320FFF7AEFE00200EBD36
:109E8800410D030007B500230193019B43F0100324
:109E98000193019BC2681361064B1169013B019153
:109EA80002D00199C906F8D40320FFF795FE0020D7
:109EB8000EBD00BF410D030008B5C268D368012973
:109EC8006FF35D736FF39E7302D143F0005302E0AA
:109ED80009B943F080433220D360FFF787FE0020A2
:109EE80008BDC368586900F001007047C3685B6922
:109EF80013F0010F14BF002001207047C368586990
:109F080000F001007047C3685A69986910407047AB
:109F1800C3685868704703691A6861F301021A60D8
:109F28007047C268002393614FF0FF335361536059
:109F380053610B4B9361C3789169002B14BF4FF4A5
:109F480000634FF4016343F4701343F4405343F048
:109F5800080321EA03010B4393610020704700BF07
:109F680000080080F8B5D0F80C3100221A600369A7
:109F780015461A6865F3CC221A60C37A012B044689
:109F88001BD10321FFF7C7FFE36880214FF480024C
:109F980061F30F0259629A62C02262F30F0561F3FE
:109FA8001F454FF4A072C3F8045162F30F056FF315
:109FB8001F45C3F80851C3F80C5110212046FFF77C
:109FC80044FF2046FFF75EFF226900234FF0FF3170
:109FD8001361204653611E469161FF25D3612146D6
:109FE80010E082691768C7F3076707F08007FFB2B8
:109FF800002F14BF4FF090470027176001331661F8
:10A008000430956062789342EBD300231D46FF200D
:10A0180010E04A6D1668C6F3076606F08006F6B2C9
:10A02800002E14BF4FF090460026166001331561CC
:10A038000431906062789342EBD323691A6942F441
:10A0480080721A61E278012A04D1054A402161F33D
:10A0580059421A632046FFF764FF0020F8BD00BF8D
:10A068000301010003699B68C3F34103013B022B11
:10A078009ABF024AD05C0320704700BF78AB04083F
:10A0880010B5036981699C680A68C4F34100022815
:10A0980002D06FF30A0202E0032060F30A020A60AA
:10A0A8005A6842F480725A60002010BD30B54D786D
:10A0B8000B780022012D00EB830405D105FA03F388
:10A0C800A46963F30F0205E0012505FA03F3646D43
:10A0D80063F31F422368C3F3072505F08005EDB23B
:10A0E8006DB98D6865F30A03CD78C98865F3934324
:10A0F80061F3995343F0805343F4004323600369A9
:10A10800D9690A43DA61002030BD30B54D780B7843
:10A118000024012D224600EB830105D105FA03F343
:10A12800896963F30F0205E0012505FA03F3496D18
:10A1380063F31F4203696FF3CF340C60D96921EAD6
:10A148000202DA61002030BDF8B54F780B78012F94
:10A1580000EB830349D19E694C69356833692A4607
:10A1680064F3120314B967F3DC430BE08F68E41956
:10A17800013CB4FBF7F7CC7867F3DC43012C08BF4C
:10A1880064F35E733361C378012B06D10B780C69D5
:10A1980000EB83039B695C610CE0CB78012B09D051
:10A1A8004B693BB103690C785E6B012707FA04F42D
:10A1B80034435C63CB78012B07D103699B68DB05CB
:10A1C80054BF45F0005245F080520B7800EB8303F2
:10A1D80042F004429B691A60CB78012B38D10A7887
:10A1E8008B8AC968FFF72CFD32E05E6D4F693568D0
:10A1F8008C6833692A462FB964F31203012464F387
:10A20800DC430AE03F19013FB7FBF4F7BF05BF0D78
:10A2180067F3DC437C4364F312033361C378012B97
:10A2280005D10B780C6900EB83035B6D5C61CB781F
:10A23800012B06D14B7913B145F0005201E045F0EE
:10A2480080520B7800EB830042F00442436D1A60A1
:10A258000020F8BD73B54D78012D3DD183694A6959
:10A268001E681C690094E4B242B962F306048DF8D2
:10A2780000409DF8024065F3C4040EE08D68AA42D0
:10A2880086BF4D6165F3060462F306048DF800404D
:10A298009DF80240012262F3C4048DF80240009A3E
:10A2A8001A61C278012A05D10A780C6900EB82028A
:10A2B8009269546146F004421A60C378002B34D185
:10A2C8004B69002B31D003690A78586B012101FAD8
:10A2D80002F202435A6328E00B784E698C6800EB5F
:10A2E80083035B6D1A681D690095EDB206B14C6178
:10A2F80064F306059DF802408DF80050012565F3CA
:10A30800C4048DF80240009C1C61C378012B05D160
:10A318000B780C6900EB83035B6D5C610B7800EBD9
:10A32800830042F00442436D1A6000207CBD4B78E4
:10A33800012B0B7800EB83000AD182691368C3F301
:10A34800076101F08001C9B221B143F0804301E007
:10A35800426D136843F400131360002070474B7874
:10A36800012B0B78C97800EB83000CBF8269426D22
:10A3780002391368C9B26FF35553012998BF43F0E6
:10A38800805313600020704703699A69D8691040A8
:10A39800000C704700EB810102694B6D9B685069A6
:10A3A8001840704703699869DB69184080B27047A4
:10A3B80082B000230093C0238DF8033001220023CC
:10A3C80062F3C4038DF8023018238DF80030009A28
:10A3D800436D1A61C278012A06D100F5B960586147
:10A3E8001A684FF080221A6002B07047D0F8143112
:10A3F80010B50446D3B103699A68D20716D5827A94
:10A4080042B1D0F80C21D0F80C116FF341026FF370
:10A4180000020A605A6842F001025A600520FFF7FC
:10A42800E5FB23695A6822F001025A6010BD837A5D
:10A4380063B103699B68D90708D5D0F80C31D0F807
:10A448000C216FF341036FF300031360704701237E
:10A4580010B5002280F8123104460346FF2104E0BB
:10A4680058698160186D01328160607804338242D6
:10A47800F6D3236900221A615A61DA614FF0FF327C
:10A488009A612046FFF7FEFC20461021BDE81040E7
:10A49800DBE44B78012B0B7800EB83000FD1836949
:10A4A8001868C0F3074000F02003DBB2CBB900F016
:10A4B8000200C0B200280CBF302020207047436D36
:10A4C8001868C0F3074000F02003DBB25BB900F066
:10A4D8000200C0B200280CBF4FF440504FF40050A7
:10A4E8007047102070474FF4805070474B78012B0D
:10A4F8000B7810B500EB83030AD19C69102A2368F6
:10A5080002D1BDE8104012E7202A0CD0302A0FE013
:10A518005C6DB2F5805F236802D143F400131BE041
:10A52800B2F5005F02D143F0006315E0B2F5405F79
:10A538000FD1C3F3074202F02002D2B222B10023A6
:10A548004B71BDE810400AE743F0806343F0802375
:10A5580002E00AB962F3CF33236010BDF8B50446B0
:10A56800FFF794FB0122002384F8122184F81331A9
:10A5780028271646194640250CE007FB03F000F58E
:10A588008C7022182354D3805670D1709560D16096
:10A598005161013362789342EFD30023282619468C
:10A5A80040250CE006FB03F000F55C7022182354EC
:10A5B800D3805170D1709560D16051610133627858
:10A5C8009342EFD32046FFF739FC2046FFF7BEFB46
:10A5D80000212046FFF770FC2046FFF7C3FC204609
:10A5E800BDE8F840FFF723BC70B5CDB20C464FF07C
:10A5F800280601F07F0106FB010115F0800F14BF4A
:10A6080001F58C7101F55C7104F07F04ED090C70A3
:10A618004D708A60CB7005B1CC80022B01D100232C
:10A628000B71FFF743FD002070BD10B5CAB201F0F1
:10A638007F034FF0280404FB030312F0800F14BFBC
:10A6480003F58C7303F55C7301F07F01D20919706F
:10A658005A701946FFF759FD002010BD38B501F0B2
:10A668007F0528246C4304F55C7401194B610023B1
:10A678008B614B70EBB20355CA60C478012C08BFDC
:10A688000A6113B9FFF7E6FD01E0FFF75DFD002061
:10A6980038BD70B501F07F042825654305F58C7534
:10A6A80041190126E4B2CA600A6100224E7044557D
:10A6B8008A614B6114B9FFF7CDFD01E0FFF744FD56
:10A6C800002070BDCAB212F0800F10B54FF02803F9
:10A6D80006D001F07F0403FB040303F58C7303E049
:10A6E80003FB010303F55C73D209012401F07F0128
:10A6F80019709C705A701946FFF719FE002010BD9A
:10A70800CAB212F0800F10B54FF0280306D001F03E
:10A718007F0403FB040303F58C7303E003FB0103CD
:10A7280003F55C730024D20901F07F0119709C7055
:10A738005A701946FFF713FE204610BD08B50B06E0
:10A7480004D501F07F01FFF780FB01E0FFF79AFBDA
:10A75800002008BD0369002261F30A1219680A4340
:10A768001A60704703695A6803206FF341025A6000
:10A77800FFF73CBA03695A68032042F002025A60A4
:10A78800FFF734BA11F0800F4FF0280306D001F01C
:10A798007F0103FB010101F58C7103E003FB01015B
:10A7A80001F55C71FFF775BE11F0800F4FF02803BB
:10A7B80006D001F07F0103FB010101F58C7103E074
:10A7C80003FB010101F55C71FFF790BE2DE9F74F1E
:10A7D8000446FFF78BFB002800F03F822046FFF776
:10A7E80092FB0546002800F03882C0F3074000F0CD
:10A7F8000800C0B2002861D02046FFF7C5FDA14679
:10A80800824627464FF00008DFF86CB32E4650E02A
:10A818001AF0010F46D05FFA88F2114620460092DE
:10A82800FFF7B8FD10F0010F0546009A20D07B6DA8
:10A8380001259D60E178A94207D11B69D9F87813F1
:10A84800C3F31203CB1AC9F88833DBF8003020466B
:10A858001B6811469847E378012B09D1B8F1000F1E
:10A8680006D194F81131052B02D12046FFF7A0FD3F
:10A8780005F00203DBB213B17B6D02259D6005F084
:10A888000403DBB213B17B6D04259D6005F0080558
:10A89800EDB23DB1DBF8003020469B6898477B6DF0
:10A8A8000820986008F101084FEA5A0A043709F1AC
:10A8B8002809BAF1000FABD135460120C5F307438B
:10A8C80003F00403DBB2002B00F0AF802046FFF753
:10A8D80069FD264683464FF0000801959FE01BF06E
:10A8E800010F00F0978023695FFA88F919695D6B99
:10A8F80004EB890225FA09F59269ED019268EDB237
:10A908000D431540EA071CD55A6B012000FA08F1DF
:10A9180022EA01025A63B369974A986013680546A8
:10A928005B68204649469847E378AB4209D1B8F1BD
:10A93800000F06D194F81131042B02D12046FFF7FD
:10A9480037FD05F00403DBB213B1B36904259D603C
:10A9580005F00803DBB213B1B36908259D6005F063
:10A968001003DBB213B1B36910259D6005F0200315
:10A97800DBB213B1B36920259D6005F04003DBB25B
:10A9880013B1B36940259D6005F00203DBB213B132
:10A99800B36902259D6025F07F0515F0FF0F39D0BA
:10A9A800282505FB084505F58C75C246AB696A691B
:10A9B800C3EB020CAB689C4528BF9C460CF1030C0A
:10A9C800B3694FEA9C0C9B696746A04614E0AA68E5
:10A9D800E9681C1B944228BF1446A3B240464A4665
:10A9E800FFF72EF9EB681B19EB60AB69E71C1C1924
:10A9F800AC61B3699B69BF089BB2BB4205D9AC691E
:10AA08006B699C4201D2002BE1D1B3698025444691
:10AA18009D60D04608F101084FEA5B0B0436BBF194
:10AA2800000F7FF45CAF019D012005F00203DBB24B
:10AA380013B1E36802225A61C5F3076303F0800388
:10AA4800DBB2CBB1A37A43B1D4F80C31D4F80C21E2
:10AA58006FF341036FF30003136023695A6822F010
:10AA680001025A60444B1B6820469B699847E3687B
:10AA78004FF000425A610120C5F3072303F0080391
:10AA8800DBB2F3B13C4B1B6820465B6998472369EE
:10AA9800E2689B684FF400615161A27A82B1DB07DA
:10AAA8000ED5D4F80C311A6842F001021A601A68FF
:10AAB80042F003021A60314B1A6942F006021A6129
:10AAC800012005F00803DBB243B12B4B1B6820467D
:10AAD800DB689847E36808225A61012005F01003F3
:10AAE800DBB2002B33D0E3689A6922F010029A6136
:10AAF8001F6A282607F00F0306FB0346C7F34343E4
:10AB0800022B06F55C7602D0062B1AD10EE047F62A
:10AB1800F0733B40ABB1C7F30A172046F1683A46D9
:10AB2800FFF7A2F8F368DB19F36007E004F5B961F1
:10AB380020460822FFF798F8C7F30A17B369DF1908
:10AB4800B761E3689A6942F010029A610120C5F37F
:10AB5800072303F01003DBB2002B39D023695A68AE
:10AB6800002622F001025A6031462046FFF76DF9AF
:10AB780023463246FF2108E09402002000ED00E061
:10AB880058698160186D01328160607804338242AF
:10AB9800F6D3236901274FF0FF3267F30F069A6156
:10ABA80067F31F460F22DE615A612F221A611A6865
:10ABB8006FF30A121A602046FFF7FAFBE3684FF4B6
:10ABC80080525A61264B1B6820461B6998473846B5
:10ABD800C5F3072303F02003DBB2EBB12046FFF7F0
:10ABE8004FFAE3682046DE68FFF73CFA032806D1EF
:10ABF8000023A3704FF40073A380092304E001230A
:10AC0800A3704023A380052363F38D26E3684FF4E4
:10AC18000052DE6001205A61C5F3074303F01003B8
:10AC2800DBB24BB10E4B1B682046DB699847E368E3
:10AC38004FF480125A610120C5F3074505F020053D
:10AC4800EDB255B1064B1B6820461B6A9847E3686E
:10AC58004FF400125A610120FFE7BDE8FE8F00BFE4
:10AC68009402002043230B80004870470402002010
:10AC780038B51F4B1A68511C052A196035D1197946
:10AC8800002201291A6030D09968B1F5006F08BF19
:10AC98009A60174B9968DC68A1421A4602D10022D3
:10ACA8001A7122E086BFC1F500631361C1EB040489
:10ACB800D0F8EC3598BF14611569B3F839300C4CED
:10ACC8009D428AB204D95918ED1AA160256104E0A1
:10ACD8006918A1600021ABB22161054901240C71FA
:10ACE80004498A188121FFF7D4FC002038BD00BF31
:10ACF8008C0D0020232D002038B528230A4D03FB96
:10AD080001010A4BB1F888131B6904462846984785
:10AD1800D4F8EC352046B3F8403001212A46FFF735
:10AD28009DFC002038BD00BFDB2C002080020020E5
:10AD380070B50B7813F0600506460C4625D0202D1B
:10AD48001FD1CD88B5B113F0800F487808D0214BBA
:10AD580021499B682A469847E2881F49304625E0E2
:10AD68001E4B1D4958641E4B30465D612A4600F053
:10AD780022FB1DE0174B48789B6829462A469847CE
:10AD880025E000F077FB022521E04B780A2B11D053
:10AD98000B2B14D0062B1AD14B881B0A212B03D15D
:10ADA800CA883A2A28BF3A220E49304600F0EAFA01
:10ADB80000250CE00C49012200F0E4FA07E08B784A
:10ADC8001BB9074A1D46936101E000F053FB284672
:10ADD80070BD00BF800200201B2D0020040200204F
:10ADE8008C0D002016020020A40D002010B5812132
:10ADF8000446FFF71AFC01212046FFF716FC8221C2
:10AE08002046FFF712FC024B5B689847002010BDF4
:10AE18008002002038B5D0F8EC350446B3F8392064
:10AE280081210223FFF7E0FBD4F8EC350121B3F8C8
:10AE3800402020460223FFF7D7FB82210822032364
:10AE48002046FFF7D1FB094B022200251A715D71DC
:10AE5800074B1B689847D4F8EC35064AB3F84030DE
:10AE680020460121FFF7FAFB284638BDC40200201E
:10AE780080020020DB2C002010B5074C606CFF28F6
:10AE880007D0064B064A9B68064952699847FF2334
:10AE98006364002010BD00BF04020020800200206F
:10AEA8008C0D00201B2D002038B510490B79012B83
:10AEB80019D10C690CB90C7115E0D0F8EC358D6816
:10AEC800B3F839309C42AAB203D95D198D60E41AEF
:10AED80003E0A3B22C198C6000240C6104495218B9
:10AEE8008121FFF7D6FB002038BD00BF8C0D002064
:10AEF800232D002000207047002070470023F0B564
:10AF0800084A094E1D4609E01468C75C37550134E4
:10AF18000133B4F5006F146008BF15608B42F3D19C
:10AF28000020F0BD980D0020232D0020104B114A61
:10AF3800D3F800C000232DE9F0410F4F16461D46F7
:10AF48000DE0146810F8038007F804800134802CA1
:10AF580008BF2C4614603468644505D001338B4221
:10AF6800EFD10020BDE8F0810220BDE8F08100BFEC
:10AF7800A4350020B83500202435002021280FD121
:10AF8800084B1A680A701A68120A4A705A888A7036
:10AF9800DA78CA701A790A715A794A719B798B7171
:10AFA800002070477802002007B502AB012103F8A2
:10AFB800010D1846FFF7A2FF0EBD002100E0013188
:10AFC800435C002BFBD199E798E70B4B0B491A68B8
:10AFD800096891420BD00A498A5C02701A680132EA
:10AFE800802A1A6005D100221A60012070470020CB
:10AFF80070470120704700BFA4350020B8350020F5
:10B0080024350020204B1A68204B1B689A42F0B563
:10B0180009D135E00133802B08BF00239A4203D1C0
:10B028001A4B1A602CE01A4CE15C0029F2D00A296C
:10B03800F0D00D29EED0154C1549134D23600E465E
:10B048000023CF182268BA5CC254226801339F18C3
:10B05800802F08BF53422F689A18974210D0B25CCD
:10B068001AB10A2A01D00D2AEBD10022C254074A8C
:10B07800116859187F29116003D98039116000E0DF
:10B0880000231846F0BD00BFB8350020A4350020C5
:10B0980024350020704700BFD0F8E43510B51B698F
:10B0A80004469847032384F81231002010BD08B5E0
:10B0B800042380F81231D0F8E435DB689847002083
:10B0C80008BD08B5D0F8E035DB6903B19847002022
:10B0D80008BD08B5D0F8E0351B6A9847002008BDC0
:10B0E80008B5D0F8E0355B6A9847002008BD002114
:10B0F80010B5402204460B46FFF776FA802140221D
:10B1080000232046FFF770FA012384F81231D4F89F
:10B11800E435A0785B689847002010BD13B56946F0
:10B12800044600F085F99DF8001001F01F03012B7B
:10B1380007D0022B0AD073B92046694600F026FAD8
:10B148000FE02046694600F007FA0AE02046694603
:10B1580000F0A2F905E021F07F01C9B22046FFF70F
:10B16800B1FA00201CBD38B5044600293DD190F83D
:10B178001131022B42D1D0F83421D0F820319A4233
:10B1880011D9C178D21A0129C0F8342104D1D0F8D4
:10B198002411CB18C0F8243192B22046D4F82411D7
:10B1A80000F000F92AE0D0F83821B2FBF3F503FBF0
:10B1B800152565B99A420AD3D0F83C319A4206D28D
:10B1C80029462A4600F0EEF8C4F83C5116E0D4F8B7
:10B1D800E035DB682BB194F81221032A01D120460F
:10B1E8009847204600F00FF908E0D0F8E0355B6991
:10B1F80023B190F81221032A00D19847002038BDC6
:10B2080010B5044659BB90F81131032B30D1D0F852
:10B218008C23D0F878339A4214D9C178D21A0129EC
:10B22800C0F88C2304D1D0F87C13C918C0F87C135B
:10B238009A4228BF1A4692B22046D4F87C1300F0EE
:10B24800CAF815E0D0F8E0351B6923B190F812214F
:10B25800032A00D19847204600F0C6F808E0D0F845
:10B26800E0359B6923B190F81221032A00D1984751
:10B27800002010BD2DE9F041069F04461646984669
:10B288000D46FEF741FC20462946C4F8E085C4F87F
:10B29800E475C4F8E865FFF761F9D4F8E4351B688C
:10B2A80098472046BDE8F041FEF782BC0020704771
:10B2B800D0F8E03510B504461B689847D4F8E43553
:10B2C8009B689847002010BD08B5D0F8E0355B684A
:10B2D8009847002008BD000012230B8000487047E3
:10B2E800C402002004230B8000487047D6020020C7
:10B2F80010B5044C04480A46214600F075FA204669
:10B3080010BD00BFBC35002046B005080A4608B588
:10B318000248034900F068FA014808BD59B0050819
:10B32800BC3500200A4608B50248034900F05CFA1B
:10B33800014808BD67B00508BC35002008B50A46B5
:10B3480008B9044800E00448044900F04DFA0348ED
:10B3580008BD00BF72B005087FB00508BC350020E5
:10B3680008B50A4608B9044800E00448044900F052
:10B378003BFA034808BD00BF8CB00508ADB005080E
:10B38800BC35002010B513460C46C0F83821C0F86B
:10B398003421022280F8112100212246FFF779F991
:10B3A800002010BD10B50C46134600212246FFF7B9
:10B3B80070F9002010BD10B513460C46C0F8902354
:10B3C800C0F88C23032280F8112100212246FFF7C0
:10B3D80045F9002010BD10B50C4613460021224641
:10B3E800FFF73CF9002010BD0021042310B50A46E0
:10B3F800044680F811310B46FFF74BF92046FEF75B
:10B40800D7FF002010BD0021052310B50A460446C9
:10B4180080F811310B46FFF721F92046FEF7C8FFE7
:10B42800002010BD282303FB0100B0F888037047F3
:10B4380090F8C8350B7090F8C9354B7090F8CB254B
:10B4480090F8CA3503EB02234B8090F8CD2590F88D
:10B45800CC3503EB02238B8090F8CF2590F8CE35BE
:10B4680003EB02239BB2CB80C0F83C31012380F868
:10B478001131704710B591F90030002B044601DBFB
:10B48800CB880BB9802100E00021FFF71BF920468B
:10B49800BDE81040FEF78CBF38B50D4604466B7802
:10B4A8000979012B10D027D3032B51D190F81231F1
:10B4B800022B28D0032B47D16B889BB991B18029E7
:10B4C80010D0FFF7FFF80DE090F81231022B1AD0D8
:10B4D800032B39D16B88002B3AD149B1802907D089
:10B4E800FFF70EF9D4F8E03520469B6829469847BF
:10B4F8002046FFF779FF2BE090F81231022B02D09B
:10B50800032B21D106E019B3802921D02046FFF76B
:10B51800D9F81DE011F0800F4FF0280306D001F094
:10B528007F0103FB010393F81A2103E003FB0101E8
:10B5380091F87223074B02B101221A60204605498F
:10B548000222FFF71FFF03E020462946FFF792FF7C
:10B55800002038BDA80D002038B590F81231032B13
:10B5680004460D460CD10B79012B09D8D0F8E035EB
:10B578009B689847EB883BB92046FFF735FF03E007
:10B5880020462946FFF776FF002038BD73B54B7873
:10B5980004460D46092B00F21C81DFE813F0D100A8
:10B5A80008011A01E4001A0172000A001A01C00019
:10B5B80092004B881A0A013A062A00F20A81DFE84B
:10B5C80012F007001A002700080108010801080105
:10B5D800D4F8E835A0781B680DF106019847EB8888
:10B5E800402B014603D094F81231012B3AD108239D
:10B5F800ADF8063036E0D4F8E035A0789B6A0DF156
:10B6080006019847022343700146C4F8EC0529E077
:10B61800DBB2052B00F2DD80DFE803F003080D1232
:10B62800171CD4F8E835A0785B6817E0D4F8E8353B
:10B63800A0789B6812E0D4F8E835A078DB680DE0C4
:10B64800D4F8E835A0781B6908E0D4F8E835A07884
:10B658005B6903E0D4F8E835A0789B690DF1060131
:10B6680098470146BDF80630002B00F0B680EA88FE
:10B67800002A00F0B2809A4228BF1A46ADF8062088
:10B688005CE08B88002B40F0A480CB88002B40F036
:10B69800A08094F812214B88032A00F09A8003F0C6
:10B6A8007F05204684F813512946FFF753F82046B2
:10B6B800FFF79AFE0DB1022300E0012384F812314E
:10B6C8008BE08978464E0129317100F2828094F826
:10B6D8001231022B02D0032B7BD108E0002962D063
:10B6E8000121032384F8101184F8123113E041B9C1
:10B6F800022384F8123184F810112046FFF7E4FD84
:10B7080051E094F81011012920464DD0FFF7DCFDD7
:10B71800317984F810112046FFF7CAFD43E0CA8842
:10B72800012A56D194F81231022B02D0032B50D1A2
:10B7380002E020462B4913E004F5887120460FE00B
:10B7480094F81231023B012B43D8D4F81431244920
:10B75800002B0CBF0123032341F80C3F2046012294
:10B76800FFF710FE39E04B88012B29D0022B34D18A
:10B778008B8813F0FF0F30D121691B0A013B4A68FF
:10B78800042B0FD8DFE803F0030507090B0001239A
:10B7980006E0022304E0032302E0042300E005237B
:10B7A80063F306124A602046FFF71EFE15E094F880
:10B7B8001231023B012B0CD84B88012B0DD10023F1
:10B7C800C4F81431D4F8E03520469B6829469847D8
:10B7D800E9E720462946FFF74DFE00207CBD00BF63
:10B7E800A80D0020B00D002030B5C8B10023DDB28F
:10B7F8000133C41814F8014C002CF8D16B1C5B0001
:10B8080013800B7003234B70022305E0CA545A1CA3
:10B81800D2B202338C54DBB210F8012B002AF5D1D6
:10B8280030BD00BF7047704770477047704770471A
:10B83800704700000000000008B5FCF705FA094B46
:10B848005A78187002435A701AB19A7801329A706D
:10B8580030B99B78034A012B02D9002353709370A7
:10B8680008BD00BFB80D00202DE9F84F3F4B1B78ED
:10B87800012B2DED028B09D002D3022B0FD108E04A
:10B888003B4B1A68802392FBF3F206E0384B1A68A8
:10B8980003E0374B1B6803225A43364B5A61364B39
:10B8A8001A8892B2002AFBD0334B00221A80FDF787
:10B8B8005FFD10EE105AFDF761FD284610EE104AA4
:10B8C80006F0F6FC80462046894606F0F1FC41EC7D
:10B8D800100B41EC180B08F0F7FD57EC106BB0EEAD
:10B8E800480AF0EE680A08F0EFFE32463B4640464A
:10B8F80049465BEC10AB06F02FFD07F00FF89FED03
:10B908001F8A07EE100ADFED1E7A57EE087A194CE7
:10B9180052465B46C4ED007A4046494606F01CFD97
:10B9280006F0FCFF07EE900A27EE888A84ED018A6C
:10B93800FDF736FD84ED020AFDF738FD84ED030AB4
:10B94800FCF790F80F4B62691B68D31A0E4A07EE92
:10B95800100A1268F8EEC77A93FBF2F3C4ED047A82
:10B968002383BDEC028BBDE8F88F00BF1C0E0020BE
:10B97800442C0020EC370020680D00200000F04225
:10B9880000008C4240260020C425002007B5042072
:10B99800012105F0DBF84FF46043009301238DF893
:10B9A800043002238DF805300448002369468DF8D9
:10B9B80006308DF8073004F021FD0EBD0008024066
:10B9C800084B1A684FF47A73B2FBF3F2064B013A4C
:10B9D8005A60064AF02182F8231000229A60072252
:10B9E8001A607047E401002010E000E000ED00E07C
:10B9F800034B5A6812B15A68013A5A60704700BF3F
:10BA0800B80D0020024B58605A68002AFCD17047D4
:10BA1800B80D002030B585B004460D4601A8674929
:10BA28000A220BF049FA664B1B78032B10D8DFE883
:10BA380003F00205080B01A8624907E001A8624962
:10BA480004E001A8614901E0614901A80BF01EFB6F
:10BA580004AA131913F80C3C5D19EDB22F2D01D867
:10BA68000A3502E0392D01D90A3DEDB204AB1C19A3
:10BA78004FF6FF7004F80C5CFAF772FA0020FAF738
:10BA880071FB0DF103050F24204623345A210023AE
:10BA980015F8012FA4B2FAF77FFBB4F5A57FF3D10F
:10BAA80064205A212C220023FAF776FB0023CD20AC
:10BAB8005A212C22FAF770FB0020FAF751FA404B72
:10BAC8001B78032B78D8DFE803F00233616C01A9F7
:10BAD8003C480BF0DBFA0A2200213A480CF0FEFB46
:10BAE8003C4A3D4B12781860012A0BD002D3022A37
:10BAF8001AD10EE0B0F5FA5FBCBF4FF4FA521A60E3
:10BB0800364A0CE0364A904201DC01321A60354A66
:10BB180005E0354A904201DC01321A60334A1B685D
:10BB28009342C4BF2C4B1A60314B1A68314B2BE03F
:10BB380001A925480BF0AAFA0A22002122480CF094
:10BB4800CDFB244A2C4B12781860012A0BD002D363
:10BB5800022A31D10EE0B0F5FA5FBCBF4FF4FA52B9
:10BB68001A601E4A0CE01E4A904201DC01321A603B
:10BB78001C4A05E01C4A904201DC01321A601B4A4B
:10BB88001B68934218DD1C4B1A6015E001A90F4889
:10BB98000BF07CFA0D4800210A220CF09FFB174B92
:10BBA80009E001A90A480BF071FA094800210A22A4
:10BBB8000CF094FB124B186005B030BDCEB00508F0
:10BBC8003F26002010260020342600204A2C002082
:10BBD800FC2500201C0E00204C26002050DA110005
:10BBE8001FA1070080D1F0085FE316008074D21A05
:10BBF80040260020442C0020642C0020402C0020EB
:10BC0800F825002010B50D4B0D4C1A680D4821463B
:10BC18000BF014FA0C4B0D481A6821460BF00EFA7B
:10BC28000B4B0C481A6821460BF008FA0A4B0B48D4
:10BC38001A682146BDE810400BF000BA4C260020D7
:10BC4800AEA6050810260020642C0020342600200B
:10BC5800402C00204A2C0020F8250020FC2500203C
:10BC68009FED010A704700BF000000009FED010A28
:10BC7800704700BF000000009FED010A704700BF39
:10BC88000000000018B1012801D1034B00E0034B6C
:10BC98001868FDF7F7BC00BF3026002040260020BA
:10BCA80010B9034B18687047024B1868704700BFFB
:10BCB8004C2600204026002010B9034B1868704716
:10BCC800024B1868704700BF642C00203026002003
:10BCD80008B54FF49570FBF7D9FE40F26523C31AF7
:10BCE800584240EB030008BD08B5C620FBF7CEFE5E
:10BCF80040F28D13C21A504240EB020008BD4FF4C7
:10BD0800957040F26521FBF7B3BEC62040F28D1155
:10BD1800FBF7AEBEDCE760EEA00AB7EE007AF0EE05
:10BD2800606A70EE077A40EE006A47EEA70A36EEC0
:10BD3800C77A08B5C7EE200A10EE900A06F0B8FADE
:10BD48000022084B06F008FB0022074B06F052F9C8
:10BD580006F0E4FD07EE900AFDEEE77A17EE900A8A
:10BD68009F3008BD000059400000E03F38B52DED78
:10BD7800028BF7EE008AB0EE608A70EE288A10EE29
:10BD8800900A28EE088A06F093FA08EEA88A00229C
:10BD98000F4B06F0E1FA044618EE100A0D4606F0BD
:10BDA80087FA02460B462046294606F0FFFB00228A
:10BDB800084B06F01FF906F0B1FD07EE900AFDEEFC
:10BDC800E77A17EE900A7730BDEC028B38BD00BFDA
:10BDD800000069400000E03F2DE9F04F884F2DED4D
:10BDE800068B97E80F0091B00CAC103784E80F0071
:10BDF8000FCF05AE0FC697E807004FF6FF7386E82A
:10BE080007009F2077216422F7F773FDA020772190
:10BE180064224FF6FF73F7F76CFD9E2077216422AA
:10BE28004FF6FF73F7F765FD9F20762164224FF6E2
:10BE3800FF73F7F75EFD4FF6FF73782164229F20AA
:10BE4800F7F757FD0020F9F768F99F207721652259
:10BE5800FAF7C8F80C349F2077216422FAF7C2F861
:10BE68000DF12C0A0394F7EE009A4FF00F0B00E047
:10BE78004D460AF1040AF7EE008A9AED009A00246A
:10BE8800B0EE68AA01E0B846354618EE900A06F00A
:10BE98000FFA59A3D3E9002306F05EFA06F03EFD37
:10BEA80008EE900A38EEE98AB0EE490AF0EE480A40
:10BEB800FFF731FFB0EE490AF0EE480A0646FFF7F1
:10BEC80055FFB2B2074683B22CB9104619460F2265
:10BED800F9F7E2F906E0A8B21FFA88F1CDF800B048
:10BEE800F9F7CAFF0134B4F5967FCCD13D46F7EE99
:10BEF800008A002401E045464E4618EE900A06F0F6
:10BF0800D7F93DA3D3E9002306F026FA06F006FD8B
:10BF180008EE900A39EEE88AB0EE490AF0EE480ACF
:10BF2800FFF7F9FEB0EE490AF0EE480A8146FFF73E
:10BF38001DFF1FFA89F2804683B22CB910461946B4
:10BF48000F22F9F7A9F905E0B0B2A9B2CDF800B00F
:10BF5800F9F792FF0134B4F5967FCCD1039B9A454B
:10BF680086D104AD0DF12C0B4FF0000A01E0B84664
:10BF7800B146043595ED009AF7EE008A002401E0F9
:10BF8800B846B14618EE900A06F092F91AA3D3E91A
:10BF9800002306F0E1F906F0C1FC08EE900A38EE3D
:10BFA800CA8AF0EE490AB0EE480AFFF7B4FEB0EECE
:10BFB800480AF0EE490A0646FFF7D8FEB2B207462D
:10BFC80083B22CB9104619462246F9F765F907E0FD
:10BFD8001FFA89F01FFA88F1CDF800A0F9F74CFF95
:10BFE8000134B4F5C87FCBD15D45C0D111B0BDECEB
:10BFF800068BBDE8F08F00BF295C8FC2F528F03FA3
:10C008007CAB0408121A06EE902A081AB8EEE67AF3
:10C0180006EE900AF8EEE67A08B5C7EE277A17EE2C
:10C02800900A06F045F90022044B06F095F9002223
:10C03800034B05F0DFFF06F029FC08BD0000744043
:10C048000000E03F8A1A06EE902A081AB8EEE67A4F
:10C0580006EE900AF8EEE67A08B5C7EE277A17EEEC
:10C06800900A06F025F90022044B06F075F9002223
:10C07800034B05F0BFFF06F009FC08BD000069404E
:10C088000000E03F70B506460D460024610704D560
:10C09800A0B231462A46F9F7FFF80134B4F5A07F7B
:10C0A800F4D170BD70B506460D460024600704D56E
:10C0B800A1B230462A46F9F7EFF80134C82CF5D179
:10C0C80070BD234B1B78012B03D011D3022B3DD11C
:10C0D80023E0204B1A68204B1A60204B1A68204B2B
:10C0E8001A60204B1A68204B1A60204B1A6811E01E
:10C0F800184B1A68184BD2011A60184B1A68184B5B
:10C10800D2011A60174B1A68174BD2011A60174BE5
:10C118001A68D201164B1A6070470E4B0E4A1968FE
:10C12800032391FBF3F111600C4A11680C4A91FB4F
:10C13800F3F111600B4A11680B4A91FBF3F111609E
:10C148000A4A126892FBF3F3094A1360704700BF6A
:10C158001C0E00204C26002040260020642C0020C5
:10C1680030260020402C0020C42500201C2600205A
:10C178005C2C0020014B1868FDF784BA402600208B
:10C1880008B5FFF79EFFBDE80840F3E770B500214A
:10C198000A222748274D284E284C0CF09FF80021EA
:10C1A8000A22286026480CF099F800210A223060FB
:10C1B80024480CF093F800210A22206022480CF051
:10C1C8008DF8224B326818602B682149D31A06EE85
:10C1D800903A2368B8EEE67A06EE903AF8EEE67AF8
:10C1E800C7EE277AFCEEE77A17EE903A9AB20B8000
:10C1F800531C07EE903AB8EEE77ADFED167A67EE51
:10C20800277A154BFCEEE76A16EE901A8AB206EE0C
:10C21800902AB8EEE67A198077EEC77AF5EEC07AFA
:10C22800F1EE10FA01DD01321A80BDE87040A7E78F
:10C23800102600204C260020642C0020402C0020D2
:10C24800342600204A2C0020FC250020F825002058
:10C258002C3A00200000803DC03A00200022F0B5B2
:10C268001346202603254FF02C0C00E02646303ECE
:10C27800F6B217460132092E10F8014B0AD897FB7F
:10C28800F5F605FB16772FB9CE1801F803C07470C0
:10C29800023301E0CC540133092AE7D12022CA54E1
:10C2A800CB1848225A707A229A700022DA70F0BDB0
:10C2B800F0B51F46144B1E78012E8DB005460C466E
:10C2C80020D0A6F1030CDCF1000646EB0C06CEB933
:10C2D8000E4908A80AF0B2FE08A86946FFF7BEFF93
:10C2E8000B496A4604A80AF0A9FEBDF84800F9F708
:10C2F80037FE3846F9F74AFE2846214604AA33464F
:10C30800F9F768FF0DB0F0BDCD250020AEA60508F1
:10C3180012AE050810B501210446F8F7E3FF014BFA
:10C328001C8110BDB80D002008B50021C620FBF700
:10C338009FFB4FF495700021BDE80840FBF798BBC0
:10C34800014B9F221A817047B80D0020002001463A
:10C35800C82240F23F13F8F7D5BF07B50DF1070023
:10C36800FEF733FE9DF807000EBD08B5FFF7F5FF91
:10C378000028FBD108BD30B5044687B010EE100A7E
:10C388000D4605F095FF02460B4601A805490AF03F
:10C3980055FE2046294601AA0023F9F71BFF07B0DE
:10C3A80030BD00BFD8B0050808B5084803F088FAC2
:10C3B8000648022103F055FB0028F9D0034803F092
:10C3C800ABFA07EE900AB8EE670A08BD00200140F4
:10C3D80010B52DED028B9FED098A1924FFF7E4FFB4
:10C3E800013CE4B238EE008A002CF7D19FED040A34
:10C3F80028EE000ABDEC028B10BD00BF0000000053
:10C40800ACC868392DE9F04F994B9A4C5D695F6863
:10C418002DED068B93ED00AAC7B006461AEE100A5A
:10C4280093ED038AD3ED04AAD3ED028A93ED069A1D
:10C4380005F03EFF41EC100BCDE9040108F028FAA5
:10C4480032468D493BA88DED0C0B0AF0F7FDA0682C
:10C4580005F02EFF02460B462BA888490AF0EEFD90
:10C46800E06805F025FF02460B462FA884490AF02C
:10C47800E5FD1AEE900A05F01BFFCDE90A01DDE99A
:10C488000A23804933A80AF0D9FD284605F010FF91
:10C49800CDE90601DDE906237B4937A80AF0CEFD80
:10C4A80018EE900A05F004FF8046894642464B463E
:10C4B800764913A80AF0C2FD18EE100A05F0F8FE36
:10C4C80082468B46524672495B4617A80AF0B6FD6B
:10C4D800DDE904236F491BA80AF0B0FD384605F0D2
:10C4E800E7FE5BA3D3E90023CDE9080105F034FF9B
:10C4F80002460B461FA868490AF0A0FD49EC118BBB
:10C508004BEC10AB08F03CF951A3D3E9002351ECF4
:10C51800100B05F021FF02460B4627A85F490AF0D9
:10C528008DFD19EE100A05F0C3FE0B4602465C4964
:10C5380023A80AF083FDD4ED047AFDEEE77A594981
:10C5480017EE902A0FA80AF079FD0022564BDDE974
:10C558000C0105F001FF06F0E1F905F0A9FE02461D
:10C568000B4643A851490AF069FDB5EEC08AF1EEC1
:10C5780010FADFED4F9A37D5304605F087FE36A31F
:10C58800D3E9002305F0E8FEF1EE487A044617EEF9
:10C59800900A0D4605F08CFE02460B4620462946B9
:10C5A80005F0DAFE02460B462DA1D1E9000105F09F
:10C5B800FDFF06F0B3F99FED3F7A07EE900AF4EE1F
:10C5C800C77AF1EE10FAC6BFC7EEA97A3A4C3B4CCF
:10C5D800F4EEE97AF1EE10FA38DD9FED357A384D50
:10C5E800384CC7EE877A78E01FA3D3E9002350467A
:10C5F800594605F0B1FE044630460D4605F046FEA4
:10C6080015A3D3E9002305F0A7FE02460B462046F2
:10C61800294605F0CBFF06F081F907EE900AB7EE40
:10C62800007AF4EEC77AF1EE10FA46BF67EEA97AFF
:10C63800254C264CF4EEE97AF1EE10FA4CDD9FED2C
:10C648001C7A234D234CC7EE877A46E01C4D44E004
:10C658006666666666A64C401F85EB51B81E194093
:10C66800000000A2941A6D420000000080842E4150
:10C67800DC390020EC370020FAB0050804B10508C1
:10C688000FB105081AB1050824B105082EB105082F
:10C6980039B1050844B105084FB105085AB1050874
:10C6A80065B1050871B10508000034C07EB1050800
:10C6B80000007A4400247449E9B00508E6B005088A
:10C6C8008AB00508F2B00508EFB00508ECB0050817
:10C6D800F5B00508F7B005089D4D17EE900A05F06E
:10C6E800E7FD2A46CDE900013FA89A4902940AF0DD
:10C6F800A5FC994B1A68994B1B689642CCBF00223F
:10C7080001229E42964BD8BF0022DA60954B1B78D7
:10C71800082B40F0AE800220F9F724FD4FF6FF7099
:10C72800F9F734FC1F20F9F71BFC192100238E4A66
:10C738002D20F9F74FFD4FF6FF70F9F727FC002081
:10C748000024F9F70DFC0F20B42132464FF6FF7391
:10C758000094FFF7ADFD0F206E2123462BAAF9F7B1
:10C7680039FDB0206E2123462FAAF9F733FD0F209B
:10C77800382123461BAAF9F72DFDB020382123467E
:10C788001FAAF9F727FD0F205C21234633AAF9F7E2
:10C7980021FD2346B0205C2137AAF9F71BFD0F20A5
:10C7A8004A21234613AAF9F715FDB0204A2123464A
:10C7B80017AAF9F70FFD0F209B21234623AAF9F7A3
:10C7C80009FD0F20842123463FAAF9F703FDB02075
:10C7D8008421234627AAF9F7FDFCB0209B2143AA10
:10C7E8002346F9F7F7FC614B1B68B3F57A7FCCBF9A
:10C7F8004FF4FC604FF47840F9F7C8FB0023A02001
:10C80800B4210FAAF9F7E6FC594B1C78012C0CD07F
:10C8180002D3022C1DD111E04FF6E070F9F7B6FBF8
:10C828004FF48C700221534A10E04FF4FC60F9F782
:10C83800ADFB4FF48C7002214F4A07E04FF6E070D1
:10C84800F9F7A4FB4D4A4FF48C7021460023F9F701
:10C85800C1FC0020F9F79AFB4FF4FC60F9F780FB64
:10C86800FFF7B6FD0F20DC21FFF785FD1F20F9F744
:10C878008DFB3C4B1B789A1FD2B2012A02D90B2B95
:10C8880040F053823E4B1B78023B052B00F24D8251
:10C89800DFE813F006007E00EF004801E6016501BD
:10C8A800DFED387A2AEE27AA1AEE100A05F000FD05
:10C8B8009DED080B8046894607F006FE404653EC7E
:10C8C800102B494605F048FD1DA3D3E9002305F0C8
:10C8D80091FB05F0DBFF9DED080B044607F0F4FE25
:10C8E800404653EC102B494605F036FD02460B46F0
:10C8F80015A1D1E9000105F07BFB05F0C7FF4FF654
:10C90800E0730093054600230520DC213246FFF73B
:10C91800CFFC134BDB6853B11B4B18881B4B4FF4F0
:10C92800784719880097A2B2ABB2F9F7A5FA164B67
:10C938001C60164B4FF6E0701D60F9F711FBF4E12F
:10C948000000000000E063400000000000C05D40FF
:10C95800F5B005088CB10508642C00204C26002091
:10C96800B80D0020CD25002099B10508741A0020C3
:10C978001C0E0020F3AF0508F8AF0508FCAF05084A
:10C98800582C00200000C84228380020CC3A00204B
:10C99800A74B1868A74B32461968FFF733FBA64B1D
:10C9A8001B784FF4FA7292FBF3F307EE903AB8EE65
:10C9B800E79ADFEDA27AF4EE498AF1EE10FAC8BFE1
:10C9C800F0EE498AF5EE408AF1EE10FA48BFF0EE33
:10C9D800678AF4EEC98AF1EE10FA044620D8F4EE1C
:10C9E800E78AF1EE10FA1BDBFDEEC97AFDEEE88A64
:10C9F80017EE901A18EE902A0020FFF723FB904BB1
:10CA0800DB68054653B18F4B18888F4B4FF6FF777D
:10CA180019880097A2B2ABB2F9F72EFA8A4B1D60BB
:10CA2800B4EE498AF1EE10FAC8BFB0EE498AF1EEC9
:10CA3800497AB4EE678AF1EE10FA48BFB0EE678A19
:10CA4800B4EEC98AF1EE10FA00F26F81B4EEE78A0B
:10CA5800F1EE10FAC0F26981FDEEE77ABDEEC99AEF
:10CA6800BDEEC88A17EE900A19EE101A18EE102AB1
:10CA7800AEE06F4B18686F4B32461968FFF7C2FA81
:10CA8800F5EEC0AAF1EE10FA044627DDDDE90A0149
:10CA980059A3D3E9002305F0D1FEF8B158A3D3E98F
:10CAA8000023DDE90A0105F057FC0B4602466749F9
:10CAB800002005F09DFA05F0E9FE614BDB680546AC
:10CAC80053B1604B1888604B4FF6FF771988009771
:10CAD800A2B2ABB2F9F7D0F95B4B1D60DDE90601F4
:10CAE80049A3D3E9002305F0C7FE002800F01D8103
:10CAF800DDE9060140A3D3E9002305F09FFE0028E5
:10CB080000F0138142A3D3E90023DDE9060105F013
:10CB180023FC02460B4600204D4905F069FA05F052
:10CB2800B5FE57E0424B1868424B32461968FFF78A
:10CB380069FA39A3D3E900230446DDE9040105F0C5
:10CB48009BFE50B19DED040B07F0A2FE002251ECB4
:10CB5800100B404B05F000FCD2E0C825D3E030A311
:10CB6800D3E90023DDE9080105F0F6FB2EA3D3E99C
:10CB7800002305F01BFD05F0D1FE2D4B08EE100A31
:10CB880018682C4B32461968FFF73CFADFED327A09
:10CB98004AEE677A2A4BFDEEE77ADB6817EE905A81
:10CBA800044625EAE57553B1264B1888264B4FF6FF
:10CBB800FF7719880097A2B2ABB2F9F75DF9BDEE1D
:10CBC800C88A214B18EE102A1D606FF0B300B421FB
:10CBD800FFF738FA1A4BDB68054653B1194B18882A
:10CBE8001E4B4FF4FC6719880097A2B2ABB2F9F755
:10CBF80043F91A4B96E000BF9A9999999999B93FC8
:10CC08000000000000409F409A9999999999B9BFEE
:10CC18000000000000408F4089B5F81400E3693F28
:10CC280000000000008076401F85EB51B81E1940B7
:10CC38004C260020642C00201C030020000000006B
:10CC4800B80D002028380020CC3A002000006940A8
:10CC580000005940000054C0000048431836002026
:10CC68003B4B187805F012FB02460B460020394969
:10CC780005F09CFC05F052FE08EE100A05F018FBC2
:10CC880041EC100B07F004FEB4EE489AF1EE10FAEE
:10CC9800C8BFB0EE489AB4EEC89AF1EE10FA5BEC51
:10CCA80010AB42D82C4B18682C4B32461968FFF74A
:10CCB800A9F9044619EE100A05F0FAFA41EC100B2E
:10CCC80007F0E6FD5946504659EC108B05F026FE54
:10CCD8009FED237A07EE900AC7EE277A17EE900A9F
:10CCE80005F0E6FA42464B4605F036FB02460B468F
:10CCF80000201C4905F07CF900221B4B05F07AF94D
:10CD080005F0C4FD0546194BDB6853B1184B18886C
:10CD1800184B4FF6FF7719880097A2B2ABB2F9F714
:10CD2800ABF8144B1D60124B1C60134B1B78022B85
:10CD380009D043B14FF6FF7300930520DC2132463A
:10CD48000023FFF7B5FA47B0BDEC068BBDE8F08FBE
:10CD58001C030020000059404C260020642C0020B1
:10CD680000004843000069400000E03FB80D002083
:10CD780028380020CC3A0020582C002010B54FF459
:10CD8800C770FAF783FEDB2805D14FF4C870FAF7AD
:10CD98007DFE84B219E041F2E104214644F201002B
:10CDA800FAF766FE44F20100FAF770FEA04214BFDB
:10CDB80080244FF4007421B24FF4C870FAF758FE7B
:10CDC8004FF4C770DB21FAF753FE204610BD024B23
:10CDD80000221A60704700BF3436002070EEA10AA6
:10CDE80088B030EE010A08B0704770EEE10A88B0EA
:10CDF80030EE410A08B07047F0EE407A20EEA10A02
:10CE080060EE810A47EEA10A88B017EE810A08B0E1
:10CE18007047D0B561EEA17A41EE017A2DED048B11
:10CE280017EE900A88B0B0EE409AF0EE609AF0EEF5
:10CE3800418AB0EE618A05F03BFA002200230646DB
:10CE48000F4605F0F1FCE8B969EE887A49EE287AD0
:10CE580029EE088A17EE900A05F02AFA32463B4670
:10CE680005F0A4FB19EEA88A05F058FD044618EE53
:10CE7800100A05F01DFA32463B4605F097FB05F00F
:10CE88004DFD01E00448044600EE900A00EE104A09
:10CE980008B0BDEC048BD0BD0050C347F0B58E4B35
:10CEA8002DED068B93ED001AD3ED011A8FB0F0EE3D
:10CEB800408AB0EE608A8DED060ACDED070A30EEA5
:10CEC800410A70EEE10A38EE811A78EE211A8DEDEA
:10CED8000C1ACDED0D1A8DED0A0ACDED0B0AFFF7F0
:10CEE80098FF8DED040ACDED050A04AA92E8030027
:10CEF80008AB83E80300DDED099A9DED08AA69EE09
:10CF0800A97A4AEE0A7A17EE900A05F0D1F941ECAF
:10CF1800100B07F043FD51EC100B05F0FFFC09EE78
:10CF2800100A19EE900A05F0C3F904461AEE100A21
:10CF38000D4605F0BDF945EC104B41EC110B07F01F
:10CF48001FFC51EC100B05F0E9FC68EE087A48EE7E
:10CF5800A87AB1EE48AAC8EEA79A604B604D5A6904
:10CF68001B8B6860EA612B8404468AEE27AA85ED4C
:10CF7800009A19EE100AC5ED028A85ED038AC5EDFF
:10CF8800049A85ED05AA05F093F94DA3D3E900238A
:10CF980005F072FCDFED537A002818BFB0EE679AEF
:10CFA800B7EE007A79EE077A37EE497A4E4BC7EE3C
:10CFB800877A1B78033BC5ED067A042B71D8DFE826
:10CFC80003F0032738664F0018EE100A05F070F9D1
:10CFD800044618EE900A0D4605F06AF906460F4613
:10CFE80047EC116B45EC104B07F0CAFB36A3D3E9AD
:10CFF800002351EC100BCDE9004505F0ADF93246A0
:10D00800CDE902013B46394939480AF017F848E0AA
:10D0180019EE900A05F04CF904461AEE100A0D466E
:10D0280005F046F92246CDE900012B463048314942
:10D038002AE019EE100A05F03BF941EC100B07F055
:10D0480027FC00222C4B51EC100B05F085F905F05C
:10D0580065FC05F02DF902460B46254827491EE0D8
:10D0680019EE100A05F024F9064620460F4605F089
:10D078001FF917A3D3E9002305F06EF9CDE90001E4
:10D088001B481F4932463B4609F0D8FF09E017EE16
:10D09800900A05F00DF902460B461548194909F0A2
:10D0A800CDFF134C00230220CA212246F9F792F83B
:10D0B800002323700FB0BDEC068BF0BDAFF30080EA
:10D0C800AE47E17A14AEEF3F6666666666A64C40E8
:10D0D800F6285C8FC2A54C405C360020EC37002057
:10D0E800DC390020A4707D3F582C0020B8B1050819
:10D0F800F8350020D2B10508000034C0E2B10508B7
:10D10800F4B1050810B2050800B560EEA07A40EE4B
:10D11800007A2DED028B17EE900A87B0B0EE408AA8
:10D12800F0EE608A8DED020ACDED030A05F0C0F835
:10D1380041EC100B07F032FC51EC100B05F0EEFB44
:10D14800DFED117A07EE100A78EEA78A38EE078A23
:10D1580068EEA87A48EE087AC7EE277A17EE900AA2
:10D1680005F0A6F841EC100B07F018FC51EC100B79
:10D1780005F0D4FB00EE900A20EE880A60EEA80ABB
:10D1880007B0BDEC028B00BD00000000F0B52DED2E
:10D19800028BDFED3A1A3A4B8DB030EEA17AF0EE01
:10D1A800407AB7EE001A8DED020A83ED001A30EED0
:10D1B800010AC3ED011A31EE671A71EEE01ACDEDDE
:10D1C800030AF0EE470A8DED077A8DED081ACDEDCA
:10D1D800091A8DED060AFFF71CFE8DED000ACDED4C
:10D1E800010A9DE8030004AB83E803009DED058A6E
:10D1F800DDED048A68EE087A48EEA87A17EE900A00
:10D2080005F056F841EC100B07F0C8FB18EE100AB1
:10D2180057EC106B05F04CF8044618EE900A0D46D2
:10D2280005F046F845EC104B41EC110B07F0A8FA55
:10D238003946304655EC104B05F070FB05F038F8D0
:10D2480041EC100B07F09EFA002251EC100B0D4B2D
:10D2580005F082F805F062FB29460646204605F0EF
:10D268005DFB00EE900AF6EE007A60EEA70A00EE8B
:10D27800106A0DB0BDEC028BF0BD00BF00000000CD
:10D28800343A00200000E03FF0EE407A86B020EE0D
:10D29800200A67EE810A06B070472DE9F04F2DEDA0
:10D2A800028B85B0FCF764F810EE105AFCF766F8AC
:10D2B800284610EE104A04F0FBFF804620468946B7
:10D2C80004F0F6FF41EC100B41EC180B07F0FCF8EA
:10D2D80057EC106BB0EE480AF0EE680A07F0F4F964
:10D2E80032463B46404649465BEC10AB05F034F805
:10D2F80005F014FB9FED138A07EE100ADFED127A92
:10D3080057EE087A114C5B46C4ED007A5246404607
:10D31800494605F021F805F001FB07EE900A27EED3
:10D32800888A04AB84ED018A94E8030003E90300CA
:10D33800DDED030A9DED020A05B0BDEC028BBDE8E8
:10D34800F08F00BF0000F04200008C42C43A002079
:10D3580030B53F4B2DED088BD3ED008AD3ED019A04
:10D368003C4BD3ED00AAD3ED01BA3B4B93ED008AB9
:10D3780093ED019A394B93ED00AA93ED01BA38EE7B
:10D38800EA0A79EEEB0A38EE4A1A79EE4B1A93B0AC
:10D398008DED0A0ACDED0B0A8DED0C1ACDED0D1AA7
:10D3A800FFF72AFD8DED000ACDED010A9DE8030087
:10D3B8003AEE6A0A7BEE6B0A04AB38EE681A79EE2D
:10D3C800691A83E803008DED081ACDED091A8DED71
:10D3D8000E0ACDED0F0AFFF70FFD8DED000ACDED1A
:10D3E800010A9DE8030006AB83E803009DED040AEB
:10D3F800DDED050A9DED061ADDED071AFFF709FDBB
:10D408008DED000ACDED010A9DE8030002AD85E827
:10D418000300134B9DED021A93ED000AD3ED010AA8
:10D42800DDED031AFFF7E8FC8DED000ACDED010AEA
:10D438009DE8030012AB03E903006C46DDED110A19
:10D4480085E803009DED100A13B0BDEC088B30BDD4
:10D45800F035002048360020B83A0020483A00202D
:10D4680010380020F7EE007A77EEC07A20EE022A14
:10D4780020EE210A07EEA00AF0EE420A47EE810AE2
:10D4880088B008B070472DE9F0432DED028B924B20
:10D498001B78012B89B08146884646D14FEAC009DE
:10D4A80001291FFA89F92BD809F58065A8B2FAF77E
:10D4B80031FB8A4C0435A8B284ED000AFAF72AFB3E
:10D4C80009F58645A8B284ED010AFAF723FB844CD6
:10D4D800043584ED000AA8B2FAF71CFBA9F5FC4054
:10D4E80084ED010A80B2FAF715FB7E4CA9F5FA40E3
:10D4F800FC3884ED000A80B2FAF70CFB84ED010ACF
:10D5080008F1FF385FFA88F8B8F1010F00F2DF8000
:10D51800A9F57C5080B2FAF7FDFA734CA9F57A594F
:10D5280084ED000AA9F17C09CBE0022B40F0CF8002
:10D538006E4B6F4A1B68012992ED007A00F2AC80AD
:10D5480007EE900AF8EE676A07EE903A46EE877A99
:10D55800BDEEE77A17EE104AA4B207EE104A04F1BE
:10D568008005ED00B8EE478AADB2284637EEC88A86
:10D57800FAF7D0FA0435A8B204F50665EE008DED89
:10D58800020AFAF7C7FAB6B230468DED030AFAF77F
:10D59800C1FA043604F58257B0B28DED040AFE00D4
:10D5A800FAF7B8FAB6B230468DED050AFAF7B2FACC
:10D5B8000436B0B281348DED060AE400FAF7AAFA0F
:10D5C800A4B220468DED070AFAF7A4FA434E0434B4
:10D5D800A0B286ED000AFAF79DFA6C1CE400A4B22A
:10D5E800204686ED010AFAF795FA3D4D0434A0B2BB
:10D5F80085ED000AFAF78EFA7C1CE400A4B22046F6
:10D6080085ED010AFAF786FA364F0434A0B287EDA1
:10D61800000AFAF77FFAD6ED001A96ED012ADDED39
:10D62800020AF0EE408A87ED010A9DED031AB0EE7A
:10D63800480AFFF717FF8DED000ACDED010A9DE8B6
:10D648000300D5ED001A95ED012AB0EE480ADDED8C
:10D65800040A86E803009DED051AFFF703FF8DED28
:10D66800000ACDED010A9DE80300D7ED001A85E810
:10D678000300B0EE480ADDED060A9DED071AB0EE8C
:10D68800682AFFF7EFFE8DED000ACDED010A9DE84F
:10D69800030087E803006C4608F1FF385FFA88F852
:10D6A800B8F1010F13D809F5C1594FEAC9091FFA92
:10D6B80089F94846FAF72EFA0B4C84ED000A09F16D
:10D6C80004091FFA89F0FAF725FA84ED010A09B06E
:10D6D800BDEC028BBDE8F083C9010020B83A0020F8
:10D6E80048360020483A0020F0350020C8250020A0
:10D6F800082600202DE9F04F6E4B2DED048B1C7889
:10D70800012CC7B0054605D006D3022C0CBF302427
:10D71800002402E0002400E010244FF47670FAF7A9
:10D72800B5F907464FF47570FAF7B0F980464FF42B
:10D738007470FAF7D3F9032DC0B21D9040F09480AD
:10D748005D4A5E4924A809F079FCC1B224A8FDF716
:10D758003BFC3B4642465A4924A809F06FFCC1B23B
:10D7680024A8FDF731FC574A544924A809F066FC5F
:10D77800C1B224A8FDF728FC04F1C800FAF7AEF9F5
:10D78800064604F1CC00FAF7A9F9054604F1D000E1
:10D79800FAF7A4F9074604F1D400FAF79FF9AB1B8E
:10D7A80006EE903AB8EEE67A06EE907AF8EEE67A69
:10D7B8002B46C7EE277A324601904349009724A8A2
:10D7C800FDEEE77ACDED027A09F038FCC1B224A863
:10D7D800FDF7FAFB3D4A394924A809F02FFCC1B2EC
:10D7E80024A8FDF7F1FBE820FAF778F90546EC20C4
:10D7F800FAF774F90446F020FAF770F90646F420AF
:10D80800FAF76CF9631B07EE903A06EE906AB8EEE9
:10D81800E77AF8EEE67A2A46C7EE277A01902A498F
:10D828000096234624A8FDEEE77ACDED027A09F0AA
:10D8380005FCC1B224A8FDF7C7FB1D9A022A06D130
:10D84800234924A809F022FC24A8142109E01D9BDF
:10D85800012B40F089821F4924A809F017FC24A84D
:10D868001021FDF7B1FB7FE21D9A012A40F00E81DD
:10D8780004F1C800FAF732F91B9004F1CC00FAF76A
:10D888002DF9074604F1D000FAF728F91B9B1C90E4
:10D89800FF1A06EE907AB8EEE67A06EE900AF8EEEF
:10D8A800E67A0024C7EE277AFDEEE77ACDED1F7AF7
:10D8B800E7E000BF1C0E002020B205081BB20508D7
:10D8C8002AB2050837B205083DB2050887B205082F
:10D8D8008DB20508A2B205081C9B1B9A204601219F
:10D8E80003FB042AFFF7CFFD914B924A186817688B
:10D8F800D3ED018A92ED019A8F4B904AD3F80090AC
:10D90800D3ED019A1368012D209392ED018A7ED1FF
:10D91800F5EEC08AF1EE10FA54BF4FF0000C4FF04C
:10D92800010CB5EEC09ABCF1000F0CBF4FF02B08EC
:10D938004FF02D08F1EE10FA54BF4FF0000E4FF0E3
:10D94800010EF5EEC09ABEF1000F0CBF2B262D2656
:10D95800F1EE10FA54BF00210121B5EEC08A00296A
:10D968000CBF4FF02B0B4FF02D0BF1EE10FA54BFFC
:10D9780000220122002A0CBF2B232D231E93BCF169
:10D98800000F01D0F1EE688ABEF1000F01D0B1EEB0
:10D99800499A09B1F1EE699A0AB1B1EE488A04F0E0
:10D9A80087FCCDE9000118EE900ACDF8088004F054
:10D9B8007FFCCDE90401384604F07AFCCDE9060184
:10D9C80019EE100A089604F073FCCDE90A014846DE
:10D9D80004F06EFCCDE90C0119EE900ACDF838B0D0
:10D9E80004F066FCCDE91001209804F061FC1E9A51
:10D9F800CDE9120118EE100A149204F059FC5246AF
:10DA0800CDE9160124A84E4909F018FB2FE0022D94
:10DA18002ED1FFF79DFC8DED220ACDED230A22AB16
:10DA280093E8030046AB03E90300DDED457AF5EE24
:10DA3800C07AF1EE10FA449805D5F1EE677A17EE40
:10DA4800906A2D2702E017EE906A2B2704F030FC2D
:10DA580002460B463046CDE90023029704F028FC25
:10DA68005246CDE9040124A8364909F0E7FAC6B2BE
:10DA780024A83146FDF7A8FA0120FDF7C3FF0134B9
:10DA8800A4B21F9BA342BFF627AF6AE11D9A022AE0
:10DA980040F06781E820FAF721F81B90EC20FAF7AC
:10DAA8001DF80646F020FAF719F81B9B1C9006EEA5
:10DAB800900AF61AB8EEE68A06EE906AF8EEE67A6A
:10DAC80004F1C800C7EE887AFDEEE77ACDED1E7A3C
:10DAD800FAF704F8064604F1CC00F9F7FFFF074609
:10DAE80004F1D000F9F7FAFFBF1B07EE100A06EEA3
:10DAF800907AF8EEC77AB8EEE67A1B9A1F9087EE0E
:10DB0800277A931B012D06EE903ABDEEC77A88EE70
:10DB1800278A0D4B8DED207AB8EEE67A87EE277AC4
:10DB280083ED007A094B83ED008A40F0D0808FE0C6
:10DB3800B83A002048360020483A0020F035002046
:10DB4800B3B20508EEB20508C82500200826002053
:10DB58001F9A002102FB046220462192FFF793FCE2
:10DB680095ED018AD8ED018AB5EEC08AF1EE10FA7A
:10DB780054BF4FF0000C4FF0010CF5EEC08A9AED3F
:10DB8800019ABCF1000F0CBF2B272D27F1EE10FADC
:10DB980054BF4FF0000E4FF0010EB5EEC09ABEF123
:10DBA800000F0CBF4FF02B0B4FF02D0BF1EE10FABE
:10DBB80054BF002101212868D8F80090DAF8003015
:10DBC80000290CBF2B222D22BCF1000F01D0B1EE91
:10DBD800488ABEF1000F01D0F1EE688A09B1B1EEB2
:10DBE800499A19921A9304F063FBCDE9000118EEE3
:10DBF800100A029704F05CFBCDE90401484604F0E2
:10DC080057FBCDE9060118EE900ACDF820B004F0D4
:10DC18004FFB1A9BCDE90A01184604F049FB199AF3
:10DC2800CDE90C0119EE100A0E9204F041FB219A7D
:10DC3800CDE910014F4924A809F000FAC1B224A87F
:10DC4800FDF7C2F901340120FDF7DCFEA4B205E0BE
:10DC5800494DDFF83481DFF834A10024209BA3422A
:10DC6800BFF676AF0024454D2DE01C9B1B9A20463D
:10DC7800022103FB0426FFF706FC95ED018AB5EEA9
:10DC8800C08AF1EE10FA286803D5B1EE488A2D272C
:10DC980000E02B2704F00CFBCDE9000118EE100A78
:10DCA800029704F005FB3246CDE90401344924A863
:10DCB80009F0C4F9C1B224A8FDF786F90120FDF7DF
:10DCC800A1FE0134A4B21E9BA342CEDA49E0022D84
:10DCD80047D142E01C9B1B9A0121204603FB0425E7
:10DCE800FFF7D1FBFFF734FB8DED220ACDED230AB8
:10DCF80022AB93E8030046AB03E90300DDED457A68
:10DD0800F5EEC07AF1EE10FA449806D5F1EE677A8E
:10DD180017EE908A4FF02D0903E017EE908A4FF026
:10DD28002B0904F0C5FA06460F464046CDE90067C0
:10DD3800CDF8089004F0BCFA2A46CDE90401104950
:10DD480024A809F07BF9C1B224A8FDF73DF90134F4
:10DD58000120FDF757FEA4B200E000241E9BA34259
:10DD6800B8DA084B1D9A1A7047B0BDEC048BBDE8B1
:10DD7800F08F00BF02B30508B83A0020F035002044
:10DD880030B30508C901002048360020483A002071
:10DD9800F0B52DED028B04468DB0002800F0D4803C
:10DDA800714B18890419A4B222B2002A05DB40F28B
:10DDB8003F139A42C8BF1C4600E00024F7F780FAD8
:10DDC800A0B24EF29C71F7F78DFA674B1C81674B36
:10DDD800586804F06DFA5EA3D3E9002304F0BCFA96
:10DDE80004F09CFD624B1860624B1B780A2B0546B9
:10DDF80024B23DD107EE104AF8EEC77A17EE900A22
:10DE080004F056FA5C4B064618680F4604F03EFAD2
:10DE180002460B4650A1D1E9000104F0C7FB0246B7
:10DE28000B463046394604F097FA064628460F4610
:10DE380004F03EFA02460B463046394604F08CFAA6
:10DE480000224E4B04F0B2FB04F068FD04F030FAF7
:10DE580002460B4604A84A4909F0F0F80020F8F7F2
:10DE680081F90520D72104AA0023F8F7B3F96BE05C
:10DE7800444B1888604304F009FA39A3D3E9002316
:10DE880004F094FB04F04AFD3F4B08EE100A1B68AF
:10DE9800FCEEC87A07EE103A17EE905AF8EEC77AF9
:10DEA8003A4B68EE277A1B68FDEEE77AADB217EEBB
:10DEB800906A28460121F618FFF7E5FAFFF748FAB5
:10DEC8008DED020ACDED030A02AC94E8030008AB1D
:10DED80083E80300681C80B20121FFF7D4FAFFF73A
:10DEE80037FA8DED020ACDED030A94E803000CAB76
:10DEF80007EE105A03E90300B8EEC70ADDED080A79
:10DF080038EE400A9DED091ADDED0A1A9DED0B2A3F
:10DF1800FFF7A8FA8DED020ACDED030A94E8030095
:10DF280006AB83E803004FF6FF7300930520002338
:10DF3800DC213246FEF7BCF9154B9DED060A187830
:10DF4800DDED070AFEF7AAFF0DB0BDEC028BF0BDB0
:10DF58007B14AE47E17A843F000000A0D954BD414C
:10DF68000000000000F07340B80D00201C030020E2
:10DF7800AC3A0020CD250020642C00200000F43F9E
:10DF880043B305082C3A0020402C00204C260020E2
:10DF9800582C00202DE9F843461F8846B6B20025C4
:10DFA8000D4F12E008EB040189B23046F7F73CF94F
:10DFB80029F814000A200134FAF766FF062CF1D17B
:10DFC80016350136F22DB6B204D06FF0040407EB13
:10DFD8000509E7E7BDE8F883683A00202DE9F04F26
:10DFE80085B00B1A0193431E9BB20293431C441F36
:10DFF80000F1060901F1FF3A01F1010B9BB20F464E
:10E008001646A4B21FFA89F91FFA8AFA1FFA8BFB7F
:10E0180003938046204651463246F7F73DF920469D
:10E0280039463246F7F738F9204659463246F7F767
:10E0380033F9019B0298E518ADB229463246F7F745
:10E048002BF9404629463246F7F726F9013403985A
:10E0580029463246F7F720F9A4B20A20FAF714FF46
:10E068004C45D7D105B0BDE8F08F2DE9F843461FE0
:10E078008846B6B200250E4F12E008EB040139F8C5
:10E08800142089B23046F7F707F901340A20FAF765
:10E09800FBFE062CF1D116350136F22DB6B204D0AE
:10E0A8006FF0040407EB0509E7E7BDE8F88300BF54
:10E0B800683A00202DE9F0432DED068B70EE007ACA
:10E0C8008DB017EE900AB0EE408A10EE904A20EE1E
:10E0D800009A04F0EDF8064620460F4604F0E8F8EA
:10E0E800F7EE008A41EC100B41EC1A0B06F0ECF944
:10E0F80079EE287A55EC104B17EE900A04F0D8F810
:10E108002246804689462B463046394604F024F993
:10E1180002460B464046494603F06AFF04F0FEFB00
:10E12800B0EE4A0AF0EE6A0A09EE900A38EEC99A89
:10E13800DFED377A89EE299A29EE279A06F0C4FA94
:10E14800304653EC102B394604F006F9044619EE14
:10E15800900A0D4604F0ACF802460B4620462946C4
:10E1680004F024FA00222B4B04F0F6F804F0D6FB56
:10E17800B4EE688ADFED287A284BF1EE10FA0446EF
:10E1880019EE100A08BFB0EE678A1D6804F090F80F
:10E1980002460B4603A8224908F050FF204604F027
:10E1A80087F802460B4606A81E4908F047FF78EE96
:10E1B800287A38EEC88A87EE888A18EE100A04F0A2
:10E1C80077F802460B4609A8174908F037FF0520DB
:10E1D800014603AA0023F7F7FDFF0520142106AA2C
:10E1E8000023F7F7F7FFC820052109AA0023F7F74E
:10E1F800F1FF4FF6E07300930520DC212A46002347
:10E20800FEF756F80DB0BDEC068BBDE8F08300BFF5
:10E218000000484200004940A4707D3F08380020B3
:10E228004CB3050854B305085CB305082DE9F04F55
:10E23800494B2DED048B1D78022D85B080467BD18E
:10E24800464E348A01212046FFF71DF9FFF780F872
:10E258008DED000ACDED010A9DE8030004AB03E94A
:10E26800030028469DED020ADDED030AFEF716FEBF
:10E278003B4B1A683B4B1B6802FB04343A4B1C604F
:10E288003A4BDFED3B7A93ED008A68EE277A5F68B8
:10E2980017EE900A04F00CF8824638468B4604F0D4
:10E2A80007F841EC100B41EC190B06F00DF950463C
:10E2B80053EC102B594604F04FF823A3D3E900235D
:10E2C80003F098FE04F00AFBB0EE490AF0EE690A82
:10E2D800054684B206F0F8F9504653EC102B59461F
:10E2E80004F03AF80B46024619A1D1E9000103F0FF
:10E2F8007FFE04F0F3FAB37C81461FFA80FA1BB95B
:10E30800B08AF18AFFF7B1FE002320465146B37464
:10E31800FFF740FE204651461F22FFF75FFEB0EE92
:10E32800480A00EE907AFFF7C5FE338AB582984412
:10E33800A6F81080A6F8169005B0BDEC048BBDE8D1
:10E34800F08F00BFAFF300800000000000E06340E2
:10E358000000000000C05D40582C0020B80D0020CF
:10E36800402C00204C26002008380020DC390020F2
:10E378000000C842124B1B78022B10B50CD1114B70
:10E388001B78022B08D1104C2078C0B140B2FFF79F
:10E398004DFF0023237010BD0C4C237E23B99F2012
:10E3A800F6F768FF01232376064B1B78022B06D16C
:10E3B800054C94F90000FFF7EBFC0023237010BD17
:10E3C800582C002034380020811A0020B80D002075
:10E3D800034B00201860034B1870FDF753BC00BFB7
:10E3E8003436002034380020034B00201860034BDB
:10E3F80002221A70FDF746BC34360020343800205B
:10E4080037B500242546A0B228213223024601341C
:10E418000095F7F731FDB4F5A07FF4D13EBD2DE9A5
:10E42800F04F2DED088B022897B080468DED070A36
:10E43800B34B05D0032805D0012805D10C2202E0F2
:10E44800092200E00B221A701878F2F745FB042124
:10E4580003914FF00009F3EE0EAA9FEDAABADFED83
:10E46800AABA7DE1A94B1A68A94B1B6802FB0933BC
:10E4780007EE103A01211FFA89F0B8EEC78AFFF7B4
:10E4880002F8FEF765FF8DED080ACDED090A08AD23
:10E4980095E803000AAB83E803009E4B1A6802EB79
:10E4A800C9030EAF19689C4B19600399521812687A
:10E4B8005A60FEF74DFF8DED080ACDED090A95E883
:10E4C80003000CAB83E80300DDED0A9A9DED0BAA6F
:10E4D800DDED0C8A9DED0D9AB0EE690AF0EE4A0A60
:10E4E800B0EE681AF0EE491AFEF786FC8DED080AC0
:10E4F800CDED090A95E80300B0EE691AF0EE4A1A64
:10E5080087E80300B0EE680AF0EE490AFEF781FCDE
:10E518008DED080ACDED090A95E8030010AB83E8F4
:10E5280003009DED0E0ADDED0F0AFEF7EDFD8DED02
:10E53800080ACDED090A95E8030016AA02E90300C6
:10E548009DED100ADDED110A149EFEF7DDFD8DED3F
:10E55800080ACDED090A95E8030087E80300DDED18
:10E568000F0AF5EEC00AF1EE10FA48BFF1EE600AA4
:10E578009DED0E0ACDED0F0AFEF708FE8DED080A97
:10E58800CDED090A08AA92E8030012AB83E803005C
:10E598000798129D03F08CFE5D4B139FD3F800B0D3
:10E5A8005E4BBDEEC87AD3F800A0CDE9040117EEA2
:10E5B800102A58465146FDF725FD07EE10AAF8EE39
:10E5C800C77A07EE10BAB4EEE78AF8EEC77AF1EE2A
:10E5D80010FAB4EEE78A8CBF00220122504B069055
:10E5E800F1EE10FAD4BF002202F00102B8F1020FD6
:10E5F800DA6012D0B8F1030F3ED0B8F1010F68D13C
:10E60800304603F055FE36A3D3E9002303F0A4FEF9
:10E618000022444B03F0EEFC2AE0284603F048FEB3
:10E62800DDE9042304460D462FA1D1E9000103F0DA
:10E63800BDFF02460B462046294603F08DFE2CA35B
:10E64800D3E9002303F088FE04F068F907EE900A86
:10E65800C7EEAA7A17EE900A03F02AFE41EC100BD7
:10E6680006F016F9002251EC100B2F4B03F074FE44
:10E6780004F00CF904462CE018EE100A03F018FE1A
:10E68800044638460D4603F013FE17A3D3E90023CA
:10E6980003F062FEDDE9042303F088FF04F03EF98D
:10E6A80003F006FE14A3D3E9002303F055FE024647
:10E6B8000B462046294603F079FF04F02FF907EEB0
:10E6C800900AB0EE6B7A07EE8B7AFDEEC77A17EEFA
:10E6D800904A002C2ADBC72CA8BFC72427E000BF1C
:10E6E8008716D9CEF753F5BF8FC2F5285CAF4340E4
:10E6F800000000000090704000000080DBC48641EC
:10E70800582C00200000C8C30000C843402C00203B
:10E718004C26002020360020F0350020642C0020F4
:10E72800B80D002000006940000049C00024114BCA
:10E73800DB685BB1104B1888104B1988069B4FF6A5
:10E74800FF759AB2A3B20095F7F796FB0B4B039AA5
:10E758001C600699084B0832196009F101090392F7
:10E76800074B1B884B45BFF67DAE17B0BDEC088B39
:10E77800BDE8F08FB80D002028380020CC3A0020E2
:10E788002C3A00202DE9F0432E4B85B01878F2F78B
:10E79800A3F92D4B0B221A702C4B1C78012C05D099
:10E7A80006D3022C0CBF3024002402E0002400E031
:10E7B8001024274B1B78012B07D104F1C800F9F767
:10E7C8008DF9064604F1D00004E0E820F9F786F94F
:10E7D8000646F020F9F782F900240746DFF8809012
:10E7E8001C4DDFF8808020E007FB046320460121F0
:10E7F8006B61A8F82040FEF746FEFEF7A9FD8DEDF7
:10E80800000ACDED010A9DE8030004AB03E903000B
:10E818000C4B9DED020A1878DDED030AFEF73EFB6E
:10E828006869FDF7EFFD0134A4B2B9F80030A342DE
:10E83800DADA094B02221A70084B00221A7605B060
:10E84800BDE8F083582C0020CD2500201C0E0020A8
:10E85800C9010020EC37002034380020B80D002012
:10E868002C3A0020DC3900201FB5044600214FF067
:10E87800804002F0CCFD2E4B18682E4B1B6800FB25
:10E8880004302D4B1B68984209DB2C4B1B689842BF
:10E8980005DCFAF7F7FE2A4B1868FDF7B3F8FCF722
:10E8A800E3FF284A284B1168526819605A60214BC7
:10E8B8001A68214B1B68D31A06EE903A1C4B1B684A
:10E8C800B8EEE67A06EE903AF8EEE67A0021C7EE60
:10E8D800277AFCEEE77A17EE904AA0B2FEF7D3FD4E
:10E8E800FEF736FD8DED000ACDED010A9DE8030027
:10E8F80004AB03E90300154B9DED020A1878DDED22
:10E90800030AFEF7CBFA124B1868124B1B6824B2A5
:10E9180000FB0430FDF776FD0F4B00224FF08040DE
:10E9280001211A7004B0BDE8104002F070BD00BFAC
:10E93800C42500202836002040260020302600204C
:10E94800F8250020EC370020F0350020582C002056
:10E95800402C00204C260020F125002008B5FFF7A8
:10E9680083FF0A4B1A680A4B1B689A420CDD4FF06A
:10E978008040002102F04BFD064B02221A70064A25
:10E9880000231370054A137608BD00BF28360020FF
:10E998003026002034380020F1250020B80D002052
:10E9A80010B500214FF0804002F031FD0A4B0024E1
:10E9B8001C700A4B20461C70F7F7FEFA084B1868C3
:10E9C800FAF760FE074B084801221A70074B1C70C3
:10E9D800BDE81040F3F7BDB8F12500203836002017
:10E9E80040260020582C0020FC170020CD250020B0
:10E9F80007EE100A034BF8EE477A0022C3ED007ABF
:10EA08005A6070475C36002007EE100A034BF8EE98
:10EA1800477A0022C3ED007A5A6070471038002008
:10EA28000F4B10491A68104B1B68D31A06EE903A20
:10EA38000E4B1B68B8EEE67A06EE903AF8EEE67AE8
:10EA4800C7EE277AFCEEE77A17EE903A9AB20B8077
:10EA5800074B188890422CBF00200120704700BF48
:10EA6800642C00202C3A00204C260020402C00204A
:10EA78004426002013B502AB011D23ED010A054A07
:10EA880089B213F8014B1454013080B28842F8D18E
:10EA98001CBD00BF6A3700202DE9F8431F4F07400F
:10EAA800002F04460D4603DA013F67F00F070137D0
:10EAB800BFB2DFF874804FEAC7091FFA89F94846E0
:10EAC80098ED000A09F10409FFF7D4FF1FFA89F04D
:10EAD80098ED010AFFF7CEFF114B10261B8894FB17
:10EAE800F6F6F6019C42B6B20CD1701980B20D4907
:10EAF8008022FAF769FA00B1FEE721B24FF47F707D
:10EB0800F8F7B6FF0F2F07D17519A8B2054980226B
:10EB1800FAF75AFA00B1FEE7BDE8F8830F00008063
:10EB28002C3A00206A370020EC3700202DE9F0430A
:10EB3800744B2DED028B1888FF2898BF4FF4807016
:10EB480093B0C00007F008FF6F4B0546186028B95E
:10EB58000520B4216D4A2B46F7F73CFB0024694F8A
:10EB68006B4E4FF000086AE0FCF77EFE20464FF43B
:10EB78004141FFF791FF674B1A685B6832600021DB
:10EB880073602046FEF77FFCFEF7E2FB8DED020A7C
:10EB9800CDED030A0DF1080999E803000AAB83E8F3
:10EBA80003005D4B9DED0A1A93ED007AD3ED017ACF
:10EBB800DDED0B1A31EE470A71EEE70A31EE071A5E
:10EBC80071EEA71A8DED0E0ACDED0F0A8DED101A14
:10EBD800CDED111AFEF71DF98DED020ACDED030AF0
:10EBE80099E803000CAB83E80300FF2C4FEAC40349
:10EBF8002B4404D9C3F80080C3F8048003E00C9ABE
:10EC08001A600D9A5A603B8840F23F10604390FBAF
:10EC1800F3F080B24FF4FC630246282100933223BC
:10EC2800F7F72AF93D4B18683D4B1B68C018FAF7EF
:10EC380029FD3C4B1868FCF7E5FE0134A4B23B887B
:10EC4800A34291DA012213464FF4807105A804F01B
:10EC58002DFF354EDFF8F880294605A805F008FA9B
:10EC680008233370314B01241C700020F6F772FC26
:10EC78002F48F2F76EFF3078F1F72EFF2D4B9FEDFE
:10EC88002E8ADFED2E8A1C700024D5ED007AB0EEB6
:10EC9800687A07EEC87A2046FCEEC77A17EE906AC3
:10ECA80003F0F4FA264B002203F056FB03F016FE9D
:10ECB800B6B2A3B2C72E28BFC72687B253B1214B1D
:10ECC800B8F8000019884FF6FF7300933A463346A8
:10ECD800F7F7D2F81B4BC8F8007001340835B4F5C3
:10ECE800807F1E60D1D1184B1868FAF7CBFC114B06
:10ECF80002221A70154B00221A7613B0BDEC028B53
:10ED0800BDE8F0832C3A0020203600201DAB050812
:10ED1800F0350020EC3700205C3600202836002033
:10ED2800C4250020F8250020582C00207B0D002049
:10ED38005817002034380020000016430000C8424D
:10ED48000000F43FCC3A002040260020B80D0020F7
:10ED580028380020F0B5294B294F2A4D2A4E012288
:10ED680085B01A7000243AE0284B1A68336802FB11
:10ED780004336B61264B1C84FCF776FD20464FF468
:10ED88004141FFF789FE234B2A681A606A682046CA
:10ED98005A600021FEF777FBFEF7DAFA8DED000ADC
:10EDA800CDED010A9DE8030004AB03E903001A4B0B
:10EDB8009DED020A1878DDED030AFEF76FF8686921
:10EDC800FDF720FB154B1868154B1B68C018FAF7A0
:10EDD80059FC144B1868FCF715FE0134A4B23B88A3
:10EDE800A342C1DA104B1868FAF74CFC034B022215
:10EDF8001A700E4B00221A7605B0F0BD3438002088
:10EE08002C3A0020EC3700204C260020402C002013
:10EE1800DC390020F0350020582C0020283600204E
:10EE2800C4250020F825002040260020B80D002029
:10EE380038B5FDF79FF90F4B0F4C9F221A810F4BE6
:10EE4800012518782570F1F747FE0D4B00221A604E
:10EE58000C4B1B78072B04D00B2B07D0062B08D1A3
:10EE680002E0BDE8384075E7257038BDBDE8384098
:10EE780088E438BDB80D002034380020582C002014
:10EE880034360020CD2500202DE9F74300258146A2
:10EE98002C46154E154FDFF85C801FE0FCF7E4FCAC
:10EEA80049462046FFF7F8FDD8F800303868C01802
:10EEB800FAF7E8FB0E4B1868FCF7A4FD308895FBC1
:10EEC800F0F080B24FF4FC6300932821024632230D
:10EED800F6F7D2FF05F59E75013403353388A34252
:10EEE800DCDABDE8FE8300BF2C3A0020283600207B
:10EEF800F8250020C425002010B5104C4FF475707B
:10EF0800B4F90010F8F7B4FD0D4B4FF47670B3F96F
:10EF18000010F8F7ADFD40F2D230F8F7B7FDB02891
:10EF280004D040F2D230B021F8F7A2FD2088FFF7D4
:10EF38005FFD034B1888BDE8104065E5C40100205B
:10EF4800C001002000210A2208B509F0C7F9D0F154
:10EF5800010038BF002008BD73B5041D0E46A4B2D9
:10EF68000C2200234FF6E075204601360095F7F78E
:10EF780027F800230C22B1B220460095F7F720F8B5
:10EF88000D4B1B78012B16D10C4E0D4D308829885E
:10EF98000024043080B20C2223460094F7F710F8BE
:10EFA8003088298800940430013180B289B20C225B
:10EFB8002346F7F705F87CBD143600205A360020A2
:10EFC8000C38002008B54FF6FF70F6F7C9FF00208F
:10EFD800F7F7C8F8E12023212C4A0023F7F7FAF8BD
:10EFE800E1204621294A0023F7F7F4F8E1206921B6
:10EFF800264A0023F7F7EEF8E1208C21244A002363
:10F00800F7F7E8F82348FFF79DFF20B12148224988
:10F01800012208F013F84B2023211E4A0023F7F79A
:10F02800D9F81E48FFF78EFF20B11C481A49012263
:10F0380008F004F84B204621184A0023F7F7CAF8CD
:10F048001748FFF77FFF20B115481349012207F041
:10F05800F5FF4B206921124A0023F7F7BBF8114846
:10F06800FFF770FF20B10F480B49012207F0E6FFB8
:10F078004B208C2100230B4AF7F7ACF80A4B188871
:10F088000A4B1988BDE8084066E700BF2DA90508A6
:10F0980068B3050810260020AEA60508342600200F
:10F0A8004A2C0020FC250020443A00200C3A00207D
:10F0B80070B5044600200D461646F7F753F80020B1
:10F0C800F6F764FF4FF4FC60F6F74AFF204629463E
:10F0D80056BB1E4A3346F7F77DF81D48FFF732FF47
:10F0E80020B11B481B49012207F0A8FF04F1700654
:10F0F800B6B230462946164A0023F7F76BF8164889
:10F10800FFF720FF20B114481249012207F096FFAB
:10F118003235ADB220462946104A0023F7F75AF88F
:10F12800304629460C4A07E00D4A0023F7F752F803
:10F1380032350B4AA9B220460023F7F74BF8094BA2
:10F148001888094B1988BDE8704005E76DB30508B4
:10F15800B03A0020C8AA0508203A002075B305086F
:10F1680068AB0508443A00200C3A002030B5144D2D
:10F178009DF80C402C70134D2880134D02FB0400A1
:10F188002980124D80B22880114D2980114D2A8086
:10F19800114A1380114B1880114B1980114B1249D9
:10F1A800E2B21A7000230B7010490A709DF8102003
:10F1B8000134013254430E4A14700E4A137030BDA4
:10F1C800C83B0020A83A0020EA370020443A002033
:10F1D8000C3A002068370020D43A00205A36002024
:10F1E8000C3800200E3A002039360020463A00201C
:10F1F800153600201436002038B5054600200C4688
:10F20800F6F7B0FF0020F6F7C1FE4FF4FC60F6F702
:10F21800A7FE0B48FFF796FE28B1094809490A4B93
:10F22800002207F00BFF284621460023044AF6F780
:10F23800D1FF064B1888064B1988BDE838408BE685
:10F24800503600208BAF05080000F03F443A0020FC
:10F258000C3A0020114B1B68002B70B505460C4674
:10F2680004DA5B420E480F492D2202E00C480D4992
:10F27800202207F0E3FE0020F6F774FF0020F6F7DF
:10F2880085FE4FF4FC60F6F76BFE054A28462146DA
:10F298000023BDE87040F6F79DBF00BF403A00204C
:10F2A800183800207DB305080F4B10B519684FF4C6
:10F2B800E170F8F7FAFB40F23D114FF4E070F8F70F
:10F2C800D7FB0020F6F74EFF0020F6F75FFE4FF45D
:10F2D800FC60F6F745FE054A192064210023BDE8C5
:10F2E8001040F6F777BF00BF403A002085B3050805
:10F2F80008B54FF4E070F8F7C9FB40F23D139842A7
:10F3080005D14FF4E170BDE80840F8F7E7BB0020ED
:10F3180008BD38B5054600200C46F6F723FF002047
:10F32800F6F734FE4FF4FC60F6F71AFE0B48FFF7C9
:10F3380009FE28B109480A490A4B002207F07EFE57
:10F34800284621460023054AF6F744FF064B18884D
:10F35800064B1988BDE83840FEE500BF2C36002072
:10F368008BAF05080000F03F443A00200C3A00201B
:10F3780038B5C501ADB20024601980B2F9F7CCFBED
:10F388000134C0B2FBF710FEA4B24FF47A70F9F75B
:10F398007BFD802CF0D138BD73B5104D00240E20B4
:10F3A800FBF702FE002609E00DF10700FBF70DFE52
:10F3B80020B19DF80730AB550136F6B23306F3D5C8
:10F3C800E00180B205498022F9F7FEFD00B1FEE7B1
:10F3D8000134A4B2B4F5007FE1D17CBD6A370020C6
:10F3E80007EE100AF8EE477A7FB517EE900A02F09A
:10F3F8005FFF02460B4601A8054907F01FFE0A20D9
:10F40800962101AA0023F6F7E5FE07B000BD00BF6C
:10F418008CB30508AFF300800EB403B070470A2818
:10F4280010B5044602D10D20FFF7F9FF064A13680C
:10F438001BB103F8014B136010BD044B1B680BB1E3
:10F448002046984710BD00BFD80D0020CC3B0020B7
:10F4580010B5044601E0FFF7E2FF14F8010B00289D
:10F46800F9D110BD2DE9F04F044685B00D464FF097
:10F478000A0A00E035462078002800F0C4802528D4
:10F4880001D0013467E06078302803D1A0780123E7
:10F49800033407E02D2802D00234002302E0A078CC
:10F4A800022303344FF0000805E00AFB080814F8AB
:10F4B800010BA8F13008A0F13002D2B2092AF4D920
:10F4C8006C2801D04C2803D114F8010B43F0040335
:10F4D800002800F09880602886BFA0F12002D2B2F0
:10F4E80002464F2A3DD006D8432A2DD0442A09D0B7
:10F4F800422A30D133E0552A04D0582A29D0532A39
:10F5080029D101E00A272DE02E1D2F68002500E0F3
:10F5180001357A5D002AFBD104E02020FFF77FFF48
:10F528004D4601E0980704D4454505F10109F4D397
:10F538004D463846FFF78CFF03E02020FFF76FFFAA
:10F5480001354545F9D395E728782E1DFFF767FF64
:10F5580090E7102706E0FFF762FF2E468AE70227AA
:10F5680000E008272E1D442A296804D1002902DA60
:10F57800494243F00803002200E02A46B1FBF7FEA7
:10F5880007FB1E11CDB2092D714607D9782814BF83
:10F598004FF0070C4FF0270C6544EDB230350DF8ED
:10F5A8000250551CBEF1000F02D0102DE5D10F22DC
:10F5B800190705D504A94D192D2105F8101C951C0E
:10F5C80013F0010F0CBF4FF0200B4FF0300B9B07CF
:10F5D8002F4604D508E05846FFF721FF4F46474518
:10F5E80007F10109F7D34F46013D1DF80500FFF764
:10F5F80016FF002DF8D103E02020FFF710FF013798
:10F608004745F9D336E705B0BDE8F08F70B5064D2C
:10F618000C462E68286001E0FFF701FF14F8010B83
:10F628000028F9D12E6070BDCC3B00200FB407B57F
:10F6380004A951F8040B0191FFF714FFBDE80E402F
:10F6480004B070470EB417B505A9084C51F8043B2F
:10F65800206018460191FFF705FF22680023137008
:10F668002360BDE81E4003B0704700BFD80D0020DE
:10F678000EB433B505A9074C51F8043B2568206042
:10F6880018460191FFF7EEFE2560BDE83C4003B047
:10F69800704700BFCC3B002070B51E4604461C488E
:10F6A8001546FFF7C3FF022E1FD0042E25D0012ECA
:10F6B8002AD105E0A15D1748FFF7B8FF013600E041
:10F6C8000026AE42F6DB2020FFF7A9FE002609E05F
:10F6D800A05DA0F12003DBB25E2B88BF2E20FFF7D0
:10F6E8009EFE0136AE42F3DB0EE034F8021B0A48F8
:10F6F800FFF79CFF013DF8D106E054F8041B0748CA
:10F70800FFF794FF013DF8D10A20BDE8704086E676
:10F7180093B305089AB30508A0B30508A6B305086E
:10F7280008B501214FF4807001F07CFA4FF4807025
:10F738000021BDE8084001F075BA43680A6823F063
:10F74800407323F4807313430A7943EA0223436026
:10F75800CA680B6930B51A4384688D68084B2A4318
:10F76800234013434A7943EA420383600B7DC26A0C
:10F77800013B22F47002DBB242EA0353C36230BD9C
:10F78800FDF7FFC000230360037143718360C3600A
:10F798000361012303757047074A084B516810B588
:10F7A8000B4090E8120021438468C068214301435C
:10F7B8000B43536010BD00BF00230140E030FCFF45
:10F7C8000023036043608360C3607047836811B19E
:10F7D80043F0010301E023F00103836070474368AD
:10F7E80023F4400323F400730B43436070474162E2
:10F7F80082627047436823F01F030B4343607047DE
:10F80800044B5A6810B142F4000201E022F40002ED
:10F818005A60704700230140044B5A6810B142F403
:10F82800800201E022F480025A6070470023014000
:10F83800092970B50CB20CD904EB44041E3CC66807
:10F848000725A54026EA0505A34045EA0304C46048
:10F858000AE0066904EB44040725A54026EA0505E5
:10F8680013FA04F42C430461062A0CD80523013A40
:10F878005A43446B1F23934024EA0303914043EA0D
:10F888000102426370BD0C2A12B20CD802EB82024C
:10F89800233A046B1F23934024EA0303914043EA6D
:10F8A8000102026370BD02EB8202413AC46A1F235F
:10F8B800934024EA0303914043EA0102C26270BD07
:10F8C800836843F08043836070478068C0F380504A
:10F8D8007047836811B143F4806301E023F48063C7
:10F8E80083607047836811B143F0020301E023F09D
:10F8F8000203836070474368013923F4604343EA95
:10F90800413343607047436811B143F4006301E039
:10F9180023F4006343607047C06C80B27047014BAA
:10F928001868704708230140836811B143F4807355
:10F9380001E023F4807383607047836811B143F456
:10F94800007301E023F4007383607047044B5A6826
:10F9580010B142F4005201E022F400525A6070479C
:10F9680000230140092970B50CB20CD904EB4404FA
:10F978001E3CC6680725A54026EA0505A34045EABA
:10F988000304C4600AE0066904EB44040725A540A3
:10F9980026EA050513FA04F42C430461836BC3F3C8
:10F9A8000154121B0232D2B202EB82021F2494408D
:10F9B80023EA040391400B43836370BD836B0139D1
:10F9C80023F4401343EA01538363704782B0002352
:10F9D80001930190019BCB180193019B1A6002B01F
:10F9E8007047836823F470230B43836070478368F0
:10F9F80023F440130B4383607047836843F4800308
:10FA0800836070478068C0F380507047436811B1C5
:10FA180043F4806301E023F48063436070474368E4
:10FA280011B143F4805301E023F4805343607047DD
:10FA380082B0002301930190019B28335B18019346
:10FA4800019B186880B202B070470123C9B213FA4B
:10FA580001F143680AB1194301E023EA0101416059
:10FA68007047036819420CBF002001207047C94342
:10FA7800016070474368006810EA112007D001222E
:10FA8800C9B212FA01F119420CBF002001207047D7
:10FA98006FEA112101607047036823F001030360D6
:10FAA8000023036043608360C360036121234361D3
:10FAB8002C4B98421CD02C4B984220D02B4B984270
:10FAC80025D02B4B98422AD02A4B98422FD02A4B2C
:10FAD800984233D0294B984237D0294B984204D1C9
:10FAE8004FF03D5243F8AC2C7047264B984203D157
:10FAF8003D2243F8082C7047234B984204D14FF419
:10FB0800746243F8202C7047204B984204D14FF47C
:10FB1800741243F8382C70471D4B984204D14FF0AB
:10FB2800746243F8502C70471A4B984203D11A4A12
:10FB380043F8642C7047194B984203D1184A43F88C
:10FB48007C2C7047174B984203D1174A43F8942CE2
:10FB58007047164B984204BF4FF03D5243F8AC2C07
:10FB6800704700BF106002402860024040600240B9
:10FB7800586002407060024088600240A060024005
:10FB8800B8600240106402402864024040640240A9
:10FB980058640240706402403D00002088640240BE
:10FBA800400F0020A064024000003D20B8640240DD
:10FBB8000268134B10B51340CC680A6822434C699D
:10FBC80022438C692243CC6922430C6A22434C6A43
:10FBD80022438C6A22434C6B22438C6B224313438F
:10FBE800036042690C6BCB6A22F00702234313437C
:10FBF80043610B6943604B6883608B68C36010BDC9
:10FC08003F801CF00023036043608360C36003618E
:10FC180043618361C361036243628362C3620363B6
:10FC2800436383637047036811B143F0010301E044
:10FC380023F0010303607047036811B143F40043E4
:10FC480001E023F4004303607047036811B143F0F7
:10FC5800200301E023F020030360704741607047F0
:10FC6800406880B27047036812B143F4002301E092
:10FC780023F40023036001617047036811B143F462
:10FC8800802301E023F48023036070470AB10161F7
:10FC98007047C16070470068C0F3C0407047006893
:10FCA80000F001007047406900F0380070470A4AC8
:10FCB8000A4B10B50A4CA04288BF13468A004CBFB5
:10FCC8005B681B6821F0F02121F0821119420CBFFA
:10FCD8000020012010BD00BF006402400060024007
:10FCE8000F64024010B5084B084A094CA04288BF6F
:10FCF800134611F0005F21F0F02121F0821114BFAA
:10FD0800D960996010BD00BF0060024000640240E5
:10FD18000F6402400B0607D5436912B143F0800314
:10FD280001E023F080034361802909D001F01E011E
:10FD3800036812B119430160704723EA01010160A9
:10FD48007047124B124A10B5124CA0428CBF144691
:10FD58001C4621F0F02323F0C3132BB1026802F0F4
:10FD68001E0202EAD12202E0426902F08002880003
:10FD78004CBF6368236821F0F02121F082101840FD
:10FD880002D0101C18BF012010BD00BF0060024047
:10FD9800006402400F64024010B5084B084A094C41
:10FDA800A04288BF134611F0005F21F0F02121F036
:10FDB800821114BFD960996010BD00BF0060024075
:10FDC800006402400F640240044B00221A605A602B
:10FDD8009A60DA60024A5A61704700BF003C0140ED
:10FDE800FFFF7F00837910B5002B29D01A4B0168DB
:10FDF8001C68CA4314401C605C6822405A6002793F
:10FE080002F1804202F59E321468214311600268B3
:10FE18009C68D1430C409C60DC682140D9604179E2
:10FE2800102906D1996811439960D9680A43DA60A4
:10FE380010BD01F1804303F59E3319680A4308E0B9
:10FE48000379016803F1804303F59E331A6822EAB7
:10FE580001021A6010BD00BF003C014000230C22C3
:10FE680003600371427183717047024B1A69024340
:10FE78001A617047003C0140034B5B6918420CBF94
:10FE880000200120704700BF003C0140014B586131
:10FE9800704700BF003C0140054B1A685B6903408E
:10FEA80004D010420CBF002001207047184670474C
:10FEB800003C0140014B5861704700BF003C0140C5
:10FEC8004FF0204318B943F2DB021A6003E043F213
:10FED800D20243F820204FF02042411C6FF07043BB
:10FEE80042F8213002F5827242F82030704770B52E
:10FEF80084684568C368C16A026825431D4303696D
:10FF08001D4343691D4383691D43C3691D43036A38
:10FF18001D43436A1D43836A1D43036B0D431D4301
:10FF28004FF02043082C43F8225005D153F82240C3
:10FF380044F0400443F82240436B9E691D683543F2
:10FF48005E6845EA06159E6845EA0625DE6845EAC4
:10FF580006451E695B6945EA0655541C45EA036572
:10FF68004FF02043B1F5804F43F8245010D1836BF4
:10FF7800986919680143586841EA0011986841EA8C
:10FF8800002118695B6941EA005141EA036101E017
:10FF98006FF07041014B43F8221070BD040100A0BE
:10FFA800022242604FF480524262416B4FF4005289
:10FFB80010B5826200230F22FF2403608360C360B0
:10FFC800036143618361C3610362C36203630A60BF
:10FFD8004A608C60CA600A614A618B61816B0A6001
:10FFE8004A608C60CA600A614A618B6110BD4FF03B
:08FFF800204321B153F8202041
:020000040801F1
:1000000042F0010203E053F82010024A0A4043F88C
:1000100020207047FEFF0F0010280CBF064B074B37
:100020004FF040024FF0180119605A604FF0FC3257
:100030009A60DA60704700BF600000A0800000A0F6
:1000400030B5836844681C43C36844F008041C430B
:1000500003691C43436944EA4324836944EA433403
:10006000C36999685A68090441EA02211A68DB6881
:10007000114341EA0361036A9A685D68120442EA27
:1000800005221D68DB682A4342EA03620368102BDD
:100090000CBF034B034B1C609960DA6030BD00BF9E
:1000A000600000A0800000A010230360C26900234C
:1000B00043608360C360036143618361FC23136019
:1000C00053609360D360026A136053609360D3609F
:1000D000704741B110280CBF074B084B1A6842F01B
:1000E00004021A60704710280CBF034A034A044BED
:1000F00011680B4013607047600000A0800000A0F2
:10010000FBFF0F0041B110280CBF084B084B1A68C9
:1001100042F040021A60704710280CBF034A044A9C
:10012000044B11680B401360704700BF600000A0D3
:10013000800000A0BFFF0F00102802D1024B5869B9
:100140007047024B58697047600000A0800000A013
:10015000054B18221A6000225A604FF0FC329A6058
:10016000DA601A61704700BFA00000A0026843680F
:1001700042F0100242EA4322836842EA4332144BBF
:1001800010B51A60C26891685468090441EA0421F4
:100190001468D268214341EA02629A600269916858
:1001A0005468090441EA04211468D268214341EAF1
:1001B0000262DA60426991685068090441EA0021EC
:1001C0001068D268014341EA02621A6110BD00BFA3
:1001D000A00000A0C2680023036043608360FC238A
:1001E000136053609360D36002691360536093603F
:1001F000D3604269136053609360D3607047054BCE
:1002000018B11A6842F0040202E01968024A0A4072
:100210001A607047A00000A0FBFF0F0062B1102819
:1002200001D10E4B03E0B0F5807F03D10C4B5A682F
:10023000114311E00B4BFAE7102804D1074B5A6821
:1002400022EA010108E0B0F5807F0CBF044B054BAA
:100250005A686FEA0101114059607047600000A0C0
:10026000800000A0A00000A0102801D1064B04E0EF
:10027000B0F5807F0CBF054B054B5B680B420CBF94
:1002800000200120704700BF600000A0800000A097
:10029000A00000A0102804D1074B5A6822EA0101EF
:1002A00008E0B0F5807F0CBF044B054B5A686FEA3D
:1002B0000101114059607047600000A0800000A05B
:1002C000A00000A0102801D1084B04E0B0F5807F09
:1002D0000CBF074B074B5B6813EA010004D013EA1D
:1002E000D1010CBF00200120704700BF600000A0BA
:1002F000800000A0A00000A0102804D1084B5A687C
:1003000022EAD10109E0B0F5807F0CBF054B064B16
:100310005A684FEAD10122EA01015960704700BFD3
:10032000600000A0800000A0A00000A008B52C4B39
:10033000984205D10120014600F048FC012048E028
:10034000284B984205D10220012100F03FFC0220F9
:100350003FE0254B984205D10420012100F036FCF6
:10036000042036E0214B984205D10820012100F0FD
:100370002DFC08202DE01E4B984205D110200121B4
:1003800000F024FC102024E01A4B984205D12020D4
:10039000012100F01BFC20201BE0174B984205D1E7
:1003A0004020012100F012FC402012E0134B984243
:1003B00005D18020012100F009FC802009E0104BCC
:1003C00098420BD14FF48070012100F0FFFB4FF4F5
:1003D00080700021BDE8084000F0F8BB08BD00BFF8
:1003E000000002400004024000080240000C0240ED
:1003F000001002400014024000180240001C02409D
:10040000002002402DE9F0470023D1F800801A4671
:100410004FF0010C03270CFA02F404EA0805A54288
:100420002ED1066817FA03F4E443264006600E79DD
:10043000D0F8009006FA03FA013E4AEA0909012EB3
:10044000C0F8009014D8866891F805902640866020
:10045000866809FA03F949EA06068660466826EACC
:10046000050545608D7946689540ADB235434560D8
:10047000C5682C40C460CC79C5689C402C43C460DE
:1004800001320233102AC6D1BDE8F0874FF6FF7360
:1004900003600023037143718371C371704782B09D
:1004A0004FF480330193019B0B430193019BC36184
:1004B000C161019BC361C3690193C369019302B028
:1004C0007047036919420CBF002001207047006982
:1004D00080B27047436919420CBF00200120704769
:1004E000406980B2704701837047418370470AB109
:1004F00001837047418370474161704743694B40B6
:100500004361704701F00703C908083130B59B000B
:1005100050F821500F249C4025EA040440F8214063
:1005200050F8214012FA03F31C4340F8214030BD3B
:1005300008B5134B984207D14FF40010012100F089
:1005400069FB4FF4001014E00E4B984207D14FF4B2
:100550008000012100F05EFB4FF4800009E00A4BAF
:1005600098420BD14FF40000012100F053FB4FF4EF
:1005700000000021BDE8084000F04CBB08BD00BFF2
:100580000054004000580040005C00407FB5044625
:10059000868868460D4600F06DFA02992C482B6853
:1005A00026F03F063604B1FBF0F0360C80B206436D
:1005B000A680228822F001021204120C2280254A11
:1005C00093420AD85B00B1FBF3F301309BB280B2D7
:1005D0002084032B98BF042321E0EE884BF6FF72A2
:1005E000964205D103225343B1FBF3F39BB206E0DD
:1005F00019225343B1FBF3F39BB243F480431A0532
:100600004FF4967208BF43F0010350434FF47A72DF
:1006100090FBF2F0013080B243F400432084A383C6
:1006200023886989AA889BB243F001032380238829
:1006300023F4816323F002031B040A431B0C1343BE
:100640009BB223802A89AB8913439BB223817FBD50
:1006500040420F00A086010041F28833036000236E
:1006600083804BF6FF72038143814FF48043C28045
:1006700083817047038819B19BB243F0010303E003
:1006800023F001031B041B0C03807047038819B17E
:100690009BB243F4807303E023F480731B041B0CB0
:1006A00003807047038819B19BB243F4007303E0E1
:1006B00023F400731B041B0C0380704712B141F03C
:1006C000010101E001F0FE0101827047038819B1C8
:1006D0009BB243F4806303E023F480631B041B0C90
:1006E0000380704783899BB201F0FE0123F0FE0373
:1006F0000B4383817047838919B19BB243F0010397
:1007000003E023F001031B041B0C83817047038863
:1007100019B19BB243F0400303E023F040031B04F4
:100720001B0C03807047038829B16FEA43436FEACB
:1007300053439BB201E05B045B0C0380704703886A
:1007400019B99BB243F0800303E023F080031B043C
:100750001B0C03807047B1F5804F838B04D023F4CA
:1007600080431B041B0C02E09BB243F48043838351
:100770007047B1F5006F038803D19BB243F4006367
:1007800003E023F400631B041B0C03807047B1F5E6
:10079000005F038803D19BB243F4005303E023F4CA
:1007A00000531B041B0C03807047038819B19BB2D4
:1007B00043F0100303E023F010031B041B0C038021
:1007C000704701827047008AC0B27047038819B130
:1007D0009BB243F4805303E023F480531B041B0CAF
:1007E00003807047B1F5006F038803D19BB243F4D7
:1007F000006303E023F400631B041B0C03807047B9
:10080000038819B19BB243F0200303E023F02003D7
:100810001B041B0C03807047008BC0F3072070473C
:10082000838819B19BB243F4006303E023F40063AF
:100830001B041B0C83807047838819B19BB243F45F
:10084000805303E023F480531B041B0C8380704708
:1008500082B0002301930190019BCB180193019B6F
:10086000188880B202B0704783889BB20AB11943DE
:1008700001E023EA010181807047838A008B9BB2EB
:1008800043EA0040084020F07F40431A584240EBC2
:1008900003007047838A008B9BB243EA004020F03C
:1008A0007F40704782B00023009301930B0F0190AB
:1008B0000093009B21F07F4113B1019B143302E0B0
:1008C000019B090C18330193019B1B6819420CBF53
:1008D0000020012002B07047C94389B2818270476D
:1008E0008388808A80B208409BB206D001F0E06124
:1008F00013EA11410CBF002001207047C94389B29F
:10090000818270470A4B1A6842F001021A60002285
:100910009A60196821F0847121F4803119600549C9
:100920005960196821F480211960DA60704700BFAE
:100930000038024010300024024B00221A70187058
:10094000704700BF02380240034B1A6822F0F802D9
:1009500042EAC0021A60704700380240014B18603A
:10096000704700BF00004742064B002201281A7062
:100970001A7002D0042804D101E0187070470522D3
:100980001A70704770380240014B1860704700BF02
:10099000800E4742014341EA821200995B08013B05
:1009A00042EA016141EA0341014B5960704700BFCF
:1009B00000380240014B1860704700BF600047429A
:1009C0008001034B40EA0171C3F88410704700BFF7
:1009D00000380240014B1860704700BF6800474272
:1009E000014B1860704700BF4C004742034B9A68A8
:1009F00022F0EC6202430A439A60704700380240DA
:100A0000034B9A6822F0784202430A439A60704787
:100A100000380240034B9A6822F0030202439A60B6
:100A2000704700BF00380240024B986800F00C008D
:100A3000704700BF00380240034B9A6822F0F00272
:100A400002439A60704700BF00380240034B9A6827
:100A500022F4E05202439A60704700BF003802401F
:100A6000034B9A6822F4604242EAC0029A607047DF
:100A7000003802401E4B9A6802F00C02042A10B59E
:100A800003D0082A03D01B4B18E01B4B16E0596813
:100A90005A6811F4800F596814BF174B154B02F0B8
:100AA0003F02B3FBF2F3124A5268C2F30142C1F3B0
:100AB000881101324B435200B3FBF2F30C4903603F
:100AC0008B680E4A0468C3F30313D35C34FA03F350
:100AD00043608C68C4F38224145D33FA04F48460A8
:100AE0008968C1F34231525CD340C36010BD00BF7E
:100AF000003802400024F40000127A003403002081
:100B000000F44073B3F5407F084B08D1996820F09A
:100B1000704221F4F81122F440720A439A601A6F6D
:100B2000000542EA10501867704700BF00380240C5
:100B3000014B1860704700BF3C0E4742014B1860E4
:100B4000704700BF400E4742014B1860704700BF1E
:100B50005C014742044B1A6B09B1104301E022EAE1
:100B600000001863704700BF00380240044B5A6B06
:100B700009B1104301E022EA00005863704700BF4A
:100B800000380240044B9A6B09B1104301E022EA9D
:100B900000009863704700BF00380240044B1A6C95
:100BA00009B1104301E022EA00001864704700BF59
:100BB00000380240044B5A6C09B1104301E022EAAC
:100BC00000005864704700BF00380240044B1A69A7
:100BD00009B1104301E022EA00001861704700BF2C
:100BE00000380240044B5A6909B1104301E022EA7F
:100BF00000005861704700BF00380240044B9A69FA
:100C000009B1104301E022EA00009861704700BF7B
:100C100000380240044B1A6A09B1104301E022EA8D
:100C200000001862704700BF00380240044B5A6A47
:100C300009B1104301E022EA00005862704700BF8A
:100C400000380240044B1A6D09B1104301E022EA5A
:100C500000001865704700BF00380240044B5A6D11
:100C600009B1104301E022EA00005865704700BF57
:100C700000380240044B9A6D09B1104301E022EAAA
:100C800000009865704700BF00380240044B1A6EA0
:100C900009B1104301E022EA00001866704700BF66
:100CA00000380240044B5A6E09B1104301E022EAB9
:100CB00000005866704700BF00380240044B1A78A5
:100CC00009B1104301E022EA00001870704700BF2C
:100CD0000D3802404309012B074A01D1136803E094
:100CE000022B0CBF136F536F00F01F0033FA00F09C
:100CF00000F00100704700BF0038024007B5002334
:100D000001933120FFF7E6FF019B01330193019B23
:100D1000B3F5A06F01D00028F3D03120FFF7DAFF40
:100D2000003018BF01200EBD024B5A6F42F0807296
:100D30005A67704700380240034BDB6818420CBF0B
:100D400000200120704700BF00380240014B18709E
:100D5000704700BF0E38024008B5154B98420BD1C2
:100D600001214FF48050FFF761FF4FF480500021C4
:100D7000BDE80840FFF75ABF0E4B984207D14FF429
:100D800080400121FFF746FF4FF4804009E00A4B05
:100D900098420BD14FF400400121FFF73BFF4FF485
:100DA00000400021BDE80840FFF734BF08BD00BF88
:100DB0000030014000380040003C00400B880288B1
:100DC00010B54C8823438C882343CC8823430C895B
:100DD00023434C8923438C892343CC8902F4415219
:100DE000234313439BB20380838B23F400631B04D0
:100DF0001B0C83830B8A038210BD838B23F47B63DC
:100E000023F00F031B041B0C8383022303848B68D2
:100E1000F0B5858B022BADB238D0294A8E88946804
:100E2000002E14BF02260126240203D5946824F460
:100E300000049460D2F88440D2F884705268DFF8DD
:100E400084C002F03F02BCFBF2F2C4F388145443A6
:100E5000C7F30272B4FBF2F4CA88B2F5007F4FF018
:100E60000A0201D1240A02E07601B4FBF6F46243DF
:100E7000B2FBF3F305330A229BB2B3FBF2F303F0A8
:100E800001021202C3F34F0392B200E000229C1E43
:100E9000A4B2FE2C28BF0022CC8828BF0223134313
:100EA00023439BB203840B884A882B4343F400639B
:100EB00013438A8813438A8913439BB28383F0BD0B
:100EC0000038024000127A000023038043808380B0
:100ED000C380038143818381C381072303827047D9
:100EE00000230222038043808380C3808260838149
:100EF0007047038819B19BB243F0400303E023F02D
:100F000040031B041B0C03807047838B19B19BB2F9
:100F100043F4806303E023F480631B041B0C83838E
:100F20007047038823F400631B041B0C03800388B1
:100F30009BB20B4303807047B1F5804F038803D108
:100F40009BB243F4804303E023F480431B041B0C57
:100F5000038070474FF6FF639942038803D09BB22A
:100F600043F4807303E023F480731B041B0C0380A1
:100F70007047838819B19BB243F0040303E023F068
:100F800004031B041B0C83807047838819B19BB238
:100F900043F0100303E023F010031B041B0C8380B9
:100FA0007047838B23F47B6323F00F031B041B0C1C
:100FB0008383022303840B88828BB3F5007F10B5F3
:100FC00092B205D0002B0CBF4FF48073002301E0D8
:100FD0004FF480734C8822438C88898942F40062E4
:100FE00022430A4392B21343838310BD808980B2A7
:100FF000704781817047038819B19BB243F4005355
:1010000003E023F400531B041B0C03807047038888
:101010009BB243F4805303807047012902D0008BB8
:1010200080B27047808A80B27047008A80B2704771
:1010300083889BB20AB1194301E023EA0101818050
:101040007047090901238B409BB21AB1828892B282
:10105000134303E0828892B222EA0303838070473D
:10106000038919420CBF002001207047C94389B28F
:101070000181704710B584880089012301F00F02B7
:1010800080B213FA02F21040A4B205D009098B40D5
:101090001C420CBF0020012010BD01F00F010123F4
:1010A0008B40DB439BB20381704700BF08B5012131
:1010B0004FF48040FFF7BAFD4FF480400021BDE8B7
:1010C0000840FFF7B3BD014B18607047003801407E
:1010D00001F0030289080A4B023130B5920053F83F
:1010E00021500F24944025EA040443F8214053F88A
:1010F000214010FA02F2144343F8214030BD00BFF2
:1011000000380140014B1860704700BFDC002742E7
:10111000014B1860704700BF00042742024B186A59
:10112000C0F30020704700BF0038014030B5048C88
:1011300024F001042404240C0484058B048CADB237
:10114000A4B225F0F305154324F00A0445EA03157B
:1011500044F00104ADB20C430583048430BD30B5C6
:10116000048C24F010042404240C0484048B058CC7
:1011700024F44074ADB22405240D25F0A00544EA02
:10118000022445F0100544EA033445EA0115A4B2EF
:10119000ADB20483058430BD08B5474B984205D1F4
:1011A00001200146FFF742FD01203DE0B0F1804FF4
:1011B00005D101200146FFF72DFD012076E03F4BD0
:1011C000984205D102200121FFF724FD02206DE0A5
:1011D0003B4B984205D104200121FFF71BFD042061
:1011E00064E0384B984205D108200121FFF712FD39
:1011F00008205BE0344B984205D110200121FFF715
:1012000009FD102052E0314B984205D120200121E8
:10121000FFF700FD202049E02D4B984209D1022024
:101220000121FFF703FD02200021BDE80840FFF780
:10123000FDBC284B984207D14FF480300121FFF7C5
:10124000F5FC4FF48030EFE7234B984207D14FF481
:1012500000300121FFF7EAFC4FF40030E4E71F4BB8
:10126000984207D14FF480200121FFF7DFFC4FF4B3
:101270008020D9E71A4B984205D140200121FFF781
:10128000C9FC402012E0174B984205D18020012173
:10129000FFF7C0FC802009E0134B98420BD14FF4BC
:1012A00080700121FFF7B6FC4FF480700021BDE88B
:1012B0000840FFF7AFBC08BD00000140000400403B
:1012C00000080040000C00400010004000140040E6
:1012D000000401400040014000440140004801403A
:1012E00000180040001C0040002000401C4A0388F9
:1012F00090429BB212D002F5806290420ED0B0F1C3
:10130000804F0BD0A2F58032904207D002F5806268
:10131000904203D002F58062904203D14A8823F0C4
:10132000700313430F4A904208D002F58062904246
:1013300004D023F440730A899BB2134303804B68A3
:10134000C3620B880385064B984203D003F5806384
:10135000984201D18B7A038601238382704700BFB4
:1013600000000140001000404FF0FF3343600023B5
:1013700003800381438083727047018582827047B6
:10138000038823F070031B041B0C0B43038070477E
:1013900041627047C1627047406A7047008D80B2F9
:1013A0007047038819B19BB243F0020303E023F0B6
:1013B00002031B041B0C03807047038819B19BB206
:1013C00043F0040303E023F004031B041B0C03801D
:1013D0007047038819B19BB243F0800303E023F008
:1013E00080031B041B0C03807047038823F0080351
:1013F0001B041B0C038003889BB20B4303807047C4
:10140000038823F440731B041B0C038003889BB2E6
:101410000B4303807047038819B19BB243F001036B
:1014200003E023F001031B041B0C03807047038CB3
:1014300023F001031B041B0C038470B5038C848808
:10144000028B0D884E8822F073021204120C2A437C
:101450008D8923F002031B0435431B0CADB22B43D3
:101460000E4DA842A4B203D005F58065A8420ED166
:10147000CD894E8A23F008032B438D8823F0040383
:101480002B430D8A354324F44074ADB22C43848041
:1014900002838A684263038470BD00BF000001407C
:1014A000038C23F010031B041B0C0384038C828821
:1014B00030B5048B0D8824F4E6442404240C23F076
:1014C000200344EA05241B048D891B0C43EA051301
:1014D0004D8843EA0513134DA84292B2A4B29BB2C1
:1014E00003D005F58065A84215D1CD8923F080038E
:1014F0009BB243EA05134FF6BF751D408B8845EA42
:1015000003130D8A22F4406242EA85024D8A42EAC0
:1015100085029BB292B282808A68048382630384CC
:1015200030BD00BF00000140038C23F480731B0416
:101530001B0C0384038C828830B5848B0D8824F0C7
:1015400073042404240C23F400731B042C438D899E
:101550001B0C43EA05234D8843EA0523124DA8429C
:1015600092B29BB203D005F58065A84215D1CD8912
:1015700023F400639BB243EA05234FF6FF351D4079
:101580008B8845EA03230D8A22F4405242EA051271
:101590004D8A42EA05129BB292B282808A688483A5
:1015A000C263038430BD00BF00000140038C23F4FC
:1015B00080531B041B0C0384038C30B58488828BFE
:1015C0000D8822F4E6421204120C23F4005342EA7E
:1015D00005221B048D891B0C43EA05334D8843EA21
:1015E00005330B4DA842A4B292B29BB203D005F5CD
:1015F0008065A84205D10D8A24F4804444EA85140C
:10160000A4B2848082838A680264038430BD00BFF0
:101610000000014000230380438083808360838136
:10162000C38103824382704730B5058C0124ADB27B
:101630008C4025EA040400F11803048409B1082948
:1016400007D149084FF68F70CC582040C850C85871
:101650000AE00439C1F34E0148F6FF70CC5820402F
:10166000C8501202C85892B20243CA5030BD4163FA
:10167000704781637047C163704701647047038B93
:1016800023F070031B041B0C0B4303837047038B75
:1016900023F4E0431B041B0C43EA01239BB20383A6
:1016A0007047838B23F070031B041B0C0B43838355
:1016B0007047838B23F4E0431B041B0C43EA012394
:1016C0009BB283837047038B23F008031B041B0C1E
:1016D0000B4303837047038B23F400631B041B0C31
:1016E00043EA01239BB203837047838B23F00803F3
:1016F0001B041B0C0B4383837047838B23F4006311
:101700001B041B0C43EA01239BB283837047038BAA
:1017100023F004031B041B0C0B4303837047038B50
:1017200023F480631B041B0C43EA01239BB2038355
:101730007047838B23F004031B041B0C0B43838330
:101740007047838B23F480631B041B0C43EA012343
:101750009BB283837047038B23F080031B041B0C15
:101760000B4303837047038B09025B0441EA534335
:101770009BB203837047838B23F080031B041B0CF5
:101780000B4383837047838B09025B0441EA534315
:101790009BB283837047038C23F002031B041B0C52
:1017A0000B4303847047038C23F008031B041B0CBA
:1017B0000B4303847047038C23F020031B041B0C92
:1017C00043EA01139BB203847047038C23F0800328
:1017D0001B041B0C43EA01139BB203847047038C68
:1017E00023F400731B041B0C43EA01239BB2038404
:1017F0007047038C23F400631B041B0C43EA012392
:101800009BB203847047038C23F400531B041B0C0E
:1018100043EA01339BB20384704710B5048C012363
:101820008B40A4B224EA03030384038C12FA01F16F
:101830000B439BB2038410BD10B5048C04238B4072
:10184000A4B224EA03030384038C12FA01F10B43CC
:101850009BB2038410BD0023012203804380828059
:10186000C38003817047406B7047806B7047C06BCB
:101870007047006C7047038B23F00C031B041B0C98
:101880000383038B9BB20B4303837047038B23F4C7
:1018900040631B041B0C0383038B9BB243EA0123AD
:1018A0009BB203837047F8B50C464988A288B4F808
:1018B00000E02389054600290CBF02270027012AE2
:1018C00014BF01260226BEF1000F10D1FFF72EFC37
:1018D0002846E188FFF7CFFF28463946324623895C
:1018E000FFF73DFCE1882846BDE8F840CEE7FFF76A
:1018F00036FC2846E188FFF7C9FF284639463246BC
:101900002389FFF713FCE1882846BDE8F840B2E7D9
:10191000838B23F00C031B041B0C8383838B9BB2F0
:101920000B4383837047838B23F440631B041B0C9E
:101930008383838B9BB243EA01239BB283837047EB
:10194000F8B50D460B88AA88498804463BB92B890F
:10195000FFF7ECFBE9882046BDE8F8408BE7042B55
:1019600007D12B89FFF7FBFBE9882046BDE8F8404B
:101970008CE7082BB5F808C0078C1DD127F48077B9
:101980003F043F0C0784868B038CB6B29BB226F0D3
:10199000F30623F4206346EA0C1C43EA01211FFAF4
:1019A0008CFC89B24CEA020241F48071828301848A
:1019B000E988BDE8F840ABE727F480573F043F0CC7
:1019C0000784868B038C26F4407623F40053360577
:1019D0005B04360D5B0C46EA022243EA013342EA1D
:1019E0000C329BB2E98892B243F480538283038421
:1019F000BDE8F84097E74A880B8813438A88134369
:101A0000CA8813430A8913434A8913438A891343B3
:101A10009BB2A0F84430704700230380438083804A
:101A2000C3800381438183817047B0F8443029B17A
:101A30006FEA43436FEA53439BB201E05B045B0CE4
:101A4000A0F844307047838819B19BB243F0040377
:101A500003E023F004031B041B0C8380704783887E
:101A600019B19BB243F0010303E023F001031B040F
:101A70001B0C8380704783899BB20AB1194301E034
:101A800023EA01018181704781827047038A1942EC
:101A90000CBF002001207047C94389B20182704702
:101AA000038A828911EA030092B203D011420CBF6B
:101AB000002001207047C94389B2018270470A4360
:101AC000A0F84820704783899BB20AB1194301E00E
:101AD00023EA010181817047838819B19BB243F0E9
:101AE000080303E023F008031B041B0C83807047EA
:101AF000038923F007031B041B0C03817047038930
:101B000023F070031B041B0C0B43038103899BB25E
:101B100043F007030381704738B50D461146012293
:101B2000602D044602D1FFF71AFB01E0FFF7FEFA31
:101B3000238923F070031B041B0C1D43258123897B
:101B40009BB243F00703238138BD038923F0700360
:101B50001B041B0C0B4303817047838823F0700325
:101B60001B041B0C838083889BB20B4383807047CC
:101B7000038923F007031B041B0C038103899BB219
:101B80000B4303817047038923F080031B041B0C64
:101B9000038103899BB20B430381704710B504890D
:101BA000E4B20C43144344EA0324A4B2048110BDFC
:101BB00010B50446FFF7F2FF23899BB243F480433C
:101BC000238110BD10B50446FFF7E8FF238923F0F9
:101BD00077031B041B0C43F07703238110BD70B502
:101BE0000489068B058C26F44076ADB226F00306F8
:101BF00024F00704360425F022052404360C15438E
